:1000000002717D32FFFFFFFFFFFFFF029637FFFF08
:10001000FFFFFF0293BCFFFFFFFFFFC28F32FFFF16
:10002000FFFFFF028537FFFFFFFFFF0204680D4D52
:100030004552435552592D31313520202056657295
:100040003A2031313552553230300D4275696C6489
:100050003A202030332E31322E323030390D0D0D12
:10006000007F01EF1200710FBF090040F6120C74FF
:1000700022C03912071E120738120761F5F078887E
:1000800090549B12BC9A12073812D9BF7600120501
:1000900008C200120761F5F078889054A33000037D
:1000A0009054C412BC9A7600120508200004D200B5
:1000B00080E1120C79D039221204CE9054E512045A
:1000C000E41204CE1200D61204CE74081204A51253
:1000D00004CE120C74227B217988120761FCEB603C
:1000E00011F7090BBB7B027BC0DCF377001205081C
:1000F00080E61207616C60057700120508229054B3
:10010000E51204E41204CE74081204A51204CE22EF
:100110007F0180027F00C202C0A853A882C082C0B3
:100120008312E1FC740A12D8697A0112016FF5F0AA
:1001300012016B45F07001FA908294BA000390822C
:100140009A12A4B7740A12D86912C2761203D14067
:100150000820070260D5BA00D2D083D082D0A83060
:100160000707EA90553A12037BEA22D2008002C2C6
:1001700000C0F07E00EF75F00FA4F5F0E5F09001FF
:100180008273200004C2B18002D2B1D2B0A2B0808A
:100190000F200004C2B18002D2B1D2B3A2B380005A
:1001A000CD33CDDED7743212D869ED300001F4D0F2
:1001B000F02220070690825512A4B712440DFA606F
:1001C0000CB43C028007B43924C2058002D2051267
:1001D00007617B547AF990550130050390550478F6
:1001E0008812043D1205081204CE12030A200704E7
:1001F000EA12036FEA60093007069054F912037B94
:10020000200713120C6F12E16DB411051202188051
:10021000F51203D160F0EA2212DBF679AB12441931
:100220006014B4390C78AB743075F00612D9648060
:100230000512036F800D79AB78BB75F00612DFB342
:1002400012DD1222C0A8C2AFC200754A0075F00AC2
:10025000786B12E11B124C47124CE4124CDD124C2D
:1002600066500280561247EB1249C1124CE4B404A6
:1002700003020306C0E0786B12E103D0E0B43C0750
:10028000786D12E10380D4B4380A3060CE786B12F6
:10029000E08080C770EAEA124D0079AB75F0051274
:1002A0004F344062EA124CF679AD124DE540D179F7
:1002B000AB787375F00212DFB380A07973786F1298
:1002C000035B796F787512D1C37975786F75F00219
:1002D00012CD552000099055211204E41204CEE5F8
:1002E0004A9055126006B4020390551C120320D2A6
:1002F00000054AE54AB40102054AB403005003026E
:10030000024D1204CEE4FAD0A82290829412A4B72F
:10031000120244600A12036F9054F9EA12037B221E
:1003200075F018788812DE6F7892796B1203417835
:1003300097796F120341789C796D12034112050879
:1003400022C8C0E0787912C53F7979D0E0C87C0432
:100350007D0075F002740112A3EE22124CACF60877
:10036000A6F018124D395006760008760018229033
:1003700082A3700390829A12A4B722CAC0E0CAABCB
:1003800083AA82905332700390533A12076178889F
:1003900012043D120508D0E0CA22C082C0839082B8
:1003A000AC12A4B712E16D6433700474338001E4BD
:1003B000D083D0822212E16DB41C04E4D3800BB44C
:1003C0001803C38005B415EDE4C32212C276C360DE
:1003D00014B41C03D3800EB41803C38008B41503EF
:1003E000D38002E4C322B430004006B43A00B340E4
:1003F0000022D322C020C2018004C020D201C2004A
:10040000200011E7200101E3540FC4300103F680FE
:1004100023F28020E7200101E3540FC0F0C0E0E6A2
:10042000200101E2F5F0D0E045F0D0F0300103F614
:100430008001F20809B200D5F0C6D02022F5F0E81C
:10044000C0E0C583CBC583C582CAC58212DE6F8B6F
:10045000838A8212D5B4C5F0CAD0E02AC395F0F8D9
:10046000740112BC9A760022203F19203B07C2CFAC
:10047000C2CEC2AD32C2CFC2CEC2ADC23B120B930E
:1004800053A0F032C0E0C0D0E53A7006C2ADC23F22
:100490008005153A120AC5D2CAC2CFC2CED0D0D07A
:1004A000E032D38001C3C0A875A880C03992E7C0EC
:1004B000E0740712071ED0E0C020D201C206D207A6
:1004C000A2E79204C2E775F007A4F583804DC0A8A7
:1004D00075A880C039740612071EC020D201D2064A
:1004E000C2078037C0A875A880C039C020D201C219
:1004F00006C2078026C0A875A880C039C020D200D7
:10050000C201C206C20780137988C0A875A880C03E
:1005100039C020C200C201C206C207E9C0E0EAC079
:10052000E0ECC0E0EEC0E0EFC0E0C230C237C29005
:1005300012073812071EC202C2B7740312D869121A
:100540000BC6603BB418028003B41702D232C0E07D
:10055000740512D869D0E0C2AD120B9353A0F0C25B
:100560003FC23ED28CD2A912A94C751C00D2308059
:100570000312E16DB417FAC2A9C230D20280B930B9
:100580000211C082C083E9C0E012D387D0E0F9D065
:1005900083D082120B97800280AA120B1940FB12A3
:1005A0000C0160063007F13004EE120761FE7A009C
:1005B000300607C313FA7E0080242007F60A2001C4
:1005C00007E7300005E38002E493B4210050011AEC
:1005D000B420004009200103098001A3DEDF1207D7
:1005E00061C39EF53E120738B40600C2054002D230
:1005F000057A02C2367410120A06C2367F0012074C
:10060000381207447E0230E2011EE53E1209D17520
:100610003F007D00C2031207A3203EFDC2A700D207
:10062000A7200303203FFD120AF5200308D203127E
:100630000751120A150DED8AF0B5F00040D8DECA58
:100640000FEF8583F020070975F00220060375F08F
:1006500007B5F000500280A67408303A0224181240
:100660000A15203FFDE53830E0087401120A152014
:100670003FFD1538120AE5203EFDC2022006222069
:10068000071F30011C1209EDB42000500C6012B499
:100690000D0F200204D20280E374011209D1020579
:1006A00036740212D869E4120CDB751C00D230C912
:1006B000D0E0CFD0E0CED0E0CCD0E0CAD0E0C9D0FE
:1006C00020D039203BFDD2B1D2B0D290D0A822CEDA
:1006D000C0E0CECDC0E0CDC0F08FF084FEE5F0D01C
:1006E000F07D09C5F033C5F033C0F08FF0B5F000F0
:1006F000400295F0D0F0B3DDEAEECDD0E0CDCED023
:10070000E0CE22B4060040027400C453390F4239CF
:1007100022E539C4540FB406004002740022C23CE2
:10072000B40900400274005339F04239120744A260
:10073000E0923CA2E1923922E539540FB40900401D
:100740000274002224018322000001000103000042
:100750000612073824018322060505060608050649
:1007600008120738B4060074184002742022BA0335
:100770000C3005097C0BBD020B7C0A800712076157
:100780008AF084FC22E53F75F01030050375F00C0B
:10079000A422120761C3953F75F01030050375F070
:1007A0000CA42212076E12078512096EE53FB53EB2
:1007B00000400A2CF53F0208C3E40208AB20010701
:1007C000E7300024E380217484200628300717EFE7
:1007D00075F00384E5F06009742423D5F0FC020869
:1007E0006B742402086BE493B4200040C63001030C
:1007F000A3800109C202B4210040BEB48202D20229
:10080000B486004007B4C00040AF24C624E0C083D3
:10081000C082900CE875F007A42582F582E5F035DA
:1008200083F583EF9375F00020053C303C393002AE
:100830000254F8F5F054F0C4241183F583E5F05424
:100840000F240883F5F0F582E583801000030C0F78
:1008500030333C3FC0C3CCCFF0F3FCFFC313C5F033
:10086000134582C5F04583D082D083300507603BB5
:100870001208E98039303C1D300210C313C5F01353
:10088000C5F0C313C5F0134407C5F012092CE5F0F9
:1008900012092C8019300207C5F0120948C5F01260
:1008A00008E9200209E41209488003120965053F9E
:1008B000DC02800F120761F5F0E53FB5F000500350
:1008C0000207AC7410300502740C8CF0A4C082C016
:1008D00083F58285F0831207922582C5F03583C5A2
:1008E000F0D083D08212096E223392B0D2B1C2B15D
:1008F000D2B1C2B13392B0D2B1C2B1D2B1C2B1336E
:1009000092B0D2B1C2B1D2B1C2B13392B0D2B1C2FF
:10091000B1D2B1C2B13392B0D2B1C2B1D2B1C2B1CF
:100920003392B0D2B1C2B1D2B1C2B1223392B0D2FD
:10093000B1C2B13392B0D2B1C2B13392B0D2B1C26E
:10094000B13392B0D2B1C2B13392B0D2B1C2B133ED
:1009500092B0D2B1C2B13392B0D2B1C2B13392B07F
:10096000D2B1C2B1227401C2B0200531801FC0E0F3
:10097000C0F0C2B0540F6007D2B1C2B1D5E0F9D017
:10098000E0C4F5F0D0E054F0C445F06043D2B1C209
:10099000B1D2B1C2B1D2B1C2B1D2B1C2B1D2B1C27F
:1009A000B1D2B1C2B1D2B1C2B1D2B1C2B1D2B1C26F
:1009B000B1D2B1C2B1D2B1C2B1D2B1C2B1D2B1C25F
:1009C000B1D2B1C2B1D2B1C2B1D2B1C2B1D5E0BD22
:1009D00022C3200105C999C9801220060F20070CE7
:1009E000C5829582C582E5839400F58322200108A3
:1009F000E7300001E30980087484200603E493A330
:100A000022EA22741922203FFDD23FD23D20361225
:100A1000753B10800D203FFDD23FC23D203603754F
:100A20003B10C2CAF53AC0F0C23B303602806A754C
:100A3000CD06E54575F002A4C3C53B953BF53B20CB
:100A400037EB120751F5F0120A0384C5F060020576
:100A5000F0120A01A4B53B004002F53B2037CED28C
:100A600036E53C2414F5F0120A01A48FCCC5F0CF72
:100A7000120751CF1206CFAFCCC5F0B53B004002F4
:100A8000F53BE545B4020075F010400375F00CE548
:100A90003BB5F000500385F03B120AA5D0F0D2CA56
:100AA000D2ADD2CF22C0F0C2CAC2CFC2CEE53B7512
:100AB000F05DA4C3C5CC74FF95CCC5CC74FF95F094
:100AC000F5CDD0F0220538533807E538240E83F5EC
:100AD0004044F052A0540F42A0120AA5220C0F036A
:100AE0000B080A020E753B64120AA5753B00D23B47
:100AF000D2CAD2AD22C2A6C28CC28DE53C75F05DD1
:100B0000A4C3C58A74FF958AC58A74FF95F0F58CD5
:100B1000D234D28CD23ED2A922E54575F002A4F59A
:100B2000F0120B83F53CE5F004120B838544F0A42E
:100B3000C5F0CFC0E0CF7F321206CFCFD0E0CFC319
:100B4000E53C95F0F53C120711602114232429831C
:100B5000601A853CF0A4120711142304241A837030
:100B60000585F03C8006E53C25F0F53C303908C3AE
:100B7000E53C13253CF53CC3228000C00000016029
:100B8000019801240183225F0C48083E07C2A62277
:100B9000D2A622D2A622227432D5E0FD3093077469
:100BA000013083027402F54522E430810274013081
:100BB00082027402F54422C020C200C290C2B774FF
:100BC0000312D8698004C020D200C0A8C2AFD2B737
:100BD000740312D86975F001748412096EC2A700FB
:100BE000D2A7200008120C01120B937004120BA95B
:100BF000E4D2B1D2B0200002D290D28CD0A8D020C2
:100C000022D2B775F005E430B703D5E0FAD5F0F697
:100C100075F008A2B733D5F0FA600864FF70E47489
:100C2000188021D28775F008E4308703D5E0FAD523
:100C3000F0F675F008A28733D5F0FA6007B4FFE349
:100C4000800074172290A57D12A4B7783C75F0043B
:100C500074FA12D869D5F0F8D8F3E587D2E1F587B0
:100C600080FE22C0A8C2AF120CC4D28AD0A82275BE
:100C7000F002800875F006800375F001C0A875A821
:100C800080C230C236D237120B977408120A06207F
:100C90003FFD746A120A15203FFDD5F0F5E53830A6
:100CA000E0087401120A15203FFD1538120AE57498
:100CB0000212D869120CDB751C00D230C237203BFF
:100CC000FDD0A822C2AD75C80075CBFF75CAA3229E
:100CD000C28CC28D758C00758A0022C28CC28D7543
:100CE0008CB7758AA8D28C2200000000000000207A
:100CF000707020200020505000000000000050F8CC
:100D000050F850002078807008F020C0C8102040B3
:100D1000981840A0486890986020200000000000CB
:100D20001020404040201040201010102040002093
:100D3000A870A82000002020F8202000000000005B
:100D4000002040000000F80000000000000000004B
:100D50006008081020408080708898A8C8887010AB
:100D6000305010101010708808304080F8708808DB
:100D70003008887018284888F80808F880F00808B3
:100D80008870304080F0888870F80810204040401B
:100D90007088887088887070888878081060000073
:100DA000600000006000006000002040081020404B
:100DB0002010080000F800F8000040201008102063
:100DC0004070880810200020708898A890807020BB
:100DD000508888F88888F08888F08888F070888043
:100DE00080808870F08888888888F0F88080F0801B
:100DF00080F8F88080F0808080708880809888708B
:100E0000888888F88888887020202020207010101A
:100E100010101050208890A0C0A090888080808002
:100E20008080F888D8A8A8A888888888C8A89888C2
:100E30008870888888888870F08888F080808070C2
:100E4000888888A87018F08888F0A09088788080BA
:100E5000700808F0F82020202020208888888888C2
:100E60008870888888888850208888A8A8A8A85072
:100E70008888502050888888885020202020F808B2
:100E800010204080F830202020202030808040201A
:100E9000100808301010101010302050880000008A
:100EA00000000000000000F84020000000000000EA
:100EB0000070087888788080F0888888F000007852
:100EC000808080780808788888887800007088F8A2
:100ED000807010282070202020007088887808708A
:100EE0008080F08888888820002020202020100022
:100EF0001010105020808090A0C0A09020202020B2
:100F00002020300000F0A8A8A8A80000F088888859
:100F100088000070888888700000F088F080800069
:100F20000078887808080000B0C8808080000078C9
:100F3000807008F020207020202810000088888809
:100F4000887000008888885020000088A8A8A850D1
:100F500000008850205088000088887808700000C1
:100F6000F8087080F8102020402020102020202039
:100F70002020204020201020204050A00000000011
:100F8000000000F8888888F800F800F800F800F8F9
:100F90008040204080F83C4494B494443CE01048A5
:100FA000684810E01CE000000000000000000000A5
:100FB000008818284888F88888F88080F08888F0A9
:100FC000F08888F08888F0F88080808080803050B9
:100FD000505050F888F88080F08080F8A8A8A87059
:100FE000A8A8A870880830088870888898A8C88839
:100FF0008820888898A8C8888890A0C0A090881861
:1010000028484848488888D8A8A8A8888888888810
:10101000F888888870888888888870F888888888A0
:101020008888F08888F080808070888080808870D0
:10103000F8202020202020888848301020C02070F0
:10104000A8A8A870208888502050888890909090F8
:1010500090F80888888878080808A8A8A8A8A8A8E8
:10106000F8A8A8A8A8A8F808C04040704848708808
:101070008888E89898E8808080F08888F0708808F0
:101080003808887090A8A8E8A8A890788888782858
:10109000488800007008788878007080F088887030
:1010A0000000F088F088F00000F880808080000068
:1010B000305050F88800007088F880700000A8A8B0
:1010C00070A8A80000F0087008F000008898A8C870
:1010D0008800208898A8C888000090A0C0A0900030
:1010E000003848484888000088D8A8A888000088A8
:1010F00088F88888000070888888700000F88888E0
:1011000088880000F088F0808000007880808078F7
:101110000000F82020202000008888780870002037
:1011200070A8A8702000008850205088000090907F
:101130009090F8000088887808080000A8A8A8A85F
:10114000F80088A8A8A8F8080000C04070487000FF
:10115000008888E898E800008080F088F00000F0BF
:10116000087808F0000090A8E8A890000078887837
:101170002848901D007C0012DFEF755001780112A5
:10118000B538B4AA0A88F0740123D5F0FC42507433
:101190000F12CC9708B806E722901E007C0012DFE1
:1011A000EF7550017801798875F00212DFE57988D2
:1011B000E7B4AA0E09E7600A88F0740123D5F0FCB1
:1011C0004250740E12CC9708B806DB22901E007CA9
:1011D0000012DFEF7550007801798875F01012DF8A
:1011E000E57988E7B4AA187A00EA232489F9E76048
:1011F0000AF5F0740123D5F0FC42500ABA05EA085A
:10120000B806D622C0E0B40600500AF5F0E5500357
:10121000D5F0FCA2E0D0E02275F010A4901E0012E0
:10122000CDE17C0012DFEF22121172754F00D24A1D
:1012300075320012133C12C27660FBB43A1312CF1F
:101240009BB407051214AF80E5B40903122319807B
:10125000DD12DA595041B4060050DB121204400589
:1012600012C7FA80D1F5F0E532232411F8E5F060D9
:1012700003F2800B7403C3953223F5F012E08978F2
:1012800011E2600274AA18F2791075F01012DFC72B
:1012900074F012CC97809CB41718E532232411F80F
:1012A000E260090532E532B4030040037532000202
:1012B0001233B4130CE54FB404005002054F021270
:1012C0002EB4120CE54F700302122E154F02122E8F
:1012D000B41125E532601E232411F8E260171213C1
:1012E000904012781074AAF2791075F01012DFC7CE
:1012F00074F012CC97021233B41502741CB41C02A1
:101300008003021233027065C0E012DBF6D0E0F514
:10131000F0E5326023FA7901E9F8E5F003D8FDA29F
:10132000E07B3050027B31C0F0E975F002A4D0F0D0
:1013300024BBF8EBF609DAE012DD1222304A23E58D
:101340004F121218791075F01012DFDB74F012CC06
:1013500097C24A7810E264AA6008781075F01012FB
:10136000E08912DBF678BBE54F2441D2E7F678BE80
:10137000791175F003E32430F608080909D5F0F572
:10138000E53275F002A424BDF8743DF612DD122298
:10139000753301853234E532232412F8E2F534E561
:1013A00034121308E53375F002A424BAF8763D121E
:1013B000DD1212C27660FB12DA595027B4020050D7
:1013C000F15401A2E0400244FE8533F023D5F0FC45
:1013D0004004523480024234E533B5320050C00537
:1013E0003380BCB4180CE532232412F8E534F2C380
:1013F0008004B41CBDD322C0E0907D2E788875F0A7
:101400001812DE6FD0E02441788CF608743AF67832
:1014100010E264AA700D781175F003E270150808E7
:10142000D5F0F8907DD9789475F00C12BC9A12051D
:1014300008807B1205087E00907DFB788875F01887
:1014400012DE6FEE24317892F6907DC9789675F0B1
:101450000512BC9AEE232411F8E2C0E0600A2430A1
:10146000799CF708E2FC800A789475F00C742D12D0
:10147000E123120508D0E06031EE602E907E0978FD
:101480008875F01812DE6F7996EEFA7B01C2D5EB03
:10149000F8EC03D8FD30E009D2D5EB2430F7090988
:1014A000090BDAEB30D5031205080EBE038A2212AF
:1014B000B762907DE61204E4120C797F00E4121208
:1014C00018791075F01012DFDBEF1213F7120C7998
:1014D0000FBF05ED786B12C98B786E12D2DE12D178
:1014E000072275F010A4901D0012CDE17C0012DFE0
:1014F000EF221211CC754F00D24A753200121572CC
:1015000012D61D60FBB43A1612C27612CF9BB407F6
:10151000051217DC80E2B409E412231980DA12DA2A
:1015200059403012C276B4170E0532E532B40400C9
:10153000400375320080C6B4130BE54FB40400506D
:1015400002054F80B3B41208E54F60AC154F80A878
:10155000B4110F7810E264AA600375320112164CC0
:10156000809B00B41502741CB41C028002808E02A1
:101570007065304A14E54F1214E2791075F01012BC
:10158000DFDB74F012CC97C24A7810E264AA6024C0
:1015900012DBF6E54F2431D2E778BBF6907C107869
:1015A000BE75F00512BC9A12DD12781075F010129B
:1015B000E08980239015D4C082C083E532B4040052
:1015C0004001E42390163C12CDE1740193C0E0E4A5
:1015D00093C0E02212DD122212DBF6E54F2431D255
:1015E000E778BBF67811E2243078BDF678BE791240
:1015F0007C047D0275F002740112DD42742578C20C
:10160000F622907BDA12E12B781475F00C1219FF98
:1016100078C1121C2622907C1F12E12B78BF791210
:101620007C047D0275F002740112DD4222907C1769
:1016300012E12B79C27811E22430F72215D8160274
:10164000162D161616AB16B0174916EC90166CC070
:1016500082C083E532B404004001E42390164412B2
:10166000CDE1740193C0E0E493C0E022403C7810E7
:10167000E2B4AA29781475F00C1219FF70107814CE
:10168000907DC975F00C12DE64E54F2431F27812BA
:1016900075F00212E053700578137401F279107539
:1016A000F01012DFC774F012CC972212C276D32248
:1016B0007879791475F00C12DFB3787975F00C1223
:1016C00019FB787975F00C121C52401EC0F0E5F041
:1016D00078146005797912DFA9D0E0B40C005002CB
:1016E000E4F2781074AAF2C38001D322907C1F1216
:1016F000E12B796B7B027C037D057E047F02E4E4B1
:10170000128E34B41841786B12DA99786B75F00246
:1017100012E05C7016E54F04121204500E907BA389
:1017200012A4B712C7FA12E16D801C7812796B759A
:10173000F00212DFA9781275F00212E05360027411
:10174000AA7810F2C38001D322907C1775330175FB
:101750003400121A2C400B7811F2781074AAF2C3DC
:101760008001D322C0E0907DC9788875F01812DE20
:101770006FD0E02431788EF608743AF67810E2647F
:10178000AA6005907DD9800D781475F00C1219FFB0
:10179000700D907D50789275F00E12DE6F800A7891
:1017A00092791475F00C1219EB1205087810E264A6
:1017B000AA7028788812DCE07811E2907DCF60036F
:1017C000907DD4789179127C0E7D0275F0027401BF
:1017D00012DD4E7425789FF61205082212B762902A
:1017E0007DB61204E4120C791217FC120C79786B96
:1017F00012C98B786E12D2DE12D107227F00E4125A
:1018000014E2791075F01012DFDBEF1217640FBFCE
:1018100005F02275F000B4A30375F001B4A80375B8
:10182000F001B4AD0375F001E5F022C2AC85124CB5
:1018300085134D85144E12DF0912193270030219F7
:101840002678A375F02012E089C24C75320012DFB1
:101850000912E00B12DFEF12B53864AA6003021917
:101860002412B538F516121813605AE532121971A0
:101870007053798875F00312DFE5742112CC9779E3
:101880008B75F00512DFE5204C17786B75F00812A8
:10189000E11B796BE516F7786C798975F00212CD4A
:1018A00055786C798975F0021219C67018E51678AA
:1018B0006E798BB4A80512DDAE800312BA72D24CD9
:1018C000E53212198AE51664CA6016E51612BB2BBA
:1018D0006052040412D5EA12BEB205325003021857
:1018E00051304C3D786F796C75F00212DFA9786F3A
:1018F000C2481224E54027743612CC9775F005795A
:101900008812DFE574FB12CC97796BE77888796EE3
:10191000B4A30B12BA7275F005798812DFD10218E0
:1019200049E480027455854C12854D13854E14D2BE
:10193000AC2275320012E00B12DFEF12B53864AA48
:10194000702C12B538F516B4B60050020532B4CC7E
:1019500002801BE51664CA6011E51612BB2B600EEF
:10196000040412D5EA12BEB240CBE5328002740004
:101970002275F0088424A3F8E2C5F06008C5F003DE
:10198000D5F0FC8002E5F054012275F0088424A310
:10199000F8E2C0E07401C5F06008C5F023D5F0FCA2
:1019A0008002E5F0D0F045F0F222784675F00A1298
:1019B000E0536011907BC412A4B712C7FA12C2762A
:1019C00012E16D740422E76670050809D5F0F7226C
:1019D000E36670050809D5F0F722E62401D4F6087D
:1019E000E63400D4F61822C2D58002D2D5E730D52D
:1019F00001E36006F60809D5F0F322C2D58002D2D1
:101A0000D5C0F0E8C0E0E630D501E2600408D5F0CA
:101A1000F5C3D0E0F8D0E095F022E608F61818D526
:101A2000F0F822E618F60808D5F0F82212E12B8526
:101A3000344C053378C2E54C2430F612DD1212C264
:101A40007660FB12DA59500EB5340040F1B5330020
:101A500050ECF54C80DEB41805E54CC38009B41594
:101A600002741CB41CD8D322C0E0C395F05004D03B
:101A7000F08002D0E022C0E025F02814F9E5F0283B
:101A800014F8E6F71819D5F0F9D0E0F5F0C9C399C4
:101A900004F8742012E12322884BFEAFF028F8EE00
:101AA000C5F0C395F06005F5F012E11B8009884B85
:101AB00012E11B7E00AFF0EEFA6F70011A7B00C2DC
:101AC0005212DBF6EE12D79478BB12D9BF78BCE67F
:101AD0004480F6EA0412D79478BD12D9BFE54B2AA8
:101AE000F8E6600578C0121C2678BF763D12DD123C
:101AF00012C27660FBB415187B00C252EED370039D
:101B0000021C07A84B8FF012E11B7E007A0080B107
:101B1000B41C4230520CE54B2AF876007B00C252CE
:101B2000809FEED37003021C07EA6E601CC3EE9A1E
:101B3000F5F0EF6E700215F0EA254B04F8E5F06061
:101B400003121A231876008008E54B2E14F876004D
:101B50001A1E021AC1B4131E8AF0EE6F700205F04D
:101B6000C3EE95F0608A305205121C0840050A7BCE
:101B700000C252021AC1B41216EA7003021AF030FF
:101B80005205121C0840051A7B00C252021AC1B449
:101B9000181530520D121C085003021AC1EA6E705B
:101BA000010E8EF0C38060B41727EA254BF8E612C9
:101BB0001C17500612C7FA021AC1D3EE9A5005EE4E
:101BC0006F60010EEF146A60010A7B00C252021AB4
:101BD000C112DA594003021AF0B40A004003021A93
:101BE000F0C0E0EA254BF8E6BB0001E475F00AA47A
:101BF000D0F025F0F60BB41A005005BB03004002EC
:101C00007B00D252021AC122E54B2AF8E6121C17B9
:101C1000500512C7FAD322B420004009B47B00B3A8
:101C20005003B4C00022C0E0C2D575F064846006E1
:101C30002430F608D2D5E5F075F00A84700330D56B
:101C4000042430F608E5F02430F608D0E022121A19
:101C5000AE22121A9822C0E0E51790050160139099
:101C60000401B40102800BB40205902100800390AE
:101C70002180D0E012CDE17C0012DFEF22C256E5D8
:101C80001790050060039004007C0012DFEF12B58E
:101C900038B409004001E4F53274FF12CC97907C0F
:101CA0002412E12B78C2E5322430F612DD1212C282
:101CB0007660FBB43A1312CF9BB408051200618022
:101CC000EDB409EA12231980E512DA59500BB40970
:101CD0000050DBF532D25680CBB41805A256B38043
:101CE0000AB41502741C641C70C4D3E53222751743
:101CF000038021751702801C75170080037517017A
:101D0000121C7D4005E53212B9B6120738F54CE5D4
:101D10003212071E753200E53275F020A4121C56EF
:101D2000797975F02012DFE5E517907C3960139022
:101D30007C32B40102800BB40205908303800390CF
:101D4000830B12E12B78BD762D08907C2A75F00369
:101D500012BC9AE532243178BFF608743DF67879E2
:101D6000121E7D1219FB12D79478C112D9BF12DD51
:101D70001212C27660FBB4113D7879121E7D1219E1
:101D8000FBC0E0121E7DD0E07879121C524088C062
:101D9000F0121E7DD0E0B5F00050052479F8E4F68D
:101DA000E53275F020A4121C56797975F02012DF07
:101DB000D1D256021D17B4200A787975F02012E1AD
:101DC0001B80DDB41209E53260A71532021D17B47D
:101DD000131CE51775F005B402028003B403037504
:101DE000F003E532B5F00050020532021D17B43A97
:101DF0001912CF9BB40708121E21120C748006B46E
:101E00000903122319C256021D17B41502741C646B
:101E10001C6002A171305606121E21120C74027051
:101E200065788812DCE0788DE517907C9A601390D5
:101E30007C86B40102800BB402059052E4800390CA
:101E400052F81204E4120C79E4121C567F06E517CE
:101E50006007B4010280027F04797975F02012DFF7
:101E6000E57879121E7D1219FB700A7879121E7DB1
:101E7000742D12E123797912050ADFDD22E517249A
:101E80000383F5F02220201412121199754F00D20D
:101E90004A753200121EFF12D61D60FBB43A1612AC
:101EA000C27612CF9BB4070512217780E2B409DF16
:101EB00012231980DA12DA59403012C276B4170EA2
:101EC0000532E532B40500400375320080C6B41314
:101ED0000BE54FB403005002054F80B3B41208E580
:101EE0004F60AC154F80A8B41105121FFE80A500ED
:101EF000B41502741CB41C02800280980270653014
:101F00004A27901F00E54F75F020A42582F582E551
:101F1000F03583F5837C0012DFEF791075F0201225
:101F2000DFDB74E012CC97C24A7810E2C394A0B40D
:101F300003004008781075F02012E089901F5CC003
:101F400082C083E532B405004001E423901FEA1209
:101F5000CDE1740193C0E0E493C0E02212DD1222CF
:101F600012DBF6E54F0478BB121C26742EF67810AF
:101F7000E2B4A105907B8F800BB4A205907B968084
:101F800003907C4D78BD75F00612BC9A22907C447B
:101F900012E12B79C27810E2C394A0B4030040018F
:101FA000E42430F722907BDA12E12B781175F016D9
:101FB0001219FF78C1121C2622907BE312E12B79C3
:101FC000C2782AE27004243080022440F72278BBD1
:101FD000792B7C087D0275F005740912DD42907C36
:101FE0004B78BB75F00312BC9A221F601F8D1FA592
:101FF0001FB91FCE2038203D2055208F20AD9020C6
:102000001EC082C083E532B405004001E423901F66
:10201000F412CDE1740193C0E0E493C0E0224017D4
:102020007910E354F064A0600374A0F375F02012FB
:10203000DFC774E012CC972212C276D322907C4480
:10204000753302753400121A2C400824A07810F25F
:10205000C38001D3227879791175F02012DFB3782B
:102060007975F0161219FB787975F016121C52402A
:1020700019C0F0E5F078116005797912DFA9D0E098
:10208000B416005002E4F2C38001D32212C7FA90C2
:102090007BE3753305753400121A2C400B121204C1
:1020A00050EA782AF2C38001D32212C7FA786B75FE
:1020B000F00512E11B907C4B12E12B786B75F0055B
:1020C00012E11B796B7B027C007D087E077F02E4B6
:1020D000128E34B41811786B12DA99786B782B79E8
:1020E0006B12E1ACC38001D322C0E0907D377888C9
:1020F00075F01812DE6F788E7420F608D0E00412A6
:102100001C26743AF67810E2B4A105907C78800C15
:10211000B4A205907C7F8004907C70E4C0E0789944
:1021200075F00712BC9A120508D0E0604978117565
:10213000F0161219FF7008907D501204E4800579A2
:10214000111204F5907D2E788875F01812DE6F79E3
:102150009F782AE27004243080022440F712050898
:10216000907C697888792B7C187D0275F005740164
:1021700012DD4E12050822907C541204E4120C79F0
:10218000901F007C0012DFEF7F00791075F02012A5
:10219000DFDBEF1220E9120C790FBF04ED120C7493
:1021A00022B404005005907CB58023B40405907CD3
:1021B000C4801BB40505907CBC8013B40705907CDB
:1021C000CC800BB40605907CD88003907CE92290EB
:1021D00020007C0012DFEF791075F02A12DFDB752A
:1021E000320012DBF6E5320478BB121C2618E644F6
:1021F00080F6E53275F006A42410F978BD75F00676
:102200001219EB12DD1212D61D60FBB43A1112C284
:102210007612CF9BB407061222AD120C7480C31243
:10222000DA59400612C276B41155788812E092B499
:1022300018B0E532B4040050227E00EE75F006A41A
:102240002410F9788875F0061219D0700AE5326EFC
:10225000600512C7FA80D30EBE04E0E53275F006C1
:10226000A42410F8798875F00612DFA99020007C6C
:102270000012DFEF791075F02A12DFC70221E2B4F5
:102280001209E532608015320221E2B4130CE53206
:10229000B40600500205320221E200B41502741C9B
:1022A000641C600302220612E13302706578881212
:1022B000DCE07891907CAE75F00F12BC9A120508A4
:1022C000120C799020007C0012DFEF7F00EF1221CA
:1022D000A1788875F01812DE6FEFB40400788F5083
:1022E00004EF2431F67898742DF6799A75F0061279
:1022F000DFE5789A75F0061219FB700A789A75F086
:1023000006742D12E1231205080FBF07C0226008D2
:10231000F608762D08121C2622907E171204E4126D
:102320000C797A207B477C6E7EDA788812DCE0EAD2
:10233000788812230E0AEB788E12230E0BEC789419
:1023400012230E0CBC7B027CC0EE789B12230E0E77
:10235000120508BE01D4120C74229000007C00E526
:102360002254037012E5822400F582E5833464F57B
:1023700083EC3400FC8025B40112E5822400F58250
:10238000E583347EF583EC3400FC8010E582240084
:10239000F582E58334EDF583EC3400FC12DFEF22A7
:1023A000787A75F00212E089E5225403700B787A8E
:1023B0007465F2087400F2801CB4010B787A74F52D
:1023C000F2087401F2800EB403005009787A74E9BF
:1023D000F2087403F222787AC3854FF0E2C5F095D3
:1023E000F0088550F0E2C5F095F0B322784F797887
:1023F00075F00212DFB3227878794F75F00212DFA0
:10240000A922C2488002D2487888204802788A757A
:10241000F00220500512CD55800312DFB33048077B
:10242000788A798812D1C3788A12E080E6F582082A
:10243000E6F583744012D561FC12235F2212235A01
:1024400074C012CC9780077978D250122402907B06
:10245000CD12A4B71223EC740112CC97784F12E17D
:10246000031223D64014743F12CC9712B538B54AE4
:10247000EB1223F774FF12CC97C322907BCD12A4EA
:10248000B77978D2501224021223EC740112CC973F
:10249000784F12E17B601E12E08012E17B601674BF
:1024A000BF12CC9712B538B54AE61223F774FF1263
:1024B000CC97C38001D32212235A784F75F00212B1
:1024C000E11B1223A0784F12E10312B53854F0B487
:1024D000A00C743F12CC971223D650E9800674FFEB
:1024E00012CC97C322884B1223A020482F7888A9AA
:1024F0004B75F00212DFB3784F798812D1C31223E3
:10250000D64018A94BD25012240612B53854F0B454
:10251000A00874FF12CC97C38001D32212235A78EB
:102520004F75F00212E11B784F12E10312B53854D7
:10253000F0B4A025742B12CC97798875F00912DFBE
:10254000E57888A94B75F0091219D0700874CB1280
:10255000CC97C3800E740B8002743F12CC97122369
:10256000D650C422784675F00A12E0897810E54A00
:10257000F27912D250122406791075F04012DFC79A
:10258000221224E54009E412B9B674FF12CC972256
:10259000788875F020742012E12322122590788823
:1025A00079127C047D0075F002740312DD5AE54A4D
:1025B000B4AA31783C75F00912E0536013907D3F66
:1025C000788D793C7C157D0075F009740B12DD4E19
:1025D0007811E2907D4830E003907D4C78A375F04F
:1025E0000312BC9A7811E230E10478A776581205FC
:1025F000082212259B781575F0201219FF7008909B
:102600007D501204E4800579151204F5122590908E
:102610007D31788879357C107D0275F00574011262
:10262000DD4E907D37789A75F00712BC9A793BE3BE
:10263000121C26907D2E78A475F00212BC9A763A70
:1026400079A7783AE27004243080022440F712051A
:10265000082212259B781575F0201219FF7008903A
:102660007D501204E4800579151204F5122590902E
:102670007DAC788879467C147D0375F00574011271
:10268000DD4E1205082212B762120738F54C74119C
:1026900012AC2612071E907D05E54AB4AA03907C71
:1026A000EE1204E4791012E14A791075150012C691
:1026B000091223A012235A784F75F00212E11BC2AF
:1026C00048784F12E1031223D6401E12B538B54A9E
:1026D00011791175F03512DFDB1225F2D248740A38
:1026E0008002743F12CC9780D8204809907D1B123D
:1026F00004E412C7FA120C79E54C12071E12259059
:10270000786B12C98B786E12D2DE12D10779101253
:10271000E14A791012E15112E13322754AA5D255EE
:102720008013754AA5C255800C754AAAD2558005FA
:10273000754AAAC255C2AC78F1E26402600F907B80
:10274000AC12A4B712C7FA12E16D027065C2491249
:10275000B762120738F54C741012AC2612071E909F
:102760007D5F788875F01812DE6F907D74E54AB44D
:10277000AA03907D69789275F01812BC9A12050828
:10278000305506907D7F1204E4791012E14A7910E9
:1027900075150012C609741112AC2612071E1223F9
:1027A000A012235A784F75F00212E11B784F12E104
:1027B000031223D6402612B538B54A19791175F09F
:1027C0003F12DFDB784675F00A12E05360DE122616
:1027D00052D24980D7743F12CC9780D0204903024F
:1027E000284720550302284D7989E54AF709E54C29
:1027F000F77988741FF712DC1D1223A012235A7870
:102800004F75F00212E11B784F12E1031223D640FC
:102810003C12B538B54A29791175F03F12DFDB78E3
:102820004675F00A12E05360DE784675F00A12E051
:102830008974F612CC97794675F00A12DFC780C703
:10284000743F12CC9780C0907D911204E4120C79F1
:10285000E54C12071E122590786B12C98B786E1208
:10286000D2DE12D107791012E14A791012E1511229
:10287000E13312C4B4742512AC267003027065E50E
:102880003104F53012C3E1547FC52F5480452FF534
:102890002F027065E54AB4AA16E532B40800400379
:1028A000753200E5326405D2456002C2458011B43C
:1028B000A50BE532B405E27407F53280DCB4A00064
:1028C00022754AA58003754AAA78F1E26402600F76
:1028D000907BAC12A4B712C7FA12E16D022A70D233
:1028E00047D2AC785075F01012E089787875F00214
:1028F00012E0891223A012243DB39249D24A7532C4
:1029000000122A7512C27660FBB43A2E12CF9BB425
:102910000503022944B40603022974B407142049AC
:102920000512C7FA80DB1226867978D2501224026B
:1029300080CAB409C712231980C2B41767053212BE
:10294000289480BD122D307009D24974C012CC97E2
:1029500080AAC0E07978D250122402D0E0B40202FA
:10296000809A12C7FAB40194907BBB12A4B712E10B
:102970006D0228FC30493E1219AA60030229049016
:102980007C00753301753400121A2C40027003026A
:102990002901122586122447500712247B5002C2B7
:1029A000490228FCB4111020490512C27680061293
:1029B0002BD60229018057B4145A3049F8907BD5A0
:1029C00012E12B796B7B027C047D047E04E54AB422
:1029D000AA027E127F00E4128E34B4182E75F00223
:1029E000E54AB4AA0375F009786B12DF77601CC260
:1029F00048B405004002D248786F796B75F009122F
:102A0000DFA9786F1224E5D24A40250228FC12C7BC
:102A1000FA022901B4120B3049F412247B4011024E
:102A200028FCB413143049E612244740030228FC62
:102A30007978D25012240280D5B42C253049CF1297
:102A40000738F54C741112AC2612071E1225F2122B
:102A50000C74E54C12071E7978D250122402022918
:102A60000400B415028009B41C030228FC022901E9
:102A7000C245027065204908907BB512A4B780500A
:102A8000304A2A791075F04012DFDB74C012CC97FF
:102A9000C24A786B791275F00212DFB3786D796BE8
:102AA00012D1C37878796D75F00212DFA9902ACD22
:102AB000C082C083E532B409004001E423902BB208
:102AC00012CDE1740193C0E0E493C0E02212DD1264
:102AD0002212DBF678BB79127C047D0075F002745B
:102AE0000212DD42783AE2700424308002244078F9
:102AF000C0F6E54AB4AA0A7811E25401243078C13C
:102B0000F67811E2035401243078C2F622907BDA81
:102B100012E12B781575F0201219FF78C1121C26CE
:102B20002278BB79357C087D0275F005740912DDC9
:102B300042907BE078BB75F00112BC9A22907BE357
:102B400012E12B79C2783AE27004243080022440EA
:102B5000F722907BE712E12B78C2793BE3B40A00BD
:102B600050052430F6800418121C262278BB793CCC
:102B70007C087D0075F009740912DD42907BEB78CA
:102B8000BB75F00412BC9A22907BF012E12B7811F5
:102B9000E2A2E074305002743178C2F622907BF8E1
:102BA00012E12B7811E2A2E174305002743178C244
:102BB000F6222AD12B0D2B212B3D2B522B6C2B884F
:102BC0002B9D2AD12C062C542C932C392CCF2C0B3A
:102BD0002CFA2D152C06902BF6C082C083E532B45A
:102BE00009004001E423902BC412CDE1740193C08D
:102BF000E0E493C0E022400D791075F03612DFC793
:102C000074CA12CC972212C276D322907BEB12E1C7
:102C10002B796B7B027C037D057E127F00E4128E94
:102C200034B4180280046414700D783C796B75F02C
:102C30000912DFA9C38001D3221219AA7014907B54
:102C4000E3753305753400121A2C4006783AF2C346
:102C50008001D3221219AA70357879791575F02080
:102C600012DFB3787975F0201219FB787975F020AE
:102C7000121C524019C0F0E5F07815600579791200
:102C8000DFA9D0E0B420005002E4F2C38001D322D7
:102C900012C7FA907BE012E12B786B75F00612E117
:102CA0001B796B7B027C017D077E087F02E4128E1C
:102CB00034B41816786B12DA99786B12D3C760D0D7
:102CC0007835796B12E1ACC38001D32212C7FA9038
:102CD0007BE712E12B796B7B027C057D037E027F13
:102CE00000E4128E34B41810E56B12D7AAB40500B4
:102CF00050DA783BF2C38001D322907BF075330128
:102D0000753400121A2C400BA2E07811E292E0F226
:102D1000C38001D322907BF8753301753400121AF9
:102D20002C400BA2E07811E292E1F2C38001D322A1
:102D30001224B75003022DCB781075F04012E089B1
:102D4000786B794F12C53F907BD512E12B796B7B65
:102D5000027C047D047E04E54AB4AA027E047F005E
:102D6000E412DE01B41868784F796B12D1C3784F42
:102D700012E17B60051223D6500512C7FA80C17894
:102D80006BC25012240612B53854F0B4A010907CD7
:102D900008753301753400121A2C40946092781231
:102DA000796B75F00212DFA9122C54122C93122C9D
:102DB00039122CCFE54AB4AA0AD245122C0BC245CF
:102DC000122CFA122D1512256480067401800274EB
:102DD0000222CAEEEDF2F0EEEBEBE5F020D4CF00EC
:102DE00012DEF590FFF0790075F040124F34500379
:102DF000022E497902902DD2E493600CF5F0E3B5F0
:102E0000F004A30980F280317A0079027888E360C7
:102E10000AB40D028005F6080980F37600098933AB
:102E2000120508A9330ABA020040E17900E36402FE
:102E300060059058B5800B80F99058D71204E4E4EF
:102E4000800E1204E474018007740412A94C74010A
:102E500022E5227B587AE39058F660099058FAB43C
:102E600002039058FE120761788812043D1205088B
:102E7000227A0080027A8012039A6050EAC0E0123F
:102E80002ECFCAD0E0CA40376401600B90590312BC
:102E900004E4120C6F803590829412A4B778007409
:102EA000FF75F04012D9649000007B0475F0407902
:102EB00000124EAB74044007DBF2DAEE0271DA1254
:102EC000A94C1203D1400570031203B5027065C00E
:102ED000A8C2AFC2078002802E7FFF90FFF079006A
:102EE00075F040124F3440EF7902902DD2E4936098
:102EF0000AF5F0E3B5F008A30980F2C3E4800A9074
:102F00005903C3740180027404D0A822D24712E18D
:102F10003B7808E516F212D366780975F00412E0E2
:102F2000897523005324F0740102832A754A0279BB
:102F300083124A8F70157885E2C3940008E29420CA
:102F400040047433800512B61D600612A94C02704D
:102F500065740D12AC2612071EC2259020807C00DD
:102F600012DFEF798875F00D12DFE5788875F003D0
:102F700012E05C7003022FFD786B798875F0031204
:102F8000CD55786E12C98B12D50D4017E5727004BD
:102F9000E5716003022FFD9055B71204E475F00748
:102FA000120C7CD225788BE67003022FFD12A94CFF
:102FB000B4110A789275F00312E05C700302706538
:102FC000787912B3D5641870F47879798C75F00635
:102FD000E66770E90809D5F0F77888799275F0030B
:102FE00012CD55789275F00312E11B9020807C0081
:102FF00012DFEF798875F00D12DFD1C225C21E7481
:103000000712AC266002D21EC21C740812AC2660E5
:1030100002D21CC21B740512AC266002D21BC21D58
:10302000742612AC266002D21D12DFF912DBDCE43A
:10303000F532F516F51712DBF612DAC975F005123E
:103040000C7CC226D22702424B12C7FA12DBF612C0
:10305000DAC912DD12C247D2ACD2A9D2AAD2AFD2FB
:103060004512D61D60FBC0E078F1E2B4031BD0E04E
:1030700012C276B49A03023110B415E5782FE270CB
:1030800003026D5112C7FA80D8D0E0B43A0280082A
:1030900012DA59500302337012C276B41503023E9D
:1030A000BCB41C03023AAEB41303023B3EB4120399
:1030B000023B42B41403023E88B49903023E88B432
:1030C0001903023E8DB42003023EC4B41703023E2E
:1030D000D2B41803024004B42C030242E5B42B031B
:1030E000023F43B41103023A7DB4211E78BBE6B41B
:1030F000631B12DBF6791DE378BB12D042766312B4
:10310000DD1212C27660FB023A2D12C7FA0230615C
:10311000C2AC7881E2B40203023165B40403023127
:1031200091B40503023200B4060302323AB4070335
:10313000023259B408030232EAB40D028003B40E1D
:103140000778827402F2800578827401F278007444
:1031500080F278017403F212C86F12C7FA12DBF61C
:10316000D2AC02304F7882E26007B4010474008070
:1031700007782FE2600774087882F280D07882E4C2
:10318000F278007480F278017403F212C86F026D55
:10319000517883E2B4A3028017B4A5028012B4ADC3
:1031A00002800DB4AE02800874037882F202314DC1
:1031B000E51512D4F16004741680EF782FE2B4C8DC
:1031C000004004741580E378A812E06560DA78B0F6
:1031D00012E06560D378AEE26005B4050040047487
:1031E0001A80C7781279B075F00512DE597883E23B
:1031F000B4AD028003B4AE057402782EF2023674C8
:10320000782FE2B4FB005006700874168004741521
:1032100080157882E2B4C4057517128010B4C50514
:10322000751713800874167882F202314D787B7915
:103230008475F00712DFB3023AFC782FE270047451
:103240001680E478CE75F01412E08978CE7420F2FE
:10325000087418F208F20230987882E2B402028010
:10326000534059B40500504C788375F00712E05371
:10327000700474038040786B798375F00712DFB3B4
:10328000E56F7008E5707004E571600474158026C0
:10329000782FE260047416801D7882E2B40309740A
:1032A00003782EF2741380077404782EF27412F5EA
:1032B00017023E3474037882F202314D782FE270A7
:1032C00004741680F17882E2600675160402402FBD
:1032D000788375F00712E053700675160002402FD0
:1032E000786B798312DFB302341B12BCF54008748B
:1032F000187882F202314D782FE26004740880F170
:10330000201904741680EA12CB056004741680E15B
:1033100002433E12A94C782EE2B400028003B401AD
:103320001512DBDCC223C221C220E515B405005012
:1033300003751500801512DBDC12DBCF12DFF9C23A
:103340002375150012DA06C247D2AC12DBF6023042
:103350004F78F1E2B4030874157882F202314D74AB
:103360002412A94C12DBDC12DBF675150002304F7B
:10337000C24812DBF6786B75F00A12E11B301B1A9B
:1033800012C27612DA596005B40A004005741A02B6
:103390003313786BF67A010234817C007D087E124B
:1033A0007F03796B7B017414301C047F02D2E3121B
:1033B0008E34B41B02742EB4171E301E0474418068
:1033C0001D740212AC266009B4050050042440802C
:1033D0000D12B4C55002741CB41C03023316F51749
:1033E000BA0003023316B41802800302346EE515E6
:1033F000B400028017B402028012B40302800DB43C
:1034000004028008B405028003023049BB03004077
:10341000030230497F02786B12DAA9782FE2700537
:10342000741A0233137827796B12E1A612AABE78B8
:103430006B792712E1B2786B793012DA89601B5010
:103440001978F1E2B4030874197882F202314D74EC
:103450002F12A94C12DBF602304FC2AC781174C0A7
:10346000F27827796B12E1A6751600024033B41189
:103470000DE51512D6C970030234E0023049B414C8
:103480000FE51512D4F17005C22002352302304930
:10349000B412028003B41311E515B40403023AB662
:1034A000B40503023AB6023049B42E17301D02802B
:1034B00021782EE2B40102800FB40002800A741A4F
:1034C00002331312DA69500AE51512D4F1700302BF
:1034D000377112C7FA12C27660FBB41CF5023316BC
:1034E000BA0A005014BB0400500F786B301C027FE6
:1034F0000312DA99786FE6600302335112BCF5408B
:1035000005742302331312DBDC7812796B12E1AC01
:1035100075150112DBF612DAC978BB7459F6D24779
:10352000023052BA0008742D12A94C02336412BC46
:10353000F540057423023313204816BA0700500FD4
:1035400078F1E2B40205BA050050DBC2488002D22D
:1035500048792EE3B4020C742012AC266005741D69
:10356000023313E51512D6C9700312DBDC781E791D
:103570006B75F00912DFA978F1E27005741A023355
:1035800013C2ACB401028003023633C2AC7880753A
:10359000F01212E089792EE3B4020474AD80027453
:1035A000A37982F309782FE2F3097884791E75F004
:1035B0000912DE59788D791212E1A075F0043048B5
:1035C0000375F005740312E0B378007480F278019B
:1035D0007412F2C0A875A88812AED6400512B0AE1B
:1035E0005012D0A8B42A028002742B12A94CB41C29
:1035F000E2023316D0A87982E36011B4130812C630
:103600004C742B02331312D3A7023313781212E037
:10361000656014781279B075F00512DCD370025031
:103620000DC0A8742980BB781279B012E1A078AFE0
:10363000E28026781E1224E55005742E023313C250
:10364000AC798375F04012DFDBC2207983E3B4A547
:1036500002D22074A3F37984E330E10574280233A5
:103660001330E0107812E2700608E2540F6005741F
:103670002902331378ADE260261475F010901E0015
:1036800012DAB97C0012DFEF12B53864AA60107844
:10369000F1E2B4030574050231AA7431023313D286
:1036A00021781E798575F00312DE59781779A8758F
:1036B000F00712DE59781775F00512E05360030227
:1036C0003703786B75F00512E11B78BB76D57C016A
:1036D0007D077E0A7F02796B7B017414301C047FA6
:1036E00002D2E3128E34B41703BA000612C7FA02EC
:1036F00033167F02786B12DA997817796B75F005BB
:1037000012DFA9781DE26011B4050040057425029E
:1037100033132440F5170237D990814B75F00878A0
:10372000BB12DE6F12DD1212D61D60FBB4171F1222
:10373000C276301E0474418010740212AC26602CD4
:10374000B40500400280252440F5170237D912DA6B
:1037500059500B12DD1E50028012F517807B12C2E9
:1037600076B4210280EDB41C0302331612C7FA802E
:10377000A8BA0A004003023351BB030040030234DD
:10378000D212BCF5400574230233137F02786B120A
:10379000DA99786FE654F0600302335178F1E26011
:1037A00025782EE2B400028011B40102800CB4022C
:1037B00015742012AC266009800C741F12AC2670A0
:1037C00005741A023313C2ACE51512D6C970031280
:1037D000DBDC7817796B12E1AC782FE2B4C80050CB
:1037E000E012D6E012D8B950030233517827797B22
:1037F00012E1ACE517642E600302389A90814F12F3
:10380000E12B12DD1212C27660FBB41C0612C7FA5D
:1038100002331612DA5950076005B406004005124B
:10382000C7FA80E1F5171475F010901E0012DAB98E
:103830007C0012DFEF12B53864AA600574310233E0
:1038400013781CE517F290814B78BB75F00A12DEF5
:103850006F12DD1212D61D60FBB4171F12C2763034
:103860001E057517418033740212AC26601EB40524
:1038700000400280172440F517801F12DA595011BA
:1038800012DD1E4007F51712DA69400E12C7FA80E2
:10389000B512C276B41CF5023316E51712DA697850
:1038A0001DF212D699B4A10830214F20200B804A76
:1038B000B4A20A302144202041742680027425C01D
:1038C000E078F1E2B4030AD0E0741A7882F20231AF
:1038D0004DD0E012A94CB41C0D12DBDC12DBF6C299
:1038E00021C22002304FB417D0301E057517418019
:1038F000A912B4C540C3F51780A0786B792712E1EF
:10390000B2781DE212CBA0501378F1E2B403087430
:10391000157882F202314D7424023313781DE212BD
:10392000D22F6035F5F0781CE2702EE5F0F2F51735
:103930001475F010901E0012DAB97C0012DFEF123D
:10394000B53864AA601378F1E2B40308740578828C
:10395000F202314D7431023313782EE2B40002804A
:1039600003B4010712DBC2602D800DB4022812DA05
:10397000396023B42402741EC0E078F1E2B403116C
:10398000D0E0B41E047419800274157882F20231FA
:103990004DD0E0023313782FE2700312B762782E15
:1039A000E2B40005782E7401F2B4020A9051CC12F0
:1039B00004E4781CE4F220230812C0F75003023319
:1039C00051302110792EE3B4020474AD800274A347
:1039D00078A8800E792EE3B4020474AC800274A13E
:1039E00078857983F309791275F00C12DE59781D08
:1039F000E2B532028005F53212C42812DBA87884C1
:103A0000F212D97712C46E782FE2B4010312E133B7
:103A100030210612BE5BE480027401129BDA782E1C
:103A2000E2B4020912DFF9751601024007301B09E2
:103A300012DFF9751600024007201E0A781DE2F514
:103A4000F0792712B892E515B403028003751502C8
:103A500078F1E2B40316782FE27883F218E4F27872
:103A6000007480F278017404F212C86FC221C2207F
:103A7000C247D2AC201E03023052023F22E515128B
:103A8000D6C9600612C7FA023061786B75F005126C
:103A9000E11B786B129770600612A94C02304F78C8
:103AA0006B12D3C760030234F4742702331312C2BB
:103AB00076C223023316782FE2B4FB004005741A55
:103AC000023313BA0E00500ABA00028005BB03008D
:103AD000400612C7FA02304F7F02786B12DAA974DF
:103AE0001812AC267007741912AC266005741A02FD
:103AF0003313787B796B75F00712CD5512DCFA78A9
:103B00006B793012E1B2786B797BE517B41207124A
:103B1000DDC64007801D12DB41501878F1E2B40386
:103B20000874157882F202314DD2A9742412A94C7E
:103B3000023049786B75F00512E11B023CBEF517A7
:103B40008002F517782FE2700BE517B41203023DDF
:103B5000C7023DCEE2B4FB004005741A023313E500
:103B600015B40402800BB40502800612C7FA0230B5
:103B70006112BCF540057423023313908159E51797
:103B8000B4130390815C12E12B12DD12E515B4042D
:103B9000028003023C5578F1E2B401F712D61D60B1
:103BA000FBB417EF787975F00B12E11B7879E51704
:103BB000B4120474B6800274B77879F608792FE3EA
:103BC00004F6C2AC740375F00712E0B37882797919
:103BD00075F00912DFA9788B793012E19A780174B7
:103BE00012F278007480F2C0A875A88012AED64098
:103BF0000512B0AE5012D0A8B42A028002742B1263
:103C0000A94CB41CE2023316D0A87982E36011B447
:103C1000130812C64C742B02331312D3A7023313AA
:103C20007983E3B4B602800AB4B7028005742B022C
:103C30003313786B793012E1B27883E2786B79854F
:103C4000B4B60512DCAC800312DD964003023D26BB
:103C50007424023313741812AC266005741A0233EC
:103C600013786B75F00712E11B796B12DDF6128E7B
:103C700034B41C03023316B41702800A12C7FA12B6
:103C8000C27660FB80EBBA00028008EAC39BB403F3
:103C900000400612C7FA023316786B12DA99E5155E
:103CA000B40403023CB1B40503023CB1741A0233FC
:103CB0001312DCFA7830796B12DA2812DBE9C2AC25
:103CC00078F1E2B40103023BACE517B4120474B618
:103CD000800274B77879F608792FE3F6E517B41304
:103CE0003B786B75F00912E11B12DCFA786B7930C6
:103CF00012E1B2786B797B12DB41786FE654F07099
:103D00000808E6700408E6601378F1E2B40308746A
:103D1000157882F202314D74240233137883797955
:103D200075F00912DFA912DBA87884F212D9771294
:103D3000C46E751700E51712E143F812E04A6036C9
:103D4000E51712E143F9789A12E1B27891793012CD
:103D5000E1B2788A798512E1B212C39A7883E2C01F
:103D6000E0E51712E143F8797AD0E0B4B70512DD47
:103D7000A2800312DCB90517E517B4050040B67838
:103D800083E2783EB4B7027845798512DC51E515B7
:103D9000B404031204CE12B35778F1E2B4031E78D0
:103DA000807402F2087405F208E4F208792FE3F255
:103DB00078007480F278017404F212C86F751505EA
:103DC000C247D2AC023F2290815F7404800590818B
:103DD000647403782EF212DFF912E12B12DD121255
:103DE000BCF540057423023313D247786B75F00796
:103DF00012E11B12D61D60FB12DBF6796B7C007D95
:103E0000087E087F027414301C02D2E3128E34B490
:103E10001C03023316B41802800A12C7FA12C276C3
:103E200060FB80EB786B12DAA9786FE6600612C748
:103E3000FA023316C2ACE517B4120C12DA49602A42
:103E4000B42409741E800512C7BF601EC0E078F15B
:103E5000E2B40311D0E0B41E047419800274157822
:103E600082F202314DD0E0023313E517B41205752A
:103E7000160380037516027811E4F27837796B1215
:103E8000E1A612B762024033D248023372E515B49C
:103E90000008782EE2B40002800612C7FA023061F0
:103EA00012DBF690815312A4B712D61D60FB12DB11
:103EB000CF12DBDC7402782EF202304F782FE270E2
:103EC0000B026D51782FE2600302754012C7FA02AF
:103ED0003061782FE26016E515B400028041B4022B
:103EE00002803CB404028037B40337803212B8F445
:103EF000701712E15F740D12AC2612071E740312C4
:103F0000AC262403F5F0120C7C12DBCF12DBDC12A2
:103F1000DFF9751500753200E412DBF602304F75DB
:103F2000150412DBF612AABE793012E16612DD1218
:103F300012D61D60FBB43A0812C276742B12D47DDF
:103F4000023052782FE2700612C7FA0230617417FD
:103F500012AC267005741A02331390816912A4B74B
:103F600012C27660FBB41C0612DBF602304F7516E7
:103F70000402402FC2AC788B796B75F01812DFA960
:103F8000786B75F03012E11B786B798B7C307D009B
:103F900075F018E412DD5A788B796B75F03012DF0A
:103FA000A9740375F00A12E0B378827400F20879FC
:103FB0002FE3F208793775F00712DE597801743B68
:103FC000F278007480F2C0A875A88012AED64005C1
:103FD00012B0AE5012D0A8B42A028002742B12A9DB
:103FE0004CB41CE2023316D0A87882E26011B413FC
:103FF0000812C64C742B02331312D3A70233137565
:104000001604802B751600C2AC792FE3702112BC08
:10401000F540057423023313741412AC2660057442
:104020001A02331312B76212DBCF782E7401F278C2
:1040300011E4F2C2AC12DD0612B250788374C9F2F8
:104040000812DBA8F208E516F208793012E19A7836
:104050008D7911E3B4C007792712E19A800312DD4C
:10406000EA12C46E12B68A78807402F20879127568
:10407000F00312DFA97884792EE3F2780912D82AA6
:104080007885790975F00412DE59787912C98B7830
:1040900089797975F00312DFA9787912D2DE788CEC
:1040A000797975F00212DFA9792EE3B40104744B1B
:1040B00080027420788EF2788F7908E3F208E51692
:1040C000F27980129DD8788374CAF212C46E12E11C
:1040D0003312CB3A12CA9B600B12A94C787975F057
:1040E0000712E11B7984E3787979306008B401081C
:1040F000E516B40406024137B4030512DD96800DBF
:10410000B402028003B4040512DCAC800078787637
:1041100003087F0075F007E6F42FFF08D5F0F8EFED
:10412000F6797812DC1D780C797975F00812DEC307
:10413000500512A94C80FE78F1E2B403028005C25A
:104140002312182B78F1E2B401557879798375F050
:104150000D12DFB37978770612DC1D801812DA06AB
:10416000C2AC9080BC12A4B712C64C600843A882AF
:1041700012A94C80E879807403F309740EF312DFFE
:1041800009E4128FB56008B420EB12A94C80FE78C8
:1041900083797975F00D12DFA9787AE6782EF2121C
:1041A000DF1379907409F3129DD8800312DF131284
:1041B00004CE12CE0FC21A12E15F740D12AC261299
:1041C000071E740312AC262403F5F0120C7CD219DE
:1041D00078F1E2B4031978807402F2087407F208E7
:1041E000E4F278007480F278017410F212C86F1251
:1041F000C4B47884E2782EF212DD06782EE2B4019F
:104200000F7811E2B4C002803D793012C835803693
:10421000B4020E793012C83578BB76B80876B38010
:104220002512DBF678BB79377C087D02740175F0C6
:104230000712DD4278BB763808792EE3B4030474A4
:10424000488002744DF6C2AC12D7D612DBCF12DF13
:10425000F9751500753200201A08740412AC26781E
:104260000DF230250C9055B71204E475F007120CCE
:104270007C75A89612DA0678F1E2B4011D20261AA0
:10428000C2AC9080BC12A4B712C64C600B12A94CF1
:1042900060FBB415EB026D51D226C221C22012BCC4
:1042A000F5503A12B61D7037C21E740712AC266064
:1042B00002D21EC21C740812AC266002D21CC21BA1
:1042C000740512AC266002D21BC21D742612AC26E5
:1042D0006002D21DC247D2ACD245023052742312C2
:1042E000A94C026D51C2AC12BCF5400574230233D7
:1042F00013782FE2B4C90050066024E532700A1228
:10430000C7FAC247D2AC02306112D68160F112BA4C
:10431000CF60ECB4A1030237D9B4A3E30235513026
:1043200019DD12CB0570D8740512AC267003024358
:104330003E740612AC26700302433E028C99780D3F
:10434000E270030242FF7881E6F50F08E6F51008F7
:10435000E6F51112D2BB7884E2C0E0788374CBF228
:10436000087908E3F212C46E12E13312DF13D0E0D1
:104370007884F2780DE214F2D21A0241B7C020C25A
:10438000008004C020D200C0F07F00E3F42FFF09BA
:10439000D5F0F8F404300001F3D0F0D02022E6B4D8
:1043A0003000400AB43A00B3400408D5F0F022903F
:1043B000000075F0051249C14037B43C04743480E4
:1043C00030B43804743E8029900000E9F82408F9DC
:1043D00075F004124C3375F00419E3C0E0C4540FB7
:1043E0002430F208D0E0540F2430F208D5F0EAE48B
:1043F000F22290000075F0051249C1400FB43C0450
:1044000074348008B43804743E8001E422754A0094
:10441000124875B43802743922742975F007800E79
:10442000741975F00D8007740975F00B8000C0F0E9
:10443000C0E0754A00124875700FD0E0D0F0C0F0AF
:10444000C0E0124CF6124C3319B438027439D0F073
:10445000D0F02212445F02706502451902706512A5
:10446000DEF579001243AF701612DBF6790078BBE7
:1044700075F00812DFB312DD121203B5024515B450
:104480003E02800302450812DBF6787975F00812C7
:10449000E11B79797B017C007D087E087F00741028
:1044A000128E34B41C02806DB4150A806812C7FAEB
:1044B00012E16D80EEB418F512DB5F9053437888FB
:1044C000740175F01812BC9A7898797D75F004190A
:1044D000E712D9BFD5F0F8120508120C7412039A2E
:1044E00060337800797975F00412DFA990000079C3
:1044F0000075F005124BD3700F79371243AF700877
:1045000012C4FA12E133800D12A94C1203D14005F6
:1045100070031203B512DEF52212DEF5754A00783B
:10452000001247F7703F7802E2F5F008E245F070BC
:104530000F90534912C7FA1204E4120C7402472C6C
:104540007900124D2C788812C98B7988788B12D219
:10455000DE7988780275F00512DFA9754A027807BE
:104560001247F76003024718C200C201754A00787B
:104570007975F00C12E11B9082B57E0A300005902F
:1045800082B87E0C78BB75F00812DE6F79797B01FA
:104590007C027D067F007410128E34B41C03024727
:1045A0002CB4150B02472C12C7FA12E16D80ECB443
:1045B00018F575F00530000375F006E5F02479F97B
:1045C000788819E712D9BFD5F0F8798875F00A789C
:1045D0000930000575F00C781912DFA975F0063066
:1045E000000375F004E412D964200005D2000245EE
:1045F0006C788812E092B418AB1203B540A660A4A0
:10460000798875F006782912DFA975F012E412D9BD
:1046100064800302471812B762740912AC261207AD
:104620001E790012473D12E15F740912AC26120791
:104630001E120C7412039A700302472C124875F56F
:10464000F07879741DF608E5F06003E4800379AB37
:10465000E3F6797912DC1D7B03124B9370B5790078
:104660001247EB124BD36024B437A8DBEC80A4755F
:104670004A001248756006B4389902472C7889E6DA
:10468000F5F079ABE365F0700702472CEA124D00B4
:10469000124A4C600302471878001247F760030281
:1046A00047187900788175F00412DFB3790012475A
:1046B000EB124C33600302471812E13B12DC107915
:1046C00018E3C0E0744BF312C5837918D0E0F312FD
:1046D000E13312B762790012473D1204CE79837834
:1046E000887C187D0075F001740190538912D70EF3
:1046F00012050879017879741EF608E9F6797912BD
:10470000DC1DC205C20612E13B786B12C98B786EC4
:1047100012D2DE12D1078014C0E012C4B4D0E0126D
:10472000A94C1203D1400570031203B512C4B41290
:10473000DEF5027065C020C200E9FF803BC020E9C1
:10474000FFC20012DB5FE3B40111D20090537C780A
:104750008D740175F01812BC9A8018905377788880
:10476000740175F01812BC9A08744EF60808E32418
:1047700030F608E4F612050812DB5F7888EF2402B1
:10478000F912DE907891EF2405F912DE7A20001FED
:10479000EF2407F9787975F00212DFB37979789907
:1047A0007C077D0075F00274019053A612D70E7637
:1047B00000120508788875F0189053AA12DE6FEF82
:1047C0002409F9789675F00A12DFB3120508788883
:1047D00075F0189053AE12DE6FEF2419F9789475C6
:1047E000F00C12DFB3120508D02022E54A2403831F
:1047F000F5F02242180D10124875600AB43829E409
:10480000F208F208800879AB75F00212DE59124CFA
:10481000ACF208E5F0F218E8F91919124D4B181826
:1048200040056003E48001D322C020C200754A0025
:10483000124875600AB4382A20001D74398023207C
:10484000000F79AD75F00312DE59181818D20080E8
:104850000779AD124DB940EA054AE54AB403004074
:10486000CFE4D02022C020D204D2058036C020D28E
:1048700004C205802EE9C0E079AB124A8FC9D0E0AE
:10488000C97010124CE4124B7A124CDD6011124CBC
:10489000478006124C47B43505124B2760D722C01B
:1048A00020C204C20212492CA2E09203C0A8C2AFE7
:1048B000E9C0E0124CE41249364065704C30042CDB
:1048C00020051279ABC8C9C8124D5DC8C9C8401EC1
:1048D00030032F801079ADC8C9C8124DB9C8C9C8F6
:1048E000400C30031DD202124CE4802CD202124C38
:1048F000E4EA124CF62003BEEA75F046A4124CEB33
:1049000080B4124CDDD20380ADB43C06EA124CF602
:1049100080A4B438033003EA74383002027400C350
:10492000124CDDC9D0E0C9D0A8D02022E54A24012C
:10493000832201010000C020C2008004C020D200F8
:10494000C0A8C2AFE8C0E0E9C0E0EBC0E07B001265
:104950004C664055200010124F144052B4FF08120C
:1049600047EB124CF6800B1247EB1249C1403FB4A3
:1049700038080BBB1E0040D7802FF8EA124D007993
:10498000B075F005124F34E8B43C02801E79B212C3
:104990004DE55004743C8013E8C0E075F00579B033
:1049A00078AB12DE59D0E080027438C38002740400
:1049B000CBD0E0CBC9D0E0C9C8D0E0C8D0A8D020C7
:1049C00022C0A8C2AFEBC0E0C0F0D260D261C26228
:1049D000C263C264E4FAFB124E5B4044124E904044
:1049E0003F7414D5E0FD124E5F403512CCC7403005
:1049F00064FF6002C26064FF6002C261C5F0B4017E
:104A000009C5F06B7012D263800EC5F02BFB12CE7D
:104A100096400D7405D5E0FD0A124D0FD5F0CCC3BC
:104A200092D112BBE372D14018C3743820611420B4
:104A30006011306306D26274008008D262743C80D8
:104A4000027404D0F0CBD0E0CBD0A822C0A8C2AF73
:104A5000124CE479AB124CC375F005124C33702C38
:104A600079AB75F007124383097451F379AB900168
:104A700000E54A75F010A412CDE17C0075F0091232
:104A8000DE9B4006124CDDE480027405D0A822C0F3
:104A9000A8C2AFE8C0E0E9F8E54A90010075F0105F
:104AA000A412CDE17C0075F00912DECD4070E8F96A
:104AB00019E3B45161C3E99408F975F00712437D15
:104AC000F5F0E365F0704FC3E99407F9124CD0128A
:104AD0004C664042E309F5F0E30945F019197019F5
:104AE000124C471247EBCAC0E01249C1124C47CAE8
:104AF000D0E0CA4025601F801A75F005124F1C4097
:104B00001970131247EB1249C1F5F0EA124D00E596
:104B1000F07003E4800A7435800674048002740522
:104B2000C8D0E0C8D0A822C0A8C2AFE8C0E0E54A1B
:104B3000124C4712489F403B7005124A4C80347813
:104B4000AB75F00912E08979AB124CC379AB75F003
:104B500007124383097451F379AB900100E54A755C
:104B6000F010A412CDE17C0075F00912DE9BE45038
:104B7000027405C8D0E0C8D0A8221247EB124CF648
:104B8000124936600BB404028008B438EDE48002A8
:104B9000743622C020C2008004C020D200C0A8C247
:104BA000AFE9C0E0124C66743D40171247EB124962
:104BB000C1400F2060062000EB2063E8EA124D00A0
:104BC0007400C9D0E0C9D0A8D020227400800A7433
:104BD000028006740380027401C020F520C0A8C2C0
:104BE000AFAAF020010EE9C0E0124F28C9D0E0C9F9
:104BF0004036703430000DE9C0E08AF015F0124DF7
:104C000011D0E0C98AF0124EAB401DEA124D00C32C
:104C1000E99AF98AF0124F1C400EF5F0EA124CF6B0
:104C2000E5F0700874008006740480027437D0A820
:104C3000D020227A00124F34400AAAF0EA124CF631
:104C4000E4C38002740422C0E0E54A23F582240D07
:104C500083F583E58204240583F582D0E0220100F8
:104C60000300140007C0E8C0E0E54A75F004A4F5AD
:104C7000F0C2D5E5F0242483C0E005F0E5F0241B64
:104C800083C3F8E58298D0E0F8E5839805F020D555
:104C9000064005D2D580DCB3D0E0F822010002CE78
:104CA000030007B014007EA407C013F0E54A23F503
:104CB000F0240783C5F0042401832200050030207E
:104CC000000195C0E0E582F309E583F309D0E02215
:104CD000C0E0E3F58209E3F58309D0E022854C8248
:104CE000854D832285824C85834D222582F582E580
:104CF000F03583F583222582F582E43583F583221E
:104D0000C3C5829582C582E4C5839583C58322A3EA
:104D100022C0F0EAC0E0E5F0600B7A00E32AFA096D
:104D2000D5F0F9EAF3CAD0E0CAD0F022E32401D4E6
:104D3000F309E33400D4F30922EAC0E0C020C0F054
:104D400075F002C200D202C203802BEAC0E0C0208C
:104D5000C0F075F002C200D202D2038019EAC0E0AE
:104D6000C020C0F075F0028007EAC0E0C020C0F0AB
:104D7000C200C202D203C0F0C3200308E69712D8D3
:104D8000A5F6800FE3FAE29A6002D2003002041224
:104D9000D8A5F20809D5F0E19201D0F0C3E895F06A
:104DA000F8C3E995F0F9A201E430000104500104D0
:104DB000D0F0D020CAD0E0CA22C0F0EAC0E075F03E
:104DC0000308080909C3E3FAE29A400970071918B1
:104DD000D5F0F2800774011918D5F0FB0809CAD084
:104DE000E0CAD0F02275F003E312D725401909D5A7
:104DF000F0F61919E3B41300500C600A19E3B43249
:104E0000005003C37001D322E212D7AAF208D5F0F2
:104E1000F722E2C0F012D794D0F0F208D5F0F322D6
:104E2000E825F014C9C0E0E5F0C313F5F06008C64A
:104E3000C7C60819D5F0F8D0E0F922E825F014C962
:104E4000C0E0E5F0C313F5F0600DE2C0E0E3F2D09E
:104E5000E0F30819D5F0F3D0E0F92274A6800274CB
:104E6000A7CFC0E0CFC0F07F02C0E075F0FAD0E07D
:104E7000C0E012BF5E500F7432D5E0FDD5F0EFDF19
:104E8000EAD374048001E4D0F0D0F0CFD0E0CF2298
:104E9000E58312B9564008E58212B956E45002740F
:104EA0000422CAC0E0C020C2018009CAC0E0C020FC
:104EB000D200D201C0A8C2AFC0F0E582543F300199
:104EC00001FA124E5B5005D374048036124E9040A6
:104ED000E9EA300105E7300001E312B95640E83055
:104EE000011A09A3D5F00280130AEA543F70E212B6
:104EF000BBE3124E5B400B12BBE380BE12BBE3125E
:104F00004E5B92D112BBE372D1D0F0D0A8D020CAB0
:104F1000D0E0CA22C020C201C2028020C020D2003C
:104F2000D201D202D2038014C020D200D201D20218
:104F3000C2038008C020D200D201C202C0A8C2AF02
:104F4000CAC0E0C0F07A00740AD5E0FD124E5B40A2
:104F50000F124E9040EF741ED5E0FD124E5F5002CE
:104F60008051E9C0E012CCC75009D0E0F9D0F0C0C0
:104F7000F080D230021530030BC0F0F5F0E365F09D
:104F8000D0F0800264FF60100A800D200103FA80D7
:104F90001F200003F78001F3E5F06401600E12CEDC
:104FA000965004D0E0800C7405D5E0FD09D5F0B52D
:104FB000D0E0C392D112BBE372D14001EAD0F0CA73
:104FC000D0E0CAD0A8D02022CCC5D0CAD3D0C8C97E
:104FD0002D31313520202020002A2A2A20CACECF88
:104FE000C8DF2020C4CECAD3CCC5CDD2C0202A2A47
:104FF0002A002A2A2A2A2A2A2A2A2A2A2A2A2A2A3B
:105000002A2A2A2A2A2A2A2A2A2A0D2020C2CDC858
:10501000CCC0CDC8C52120C2D1C520D1D3CCCCDBDA
:105020002020200D20C2CED1D1D2C0CDCEC2CBC542
:10503000CDDB20C8C720DDCACBC721200D2A2A2AF4
:105040002A2A2A2A2A2A2A2A2A2A2A2A2A2A2A2AC0
:105050002A2A2A2A2A002A2A2A2A2A2A2A2A2A2ADA
:105060002A2A2A2A2A2A2A2A2A2A2A2A2A2A0D2ABD
:1050700020202020C2CDC8CCC0CDC8C52120DDCA8B
:10508000CBC7202020202A0D2A20C1CBC8C7CAC0E8
:1050900020CA20C7C0CFCECBCDC5CDC8DE21202AA7
:1050A0000D2A2A2A2A2A2A2A2A2A2A2A2A2A2A2A7D
:1050B0002A2A2A2A2A2A2A2A2A0020CDC5D220C40E
:1050C000C0CDCDDBD520C220C7C0C4C0CDCDCECC95
:1050D0000D2020202020C4C8C0CFC0C7CECDC52100
:1050E00000202020D1CED1D2CEDFCDC8C520CECF5A
:1050F000D6C8C90020CECFD62020203D2020202099
:1051000020CECFD62020203D2000C220D2CECC20E1
:10511000D7C8D1CBC500CDC520D3D1D2C0CDCEC24A
:10512000CBC5CD0020202020202020CDC0CBCEC359
:10513000C820CDC50D202020C7C0CFD0CEC3D0C041
:10514000CCCCC8D0CEC2C0CDDB0D00202020CDC03D
:10515000CBCEC3CEC2DBC520D1D2C0C2CAC80D00DF
:10516000CDC0D7C8D1CB2E00C2DBC4C5CB2E002A00
:105170002A2A20D7C5CA20C0CDCDD3CBC8D0CEC215
:10518000C0CD21202A2A2A002D2D2D2D2D2D2D2D6B
:105190002D2D2D2D2D2D2D2D2D2D2D2D2D2D2D2D3F
:1051A00000D7CFCC2000D7C5CA3A00C1C8CBC5D2E2
:1051B0003A00CF2EC8D2CEC300C8D2CEC300D1CAC7
:1051C000C8C4CAC000CDC0C4C1C0C200202A2A2A97
:1051D0002A2A2A20C2CEC7C2D0C0D2202A2A2A2AEE
:1051E0002A2A2A20002D2D2D2D2D2D20C0CDCDD3C6
:1051F000CBDFD6C8DF202D2D2D2D2D2D2D00CDC0A0
:10520000CBC8D7CDDBCCC800C2CDC5D1C5CDCE0073
:10521000D1C4C0D7C000CAD0C5C4C8D200CA20CE2D
:10522000CFCBC0D2C500CFD0CEC4C0C6C800C0CD81
:10523000CDD3CBDFD6C8C80020D1CAC8C4CAC800E5
:1052400020CDC0C4C1C0C2CAC800C2CEC7C2D0C06F
:10525000D2DB00C2DBCFCBC0D2DB00C220CAC0D1C0
:10526000D1C500C3D0CED1D12DC8D2CEC300C3C0CA
:10527000D8C5CDC8C5204E2000203C3C3C20CFCE18
:10528000C2D2CED0CDDBC920D7C5CA203E3E3E20FB
:105290002000202020CACECDD2D0CECBDCCDC0DFA6
:1052A00020CBC5CDD2C000CDC0CBCEC300C2CEC7AF
:1052B000C2D0C0D200C2CDC5D1C5CDC8C500C2DBE9
:1052C000CFCBC0D2C0000000CECFC5D0C0D2CED090
:1052D000204E3A00CED2C4C5CB204E3A00C220D2D6
:1052E0002ED72E002020202020D4C8CE20CECFC5FF
:1052F000D0C0D2CED0CEC2002020C4CECBC6CDCE20
:10530000D1D2C820CECFC5D0C0D2CED0CEC200D44C
:10531000C8CE3A00CFCEC4CFC8D1DC3A5F5F5F5F62
:105320005F5F5F5F5F5F5F5F5F5F5F5F00CECF3A32
:105330002000CEF8E8E1EAE02100D3F1EFE5F8ED56
:10534000EE2100C7C0C22E4E00CDC5D220D1C2CEA4
:10535000C1CEC4CD2EC0CAD2C8C2C0D6C8C92100D1
:10536000CDC5D220D1C2CEC12ED0C5C3C8D1D2D0D6
:105370002EDDCACBC7210020CFC5D0C5C0CAD2C838
:10538000C2C0D6C8DF20DDCF00CED1D22E20C0CA09
:10539000D2C8C2C0D6C8C93A00CDCECCC5D03A001A
:1053A000C4C0D2C03A00D1CC3A00D0CD3A00C8CD6A
:1053B000CD3A00DDCACBC720F3E6E520E0EAF2E80B
:1053C000E2E8E7E8F0EEE2E0EDE02100DDCACBC77D
:1053D00020EDE520E0EAF2E8E2E8E7E8F0EEE2E0DE
:1053E000EDE02100C0F0F5E8E220F3E6E520E7E09B
:1053F000EAF0FBF2210020202020C0CAD2C8C2C897
:10540000C7C0D6C8DF20DDCACBC700C0CAD2C8C259
:10541000C8C7C0D6C8DF204E00CED1D22EC0CAD257
:10542000C8C2C8C7C0D6C8C93A00DDCACBC72000A9
:10543000D2E5F1F220E0F0F5E8E2E03A00C7E0EA78
:10544000F0EEE9F2E520F1ECE5EDF32100C0F0F536
:10545000E8E220DDCACBC720E7E0EAF0FBF221005A
:10546000C2EDE8ECE0EDE8E52120C0F0F5E8E2204F
:10547000DDCACBC70D20202020E1F3E4E5F220E7D0
:10548000E0EAF0FBF2210D20205B335D202D20EFC0
:10549000F0EEE4EEEBE6E8F2FC2100D8F0E8F4F2FE
:1054A0003A2000D2C5D1D2CEC2C0DF20D1D2D0CED8
:1054B000CAC0203031323334353637383920D8D06D
:1054C000C8D4D200F2E5F1F2EEE2E0FF20F1F2F012
:1054D000EEEAE0203031323334353637383920F8CF
:1054E000F0E8F4F200202020202020D2C5D1D220E4
:1054F000CFD0C8CDD2C5D0C000D2E5F1F220DDCFEB
:1055000000CDE520C0EAF2E8E2E8F0EEE2E0EDE00E
:105510002100D0E5E33A00C0EAF23A00CEF2F73AD1
:1055200000202020202020202020C2F1E5E3EE7C76
:10553000D1E2EEE17CCFEEE2F00052532D32333275
:1055400020CFDDC2CC00693D30202D20E0F0F5E811
:10555000E220EEF2EAF0FBF2202000663D30202D42
:1055600020E0EAF2E8E2E8E7E8F0EEE2E0EDE00071
:10557000613D30202D20EDE5E8F1EFF02E20EEF832
:10558000E8E1EAE000733D30202D20EEF2EAF0FB86
:10559000F2E020F1ECE5EDE02000643D30202D202C
:1055A000EEF2EAF02E20E4EEEAF3ECE5EDF2002074
:1055B000C4C000CDC5D2002020C2EDE8ECE0EDE88B
:1055C000E52120D2F0E5E1F3E5F2F1FF0D20EFF067
:1055D000EEE2E5F1F2E820F2E5F5EDE8F7E5F1EAD3
:1055E000EEE50D20202020EEE1F1EBF3E6E8E2E02D
:1055F000EDE8E52100CED2D7C5D22020D1CCC5CD53
:10560000CDDBC900CED2D7C5D220CFCE20CAC0D1E3
:10561000D1C8D0C0CC00CED2D7C5D220CFCE20CEDC
:10562000D2C4C5CBC0CC0020202020CFCED7C0D143
:10563000CEC2CEC920CED2D7C5D200CFD0CEC4C024
:10564000C620CDC520C1DBCBCE2100CFD0CEC2C578
:10565000C42ED7C5CACEC200CFCEC2D2CED0CDDBEB
:10566000D500C0CDCDD3CBC8D0CEC2C0CDCE002DBD
:105670002D2D2D2D2D2D2D2D2D2D2D2D2D2D2D2D5A
:105680002D2D2D2D2D2D2D0D2A20C0C2C0D0C8C9E5
:10569000CDCEC520CED2CACBDED7C5CDC8C5202A37
:1056A0000D2D2D2D2D2D2D2D2D2D2D2D2D2D2D2D4A
:1056B0002D2D2D2D2D2D2D2D2D002020202A2A2A77
:1056C00020C2CDC8CCC0CDC8C521202A2A2A00C2FC
:1056D0002020DDCF20CED1D2C0CBCED1DC202020E7
:1056E000202020C3C0D82E00D1CCC5CDCDCEC52022
:1056F000C3C0D8C5CDC8C5204E20004320202020DF
:105700002020202020202020CFCE00D1CCC5CDC00D
:1057100000C2D1C5C3CE20C7C0CFC8D1C5C90020E3
:1057200020202020CFC5D0C5CFCECBCDC5CDC8C57C
:105730000D20202020D0C5C3C8D1D2D0C020C8D2CF
:10574000CEC3C0002020202020CE20D220D720C5CC
:1057500020D22020CF20CE0DDDCDC5D0C3CECDC5EB
:10576000C7C0C2C8D1C8CCCEC920CFC0CCDFD2C838
:105770000D0020CED2D7C5D220CFCE20C0CAD2C8ED
:10578000C2C0D6C8DFCC20DDCF0D00CED2D7C5D267
:1057900020CFCE20C0CAD2C8C2C8C7C0D62E20DDF6
:1057A000CACBC70020C7C0CFC8D1DC20CDC5C4CE6E
:1057B000D1D2CEC2C5D0CDC02100DDCACBC700C278
:1057C000E5F0F1E8FF20CFCE3A20313135525500D7
:1057D000CDC520C0CAD2C8C2C8D0CEC2C0CDC0219B
:1057E000002020202020CFC0D0C0CCC5D2D0DB20CC
:1057F000D7CFCC00C4E0F2E020DDCACBC73A00C26C
:10580000F0E5ECFF20DDCACBC73A0020DDCACBC7EC
:1058100020CDC520C8D1CFD0C0C2CDC020C8CBC8F4
:105820000D202020CDC520D3D1D2C0CDCEC2CBC536
:10583000CDC000202A20CED8C8C1CAC020444154BF
:105840004120464C41534821202A00202A2A20CEBC
:10585000D8C8C1CAC02020D2C0C9CCC5D0C0212060
:105860002A2A00202A2A2A2A2A20CED8C8C1CAC019
:1058700020DDCF21202A2A2A2A2A0020D2C5D5CDF0
:10588000CECBCEC3C8D7C5D1CAC8C920D2C5D1D204
:1058900000D2C5D1D220C7C0C2C5D0D8C5CD00D690
:1058A000C8CACB00D2C5D1D22020CED1D2C0CDCE55
:1058B000C2CBC5CD00CED82EC2C5D0D1C8C820CA53
:1058C000CECDD2D02EDDCF2100CED82ECACECDD493
:1058D000C8C32EDDCF2100DDCF202D2045455052FD
:1058E0004F4D00CEC1DAC5CC20CFC0CCDFD2C8200E
:1058F000D7CFCC3A200033324B0036344B00313214
:10590000384B00D3F1F2E0EDEEE2EBE5EDEDFBE933
:1059100020E1EBEEEA20DDCF0DEDE520ECEEE6E553
:10592000F220E1FBF2FC20F1E1F0EEF8E5ED0DE212
:1059300020FDF2EEEC20F0E5E6E8ECE5210075173D
:1059400001751558C2AFE517C0E07882E2F52AE587
:1059500015645A6003025B1FD0E0C0E06003025B85
:105960001F754A027983124A8F700E7885E2C394BC
:105970000008E294204008743312A94C0260E178D8
:10598000F1E27003025A0B741512AC267003025A2E
:105990000B75A8809080BC12A4B712DA06C2AF12B1
:1059A000C64C601343A88212A94CB415E4741612B5
:1059B000AC2670570270659080B312A4B712DB9AC0
:1059C00012DA06C2AF12CF4578807401F20874155E
:1059D000F278007480F278017402F212DB9A12AE4F
:1059E000D6400512B0AE5009B42A02800B742B8049
:1059F000077982E36015744443A88212A94CB41558
:105A000090741612AC267003027065D0E0C0E0906E
:105A10005A1512CE69740112AC266024C0E012D966
:105A20009B7004D0E0801990813912A4B7C21B7416
:105A30000512AC266002D21BD0E075F0AA026832D3
:105A4000D0E0C0E0905A4A12CE6990813112A4B7DA
:105A500075170078AB75F01812E089780075F08042
:105A600012E08990060012DAF612DFEF790075F085
:105A70008012DFDBE517600924AAF8E27003025AFE
:105A8000A5E51712DA797851790B12E19A785179F4
:105A90005F12DC51900F0012DAF612DFEF79007519
:105AA000F08012DFC70517E517B409005003025A4A
:105AB0005B12E133751700D0E0C0E0905AC112CEFE
:105AC00069E517600624AAF8E26022900F0012DA56
:105AD000F612DFEF790075F08012DFDB900600121E
:105AE000DAF612DFEF790075F08012DFC70517E5EF
:105AF00017B4090040C112E133D0E0C0E0905B036D
:105B000012CE6990813112A4B712A707D0E0C0E08D
:105B1000905B1612CE6912DA1712E13B75155AD056
:105B2000E0C0E0905B2912CE6990813912A4B7D011
:105B3000E0C0E0F51779A312E14A75F003120C7C7E
:105B400012B762741012AC2612071E788812DCE0BD
:105B5000788AE515F608742DF608D0E0C0E07005E7
:105B60009055F5800BB401059056048003905616AD
:105B700075F01612BC9A12050879A312C609D0E076
:105B8000C0E0905B8812CE69788812DCE0E517B43B
:105B90000200501212CB6D788812DCE0D0E0C0E039
:105BA000905BA612CE69D0E0C0E06056B4011190BF
:105BB00052C8788875F01812BC9A7891E51780124F
:105BC0009052D4788875F01812BC9A788FE517C374
:105BD000940412D042D0E0C0E0B40520E517C3948D
:105BE0000412D699B4A1028013907C70B4A20390E1
:105BF0007C7F789475F00C740112BC9A1204CE125A
:105C00000508780075F08012E08912E13B900600EB
:105C100012DAF612DFEF790075F08012DFDBE5179C
:105C2000C0156008B401028003B4050A78AB75F0B2
:105C30001812E089800624AAF8E26005E51712DA56
:105C400079D0157851790B12E19A7851795F12DC8D
:105C500051D0E0C0E07003025C99B40502501078A6
:105C60000B75F06912E0537003025D44025C997891
:105C70000B75F02312E053700D785175F00712E0A8
:105C8000537003025D44905226795112C7479052D7
:105C90004A791912C747025D449051FE790B12C729
:105CA00047905216795F12C747741312AC267003DF
:105CB00012D406905208796612C747905253796DF4
:105CC00012C74790524A791912C747D0E0C0E07016
:105CD00024786B790B12E1B2786B796612DD9678D5
:105CE0006B796D12DCAC786B791912DCAC90525B7D
:105CF000796B12E158782E75F023E2700608D5F022
:105D0000F9804175320012DB5FE53275F007A4249B
:105D10002EF978917C0F75F0077D02740112DD5A1F
:105D200078889052A775F01812BC9A788EE53224C4
:105D300031F61205080532E532B4050040C875F0A9
:105D400001120C7CD0E0C0E0B4050050089051B9BD
:105D5000795112C7477800795112DC51905263791A
:105D60000012C7470517D0E0C0E06017B4050AE588
:105D700017B40900500D025B7EE517B4050050030F
:105D8000025B7ED0E0C0E0B40100501E905188124A
:105D900004E490564B797412C954905662797C127F
:105DA000C954905658797812C954C207E515B458A9
:105DB00003025FE4D0E0C0E06003025F6F79CE12BF
:105DC0004420600DB43905C207025F6F12A94C80F0
:105DD000FE789112D2DE789512C98B7988770E12EF
:105DE000DC1D754A021248756010B4380878ABE4BF
:105DF000F208F2800512A94C80FE788A12E10B7835
:105E00009379ABE32401D4F60809E33400D4F6799E
:105E10008D7406F77988770F12DC1D788DE6D5E052
:105E2000057434025DF5F6798A12E113754A02129F
:105E30004B9960057434025DF5788E12E10B798818
:105E4000771012DC1D780074FF75F02012D9647889
:105E500000799375F00512DFA9790512D4D4798EF3
:105E600012E113754A021247EB1249C120603179E1
:105E70008E12E11379201247EB124C336003025D5E
:105E8000F5780079201247EB15F0E2F582E36582A0
:105E90006003025E1B0809D5F0F0206322025E1B3E
:105EA0007988771012DC1D798E12E1131247EB7995
:105EB00000124BD76009B43703025E1B025DF5790F
:105EC00088771112DC1D798E12E113124CE4754AA9
:105ED0000212489F124A4C600512A94C80FE7800BD
:105EE000798875F01012DFA91204CE7810790B753D
:105EF000F00212DE59E4F208F29056E8791012C965
:105F000054786B790D75F00312DFB3786E790975EB
:105F1000F00212DFB312E0C3120C7979007412F3AD
:105F2000129DD8800A7800798875F01012DFA99048
:105F3000503D1204E4790BE3C3947012D8A5F56BBD
:105F400009E3941940219056BA1204E478889056D7
:105F5000CF75F01812BC9A78997430C3956B12D82B
:105F6000A512DCED12050875F005120C7CD207D0E5
:105F7000E0C0E0F517D0E0C0E0905F7F12CE6990FE
:105F80000F0012DAF612DFEF790075F08012DFDB16
:105F90007800795112DC51780B75F07512E0899018
:105FA000060012DAF612DFEF790075F08012DFC713
:105FB00012E133D0E0C0E0700FD0E0C0E0905FC3EA
:105FC00012CE6912CC67801C0517D0E0C0E0B40582
:105FD0000AE517B40900500C025F75E517B4050017
:105FE00050028091D0E0C0E0905FEE12CE6979A3BC
:105FF00012E14A79A312E15112E133E515B45A30A6
:10600000D0E0C0E090600A12CE69D0E0C0E079A78D
:1060100012C70A20071A9051881204E490526E7930
:10602000A712C954D0E0C0E079A712E0BB12E13357
:10603000D0E0C0E090603A12CE69D0E0C0E07003DA
:1060400020071390604912CE69786B12C98B786E65
:1060500012D2DE12D107D0E060030260E1E515B490
:106060005A4478F1E2B4013ED0E0C0E09060721290
:10607000CE69C2AC79807403F309740FF3780074AD
:1060800080F278017402F212AED6501AB42A02805D
:1060900002742B12A94C641C600512C27680D37462
:1060A0001A12AC2660CC9020807C0012DFEF796B56
:1060B00075F00312DFE5786B75F00312E05C602188
:1060C000786E12C98B12D50D400BE5727013E57115
:1060D000B40600500C9055B71204E475F007120C8A
:1060E0007C12C4B4E5177015E515B45A1074231268
:1060F000AC26600975170575155A025944740912C2
:10610000AC2612071E742512AC266005E53104F595
:106110003075A89212D366027065C0A875A880C0B9
:106120002075A880F5178D568E578F5875160085E7
:106130005653855754855855E4F552532086E51734
:106140006007B405005002D206300710785175F090
:106150000E12E089788075F02312E0891267A81288
:10616000DFEF12B538B4AA028028B4FF20E517B4D7
:106170000A00401975F06412B538B4FF10D5F0F775
:106180001267A812DFEF74AA12B9B680CF7420028A
:10619000679E12B538B4FF02800EC0E012BB2B60C0
:1061A00003026275D0E080E5755200E55664004256
:1061B00052E55764224252E558640045527019E591
:1061C00017B40E0574220267A3787975F00F12E1F7
:1061D0001B12D8DFE40267A3E517B40E0574220290
:1061E00067A3E516B4CA2BE517B40D05742302673F
:1061F000A3B40A028003B40B04741F8024B40C0EF1
:106200007552007988E7B4C92C755200802AE402DF
:1062100067A3B4CB39E517B40B028003B40A137437
:1062200045C0E0780F12681A781212681AD0E0029E
:1062300067A3B40C0D755221780512681AE5520255
:1062400067A3B40D0574450267A3E40267A3B4CC49
:106250001FE517B40B028003B40A04744580C2B46E
:106260000C0280D1B40D0574450267A3E40267A354
:1062700074210267A3D0E0F516B4C91F7988F70925
:1062800012BB2BF5F012DFE5E517B4090050093019
:10629000070620060302663202635EB4CA537979A8
:1062A000F70912BB2BF5F012DFE5E517B40A005031
:1062B000030266FEB40C030261FDB40B028003B45A
:1062C0000A0B85536B85546C85556D8079B40D052B
:1062D00074230267A3B40E6E786B797BE7656B70ED
:1062E0006509E7656C705FAD53AE54AF55E4026766
:1062F000A3B4CB1AE517B40500500E600712B538E9
:1063000065177005787812D82AC202026346B4CCA9
:1063100047E517B4090050296016B4050050111262
:10632000B53865177005787C12D82AC20202634618
:106330002002F3D202855356855457855558026181
:106340004CD202026346E51612BB2B04041267B15D
:106350001267C0501B02612F300703300617E51685
:1063600012BB2B04041267B11267C0500302615CB8
:10637000742002679EE517B40900400280E0E5162C
:106380007988F70912BB2BF5F0E516B4A302800D4E
:10639000B4A8028008B4AD028003B4AE1112B538BF
:1063A000F709742312CC97E5F0C39423F5F012DFBC
:1063B000E5E516B4A100500302616AB4AE00502EA8
:1063C000C394A133C0E0240B83F583D0E02405837C
:1063D000F582E4736430635E6430635E635E642AF6
:1063E000635E642A635E616A635E64246424B4B19C
:1063F00000500302616AB4BA00400302616AC394A8
:10640000B133C0E0240B83F583D0E0240583F5820B
:10641000E47364E864D864E064D0635E657C656CB2
:1064200065746564D205C204800AC205D204800482
:10643000C205C204E5176008B401028003B405096F
:106440007895E624AEF874AAF2788A798F12A31CA4
:1064500012D2527851797B30040512DC92800312FB
:10646000DD8AE517B405004019B409005014E5179A
:10647000C39404F5F07895E665F060067552000265
:10648000635E7858797B30040512DC92800312DD5C
:106490008A3005028012797B30040D7812300205B3
:1064A00012DC92800312DD8A7894E6601EB4060046
:1064B0004003E48016C0E01412DE0CF8797B30044F
:1064C0000512DC92800312DD8AD0E0F55202635E91
:1064D000D205D20474278016C205C2047427800E28
:1064E000D205C20474208006C205D2047420C0E024
:1064F0007851798C30040512DC92800312DD8AE534
:1065000017B405004018B409005013E517C39404EC
:10651000F5F07892E665F06005D0E002635E7858A9
:10652000798C30040512DC92800312DD8A30020A75
:10653000A204B39204A205B392057891E660121406
:1065400012DE0CF8798C20040512DD8A800312DC3F
:1065500092D0E0F8798C20050512DD8A800312DCE8
:106560009202635ED205D20474278016C205C2046B
:106570007427800ED205C20474208006C205D2049E
:106580007420C0E07891795112E1B27851798A2073
:10659000040512DDA2800312DCB9E517B405004042
:1065A00019B409005014789A795812E1B212C39ABA
:1065B000788A797A75F00712CD5578A1795812E169
:1065C000B27858798A20040512DDA2800312DCB962
:1065D00030020AA204B39204A205B39205D0E0F8F7
:1065E000798A20050512DDA2800312DCB9755200FC
:1065F000E55212DE0CF812E04A602B789179A17511
:10660000F00712CD55789AE55212DE0CF912E1B27C
:1066100012C39AE55212DE0CF8797A20040512DDD5
:10662000A2800312DCB90552E552B4050040C10254
:10663000635E788AE67004780B8025B401047819CB
:10664000801EB4020478668005B40312786D798BDD
:1066500030020512DCB9800312DDA202635E785FAE
:106660008851795830020512DCC6800312DC51755E
:106670005200E55212DE0CF812E04A6072E55275E3
:10668000F010901E0012DAB97C0012DFEF12B5385C
:1066900064AA6005743202679E797975F00612DF8C
:1066A000E5E55212DE0CF912926A753200E5327598
:1066B000F00AA42488F9E7602D1475F007A4242EAD
:1066C000F80909E9C0E00930020512DCB9800312BB
:1066D000DDA2D0E0F9E7700E09A85130020512DC06
:1066E000B9800312DDA20532E532B4030040BE05D5
:1066F00052E552B40500500302667202635EE5176C
:106700006003B4010B7885E624AAF874AAF2E517B1
:10671000B4090280367007787412D82A8005B4054F
:1067200000400302634620060A787412D82AD20673
:106730000263467885E66517600302634685535613
:10674000855457855558C20602615C788AE6600315
:10675000B40448E54AB4FF028024755200E552753E
:10676000F009A4F8E2797F67700A087982E267701D
:10677000030880220552E55214B54A0040DF054A5D
:10678000E54AB41800501475F009A4F8797FE7F2CF
:10679000087982E7F208798B12DDA202634612A91A
:1067A0004C80FED020D0A822855682855783AC58D5
:1067B000222556F556E43557F557E43558F5582255
:1067C00078F1E2B4022AE5225403700BC374649595
:1067D0005774009558B322B4010BC3747E95577457
:1067E000009558B322C374ED955774009558B322A1
:1067F000E5225403700BC3747F955774009558B30A
:1068000022B4010BC374FF955774009558B322C38B
:1068100074FF955774019558B322E556F608E5576D
:10682000F608E558F622E553F608E554F608E5556E
:10683000F62275A880F51785F029D24775F0041265
:106840000C7C12B762740A12AC2612071E90529288
:106850001204E479A312E14A79A312C609740F1253
:10686000AC2612071E12D8DF12DBCFD207C206C237
:1068700003E4F532F515E517B404004002803978D9
:1068800089790F75F00612CD557890E520F608E568
:1068900017F608E515F608E516F608E532F608D00D
:1068A000E0C0E0F608E52AF608E529F608E523F653
:1068B0007988740BF712DC1D12E00B12DFEF12B5B2
:1068C00038B4AA0280057420026D2012B53860F633
:1068D000F4600302694F12D9F560082003057421A2
:1068E000026D20E517B404004004E4026D207889AD
:1068F000E520F608E517F608D0E0C0E0F608E52A3E
:10690000F608E529F608E523F67988740CF712DC19
:106910001D740A12AC2612071E786B12C98B786E92
:1069200012D2DE12D10790812812A4B7D2AFD2A919
:1069300012C27660FB75A880B42C0302683A79A372
:1069400012E14A79A312E15112E133E4026D20F41D
:10695000C0E012BB2B70030268C6D0E0F516B4CCC1
:1069600005D203026CFBB4CB05D203026CFBC2035D
:10697000B4CA03026CA6B4C926100703026C0D75D5
:10698000F002798412DFDB7985E3B401069051CC03
:106990001204E412DF0975320012DBCF0268B8205E
:1069A0000707E517B402005015E51612BB2B0404C7
:1069B00012D5EA12BEB250030268B80268DBE516CF
:1069C0007983F312BB2BF5F00912DFDBE516B4A1D6
:1069D0000050030268C6B4AE00502EC394A133C069
:1069E000E0240B83F583D0E0240583F582E4736A09
:1069F0004369A96A5869A969A96A3F69A96A54697A
:106A0000A969A969A96A436A58B4B1005003026828
:106A1000C6B4BA0040030268C6C394B133C0E024D0
:106A20000B83F583D0E0240583F582E4736B116B4F
:106A3000016B096AF969A96B6B6B5B6B636B53D272
:106A4000058002C2057812798575F00C12DE59C2F4
:106A500004026A66D2058002C205781279A875F030
:106A60000C12DE59D2043005069051E51204E430D0
:106A700006089051881204E4C206E517B4030040EA
:106A800031781DE2B532028014F53212C428E517C0
:106A9000B404005008740F12AC2612071E30041202
:106AA00012BE5BE517B404005008740F12AC261236
:106AB000071E12D6E07827797B12E1A6E517B40409
:106AC0000720040474018001E4129BDA78377927E7
:106AD00030050512DCC6800312DC51781CE260121E
:106AE0001412E143F8792730050512DCC680031241
:106AF000DC51A20592060269A9D205D2047845802C
:106B000016C205C2047845800EC205D204783E80C4
:106B100006D205C204783E798730040512DC9F80D6
:106B20000312DC44788CE260121412E143F8798796
:106B300030050512DC9F800312DC44E517B4030026
:106B4000400312B3573004069051881204E4C20681
:106B50000269A9D205D20474458016C205C2047424
:106B600045800EC205D204743E8006D205C204746C
:106B70003EC0E07830793712E19A7830794512DCFE
:106B8000517830793E12DCC6C016751600E5161233
:106B9000E143F812E04A602F788A798512E1B278F1
:106BA00091793012E1B2E51612E143F9789A12E1D7
:106BB000B212C39AE51612E143F8797A300505124C
:106BC000DCB9800312DDA20516E516B4050040BD50
:106BD000D016D0E0F8798530040512DCC6800312A7
:106BE000DC51E517B40300401F7883E2B4B602809D
:106BF00003B4B70512B357800F9051E51204E412A5
:106C0000B3579051881204E4C2060269A9300608FD
:106C10009051881204E4C206E51612BB2BF5F079F8
:106C20008412DFDBE517B40200405912DD0612B210
:106C30005012E00B12DFEF12B53874C912BB2BF5FE
:106C4000F0798312DFDBE517B4040040237827795D
:106C50008D12E19A12B68A7885E2B402028003B4FA
:106C600003297985E3782EF209783712E19A801B9F
:106C7000788D12DDEA7985E3B40200500779861237
:106C8000CEEF80077985E30912D093E517B4051399
:106C9000E51612BB2B040412D5EA7401792EF31405
:106CA000026D200269A9E5167983F312BB2BF5F07A
:106CB00009798412DFDB100702801A7984E3F51565
:106CC000B402069051CC1204E412DF0975320012AE
:106CD000DBCF0268B8E517B4040040091204CE12F5
:106CE000CE0FE4801612CAD07984E30912C0A8E559
:106CF000176401600675F001120C7CE51612BB2BBF
:106D0000040412D5EA12DF13E517B40400400A792F
:106D100084E3792EF3E4026D20D207C2060268767E
:106D2000B4200512A94C80FEF5F0E517B40400402C
:106D300007E5F0D020D0A82275155AE5F070E4E5FB
:106D400029B4AA03025A406005E4F530F531028700
:106D50008612D366E412DEF512DBF6740912AC2655
:106D600012071EE52F5480F52FC22712E1FC12DA1C
:106D700006D2ACD2AAE4F530F53102705112D61D1C
:106D800060FBB43A03026DDA12DA594003026DDA9D
:106D9000E530B41D0912C27612C7FA026D7DE52FE7
:106DA00054037031786B12B3D56418700BE530045E
:106DB0001270C8F516B4FF0612C7FA0270A1E530CA
:106DC0007003026FE412B01A60030270A1853031C3
:106DD000053002705112C27680A312C276B49A02B4
:106DE0008003026EDB78F1E2B403028003026EDB03
:106DF000C2AC7881E2B40202800CB40D03026E4B87
:106E0000B40E13026E587882E2700474008029B4C4
:106E10000104E52F60047402801EC2A978CE75F0CB
:106E20001412E08978CE798375F00612DE59E4F504
:106E300030F531D2A9026FAA7882F278007480F21C
:106E400078017403F212C86F026D51207F0575300E
:106E5000018003753004800B207F057530078003A7
:106E6000753003E52F6003026E16786B798375F039
:106E70000612DFB3E530041270C8B4FF05741002C7
:106E80006E387882E2C0E012B01A6006D0E0741B5F
:106E900080A6D0E0B4030050F5D33530C530F531CD
:106EA000E53012CDA0602FC082C08312B01A7022CC
:106EB0007882E2C0E0E4F278007480F27801740332
:106EC000F212C86FD0E07882F2853130753100C29D
:106ED000AC22D082D0837402026E38B41B0612B684
:106EE000F6026D7DB42C06122319026D7DB4140DCB
:106EF000E530B41DF579897403F7027023B43A08BC
:106F0000C22412ACD9027065B41228E530700302B5
:106F10006D7DAD301DED12C3E15403F5F0E52F5446
:106F200003B5F0058D3002705140E912C407F53009
:106F3000027051B41302801DB4154DE52F54037037
:106F4000028012E4307F07F530F531027051C5310F
:106F5000C530027051E52F5403F5F0AC30AD310D62
:106F60000CEC12C3E1B4EE0FE5F0700675300002D0
:106F700070518D300270515403B5F0058C300270A1
:106F80005150DD8D30027051B41C14E52F54037044
:106F900006753000027051E53104F530027051B4CD
:106FA0001878E530B41D03026D7DE52F540370346D
:106FB000786B75F006743012E123E5307011786B50
:106FC0007431F6740712AC266005751601800EE563
:106FD00030041270C8F516B4FF03026DB8E53060D6
:106FE00003026DC5E530207F05B402118003B405AE
:106FF0000C78F1E2B4030612C7FA026D7DE5301297
:10700000CDA0605EC082C08312B01A7003C2AC22F1
:10701000D082D08312DBF60270A1B41703026F5541
:10702000026D7D786B12B3D5B4180280028072E5D0
:1070300030041270C8B4FF0C12C7FAE530B41D0258
:1070400080E1805D12B01A60030270A185303105C5
:1070500030E53012C3E1547FC52F5480452FF52F02
:10706000803F026D7D12E13B12D91812C5C674092A
:1070700012AC2612071EC22A742412AC266002D259
:107080002AC22712E1FC12DA06C247C227C245D241
:10709000AFC28D758CB7758AA8D28CD2A9D2ACD26A
:1070A000AAE53012CD8DE52F5403700778BB75F03B
:1070B00008800978BB742DF60875F00712DE6F1290
:1070C000DD12307C9D026FE4B4010412713A22B4E7
:1070D000010412713A22B4020412713222B4020481
:1070E00012713222B4080412712A22B40F041271F0
:1070F0001222B4070412711222B41E0412C36122B8
:10710000B4230412711A2274FF22C020C20774072C
:10711000802EC020C20774068026C020C2077409D2
:10712000801EC020C20774088016C020C2077405E4
:10713000800EC020C20774048006C020D2077400ED
:10714000C0E012C3527C0012DFEF797975F00612AD
:10715000DFE5786B797975F006E667700F0809D579
:10716000F0F7D0E004200701E4D02022D0E030077F
:107170000705E0B4040040C874FFD0202275A88041
:107180007581C47580FF7590FF75A0F075B0DF75CF
:107190008921758825C2D3C2D4E5BF441075F6870E
:1071A00075F659F5BF75F600E412D86912D869E58D
:1071B0008720E42290A57D12A4B775F00AC0F012D2
:1071C000C7FA740CC0E0E412D869D0E0D5E0F5D07D
:1071D000F0D5F0E980FEC2E4F5877808E4F608B857
:1071E00000FBF875F00012E08912E1F990816C1251
:1071F000A4B7120CC4120C63120B97D23079181278
:10720000A88CF532792C12A88CF517453270030240
:1072100072A8752000E532B4A00AE517B4A00302F5
:107220007292803AE517B4A00280370520E532B4A7
:10723000AA0AE517B4AA030272928022E517B4AA3B
:1072400002801F0520E532B4A50AE517B4A50302A4
:107250007292800AE517B4A502800702729279192A
:107260008002792D78887F0075F01212A88CF6F4D0
:107270002FFF0809D5F0F412A88C6F601B0520E5DC
:1072800020B403004003027292B4010302722D0283
:107290007245788876FF80107888E6B41900400837
:1072A000B41C0050030274FB12D7EBD2AF7F641200
:1072B000C2767008D5E0FDD5E0FDDFF3F530B419F6
:1072C00002802412C2C0601212D7EBD2AF74061231
:1072D000A94C12C9C260F602736212D7EBD2AF1288
:1072E000C9C270030273BC751700802912C2766090
:1072F000FBB418028036B41C0D12C9C270030273AD
:10730000BC12C7FA80E6B417F80517E517B40500F4
:10731000400375170078BB9082C975F00812DE6FC4
:1073200078C1E5172430F612DD1280C0E517700F22
:1073300012D80012CC6712C4B478887600806F121D
:10734000E13BE517B4010812A70712CC67805FB4D0
:10735000020512DC038044B4030512C22B804FB433
:1073600004B090817312A4B7129ECF700A12C2C0EB
:10737000700512E2026008740512A94C0273121221
:10738000D93E12D54512C22B12C8A912A70712D88E
:107390000012CC6712C4B47888E4F612AB7290067F
:1073A000007C0012DFEF797975F00712DFD1908150
:1073B0009112A4B712C27660FB0273127888E6B409
:1073C000FF07740912A94C80FE79371243AFC0E061
:1073D000601012A94C783775F00C743012D96475AE
:1073E000170112C4FAD0E0601DB43E028018781E66
:1073F000E4F208743F75F00C12D964791E12C5834B
:1074000012E1330274D6754A007983124A8F6005FF
:10741000B4350F8008124B7A600DB43605124B2735
:10742000600512A94C80FE054AE54AB4030040D924
:10743000741212AC26120703C22A742412AC2660FE
:1074400002D22A12C007C0E0791E12C58312E133AE
:10745000D0E07003027491B43902800312A94CC2C7
:107460002412D0E1600612C7FA12AA08786B12D271
:10747000DE786B12D06B601612C7FAE4F520FDFEC1
:10748000FF129FB3B418F1790512DAD880DE0274C6
:10749000D6786B12C98B796B12CEC3700F79847852
:1074A0006E75F00312DFB312D50D500A12C7FAC27F
:1074B0002412AA0870F6786B12D2DE786B12D06BA9
:1074C000601412C7FAE4FDFEFF129FB3B418F379FB
:1074D0000512DAD880E012CA9B600612A94C12CCC1
:1074E00067742512AC26600BD27FE530B42C0CC239
:1074F0007F8008C22412C68D12C1E0C0A875A88082
:1075000012D91812C5C67988E7602FB4200040034D
:1075100002729290566F1204E47988E71475F002B3
:10752000A424CCF582E434C6F583E493F5F0740129
:1075300093F58285F083E4D0A873D0A8E402832A6F
:10754000C24890814012A4B712D61D60FB12DBF630
:1075500012DAC912C27660FBB41C03027870B41848
:1075600002800302765590814412A4B712C276605D
:10757000FBB41C0302785D6418600512C7FA80EC46
:10758000C0A875A88012E00B12DFEF12B53864AA0C
:107590006007D0A8742002786274CC12B9B678085B
:1075A000E212B9B6850C12850D13850E1474AA1259
:1075B000B9B612E13378F1E2B401507889790F75E8
:1075C000F00312CD5579887407F712DC1D8018126C
:1075D000DA06C2AC9080BC12A4B712C64C60084355
:1075E000A88212A94C80E878807403F208740EF225
:1075F00012DF09E4128FB56008B420D312A94C80C1
:10760000FE7884798C75F00C12DFA912DF1390518B
:107610006F1204E4740312AC262403F5F0120C7C00
:1076200078F1E2B4031FC0A8C2AC78807402F208FB
:107630007406F208E4F278007480F278017403F2C0
:1076400012C86FD0A812DBCFE4F515782FF2C2195B
:10765000D0A8027856B41702800612C7FA027553F2
:1076600012D681700812C7FA741C02786212BCF537
:107670004005741902786212DBB512DFEF12B538DB
:10768000B4AAE212B538F516B4A1030276DAB4A3AF
:10769000030276ABB4B6030277CDB4B7030277C763
:1076A00012C7FA12DFF9741C0278627516A812BBB1
:1076B0002BF5F0798412DFDB781279A875F00C12C3
:1076C000DE59788374A8F20812DBA8F212C46E9017
:1076D00051E51204E412BE5B802C12BB2BF5F0794D
:1076E0008412DFDB74A67811F27812798575F00CBC
:1076F00012DE5974A67883F20812DBA8F212C46E67
:107700009051E51204E412D6E07827797B12E1ACBF
:10771000E516B4A1028001E4129BDA7837792712CA
:10772000DCC6781CE2600A1412E143F8792712DC07
:10773000C6E51612BB2B040412D8CC12DBB512DF3F
:10774000EF12B538B4AA0302774F742002786212A0
:10775000B53860F6B4FF028015F51612BB2B60EA4F
:10776000E516B4B10302777CB4B203027778905186
:10777000881204E4E402787074B4800274B37883ED
:10778000F2E51612BB2BF5F0798412DFDB12DBA8D1
:107790007884F212C46E7983E3783E7987B4B402B8
:1077A000784512DC9F788CE260181475F007A424E9
:1077B0004CF87983E37987B4B30512DC4480031273
:1077C000DC9F12B35780A774B9C207800474B8D283
:1077D00007F5167883F212BB2BF5F0798412DFDB04
:1077E00012DBA87884F212C46E12DCFA751600E57A
:1077F0001612E143F812E04A6032788A798512E184
:10780000B27891793012E1B2E51612E143F9789A33
:1078100012E1B212C39AE51612E143F87983E379D3
:107820007AB4B80512DDA2800312DCB90516E5169C
:10783000B4050040BA7983E37985783EB4B902781B
:107840004512DCC69051E51204E412B357905188FA
:107850001204E475150512DFF9E402787012C7FA14
:10786000741B600CC0E012A94CD0E0B4200280F27E
:1078700012AABE7930740112E00212DBDCC221C20E
:1078800020C223753200023052752000780475F052
:107890002012E089C20012DBF678BB744330000688
:1078A000744DF608744FF6786B75F00412E11B8086
:1078B0000512C7FA80E0796B7C047D047E047F00AA
:1078C0007414128E34B41C0280CCB41503027B8570
:1078D000B418DE796B12A20E50D7781C30000278F3
:1078E00005796B75F00212DFA930000F791C786BF7
:1078F000D3E3960809E396400780B6D20002789653
:107900009080F912A4B712C27660FBB418028016F8
:10791000B417028015B41503027B85B42003027BE3
:107920008512C7FA80E0D2068002C2069081131247
:10793000A4B7D204754A02124C47791C78BB75F083
:107940000312DE5978BB20070512486D80031248E8
:10795000656023B4381A9050BA1204E475F0051229
:107960000C7C90819812A4B712C27660FB027B85D2
:1079700012A94C027B85124CE479201247EB792046
:10798000124C33600612A94C027B85200707792030
:1079900012A2178005792212A2314003027956758E
:1079A000F003120C7C12B762740A12AC2612071E86
:1079B0009057441204E4790012E14A790075155A8F
:1079C00075170012C60978889056FB75F01812DEFC
:1079D0006F200722791C788B7C047D00740275F07F
:1079E0000212DD5A790578987C047D00740275F0E6
:1079F0000212DD5A800E788A791C12DE907898790E
:107A00000512DE9012050875F001120C7C7410123C
:107A1000AC2612071E7809794C75F00312DFA9789D
:107A200008E520F212A1A9601180FE7809794C7551
:107A3000F00312DFA97808E520F279047414F31238
:107A40009DD8790912A240C200754A0212493C60D1
:107A500012B43803027B20B43C04D200800512A982
:107A60004C80FE124CE47809794C75F00312DFA9C2
:107A700079201247EB7920124C3370E22000372036
:107A80000707792012A2178005792212A23140033C
:107A9000027B20786B790E12E1B2786B792512DDCA
:107AA00096500990571F1204E4027B20780E796BE0
:107AB00075F00712DFA9780CE22401D4F208E23451
:107AC00000D4F230064B788890570B75F01812DE10
:107AD0006F7920788E7C047D00740275F00212DDCF
:107AE0005A7894792212DE90120508788812DCE028
:107AF0007891792512DB237888743DF60874851215
:107B0000D9E31205083000099057A41204E4120CBE
:107B100079124CDD1247EB124CF6124CE4027A2B30
:107B200079047415F3129DD8788890571175F01860
:107B300012DE6F7896790C7C047D00740275F00279
:107B400012DD5A12050878889051B975F01812DEC6
:107B50006F7891790E12DB2312050879047416F3FD
:107B6000129DD8796B12D179796B12D44379047450
:107B700017F3129DD8786B12C98B786E12D2DE1271
:107B8000D10712C4B4027065434D5041B83F005450
:107B90004F384150200059434C593E55004843004E
:107BA000483E0048432055434D30CD004845204FC6
:107BB00046462D4C004D5943544F00484554204DE6
:107BC0004543D4004F433E2036413341004D4F558D
:107BD00043CBA0A0004B4F7D3D00484133383D00D2
:107BE000D53D00483E3D0043453D00504C553D00CD
:107BF000457D20312D303D003341B6312D303D00E3
:107C0000597D20312D303D004D4FB8312D303D0094
:107C1000484520304D5000384820312D303D00433C
:107C200054253D00464F4E543D00435450004D50A6
:107C30003E204834004D503E203034004D503E2010
:107C40004D415000332D542D593D00D50020203397
:107C5000414B500020202020D1CED1D2CEDFCDC844
:107C6000C520D1C5CAD6C8C900CEC3D02ED63A00C9
:107C7000C7C0CAD0DBD2C000D2CEC2C0D0DB00D3D6
:107C8000D1CBD3C3C8002020202020C7C0C3CECB77
:107C9000CEC2CECA20D7C5CAC0002020202020CE08
:107CA000CACECDD7C0CDC8C520D7C5CAC000CFC0A9
:107CB000D0CECBC800CAC0D1D1C8D000582DCED2AA
:107CC000D7C5D2005A2DCED2D7C5D200D1CFD0C081
:107CD000C2CED7CDC8CAC800CFD0CEC3D0C0CCCCBE
:107CE000C8D0CEC2C0CDC8C500DDCACBC7002020D9
:107CF0002020202020202020C1C0C7C020D2CEC2FA
:107D0000C0D0CEC2002020202020202020202020F3
:107D1000C1C0C7C020D3D1CBD3C300202020202096
:107D20002020202020202020CFD3D1D2C000CDC3BE
:107D300000D6C5CDC03A00D1C5CAD6C8DF3A00D8F2
:107D4000CA3A00C5C42E3D00C2C5D100D8D22E000B
:107D50003CEDE0E7E2E0EDE8FF20EDE5F23E00205B
:107D6000202020CED2D7C5D200CFCE20D2CEC2C0C6
:107D7000D0C0CC00CFCE20D3D1CBD3C3C0CC002039
:107D8000202020202020D120C3C0D8C5CDC8C5CCFC
:107D9000002020202020CFD0CEC4C0C62FD3D1CBEE
:107DA000D3C320CDC520C1DBCBCE210020CFD0CE88
:107DB000C4C0CDCE3A00202020202020C1C0C7C0A2
:107DC00020CDC0CBCEC3CEC200CDC0CBCEC300CD64
:107DD000C0D72E00C2DBC42E00CDC520CECFD0C56B
:107DE000C4C5CBC5CD0020202020CDC0CBCEC3CE76
:107DF000C2DBC520C3D0D3CFCFDB002020CFCEC77E
:107E0000C8D6C8DF2020202D0020202020C2CACBC9
:107E100020CFCEC72E3A0020202020D2C0C1CBC810
:107E2000D6C020D1C8CCC2CECBCEC200784A75F025
:107E30000E12E11B755401C2009082D630000390EF
:107E400082DD12E12B79797C057D037E037F00744E
:107E500014128E34B418028016B41C03027065B478
:107E6000110830000575540A800512C7FA80CA78D7
:107E700079E612D7AAFF08E6B40300502575F0642E
:107E8000A42F401E30000B6019B4FB005014F54CB9
:107E90008015B40200400BB4F1005006F54DD2003D
:107EA000809712C7FA809E75F005120C7C1204CEE2
:107EB00090587B1204E41204CE754A00122E51052C
:107EC0004BE54BD3954C40439058911204E4C219B2
:107ED000786B12C98B786E12D2DE12D10712D7EBF3
:107EE000D2AF9081913019039082E712A4B7753216
:107EF000FA12C7FA7406C0E012C276700B12D86983
:107F0000D0E0D5E0F1D532E902706512DBF690825F
:107F1000E312E12BE54B78C212D04212DD127888D1
:107F200090589F75F01812DE6F788DE54B12D04295
:107F300078921280855003027FD8120508784F7915
:107F40007C75F00212CD5575F00012C2C0700A1295
:107F5000E202700512E20460089058337405028052
:107F600021122DE06007D223D22202805B780079B3
:107F70004A75F00E12DFA9D2071201B2C0E0784AAA
:107F8000790075F00E12DFB3D0E0600302805BE58C
:107F900054C0E01200FED0E0D5E0F6E54A1280744D
:107FA00078BB75F00812BC9AE54A60167408C39550
:107FB0004A24BBF8854AF0908069E493F608A3D57B
:107FC000F0F8054AE54AB40A004003754A0012DD9C
:107FD00012785112D2DE500890584B74030280215F
:107FE000E551C3954F60187460C3955012D8A5121F
:107FF000D7AA254EF54EE55212D7AA254E800DC3BD
:10800000E552955012D8A512D7AA254EF54E8551A6
:108010004F855250E54EB54D004014754E00027E1E
:10802000BF1204E49058A41204E4D219027ED07561
:10803000F00079371243AF60069058630280211236
:10804000D7EBD2AF758200758304D5E0FDD582FAF7
:10805000D583F712C276600EB4150B9058A41204A3
:10806000E4D219027ED0027F9BB0B1B2B3B4B5B6F0
:10807000B7B8B900B40A00400274002469F582E47C
:108080003480F58322E8C0E0787912C98B40077804
:108090007C12D2DE5003D0E022D0E0C0E0F8797943
:1080A00012CA65D0E02409F8797C12DE85C3224625
:1080B000756E004D4550457D4134410050453E2090
:1080C00043455038005045724D5900342D504143BE
:1080D0004D453400454C2034C53F00454C204C45AF
:1080E000C83F00454C2055C33F00454C432048EF56
:1080F0003F00454C4320FD3F00204D4F2D43CF3FD7
:10810000007D313D007D323D00B043B03F00B04DB9
:10811000B03F00204D504F3820334D00D0504136F5
:10812000002020202D2D2D004D4550454D45B43FBC
:108130000020504143344574002020204D45340038
:108140004148480041484820B43F0043C53F0048EB
:10815000BE3F003830333850002D2D002B2D003815
:10816000627C4D00384845430036480020204D5081
:108170004F3800435B50C3204F335900435B504F8F
:10818000C33F003341CD3F00204845424550484F52
:1081900000202020484F500020484520484F5000E4
:1081A0002020202D2D2D004F4D7F7F7F7F7F7F0052
:1081B0004F3E7F7F7F7F7F7F004F433E31004F43A5
:1081C0003E32004F433E33004F433E34004F433E68
:1081D00035004F367F7F7F7F7F7F004F363E3100F7
:1081E0004F363E32004F363E33004F363E34004F5E
:1081F000363E35004F363E36004F334D31004F335B
:108200004D32004F334D33004F484D34004D507FB9
:108210007F7F7F7F7F004D503E207D004D503E2070
:10822000304D004D503E20434500334D7F7F7F7FD2
:108230007F7F00454C7F7F7F7F7F7F0043507F7F24
:108240007F7F7F7F004D504F38205043004D504F6F
:10825000B8434B41004D504F3820334D004D504FE7
:1082600038204D590059432038384F7D41004D503A
:108270003E2033C83F0050453E20334D0050453E20
:1082800020454C004D504F3820454C003320415084
:1082900020454C005041B62E2E00202020202048A2
:1082A0004F50002020204845484F5000332D334187
:1082B0004D55434200504800554848004D00C34FBB
:1082C0004D004D50BE4D415000434C454172004D54
:1082D000504F3E4F48004D4550553064003843459F
:1082E0003E3000486FD5002020453E3E303E0043E2
:1082F00036D033CD3332004336D033CD3634004D13
:10830000503E204F4D45004D503E207D4F004120B6
:108310007F7F7F7F7F7F004D003E004D504F3E208E
:1083200030002D4330002D363E00C0A875A880C017
:10833000E075200070030283397809E4F208B86F11
:108340000040F8D0E0C0E0B4080A781E798875F0E3
:108350000F12DFA912CB0570107981E7F50F09E73D
:10836000F51009E7F5110283BFB4030512A94C808B
:10837000FE9081A012A4B712D599D2007003028397
:1083800099B4200280E6B41F03028407B44505D2E5
:1083900002028407D201028407750F00751022754E
:1083A000110012CB3A700512CC67600302836CD0C7
:1083B000E0B40200400412C4B4E4C0E00284F5D387
:1083C0007400950F7422951074009511500512E0F9
:1083D0009B400B200003028371742002836C79811F
:1083E000E7FD09E7FE09E7FF787975F00C12E11B5C
:1083F00012DD36C0E0E56B456C456D7005D0E002DE
:108400008371D0E002837CE56B456C456D600E1294
:10841000852412CB3A600302836C128524D0E0C01D
:10842000E06037787975F00CE44608D5F0FB70020F
:10843000D2037883797975F00D12DFA9782E797AD5
:10844000E7F209780975F00412DFA9D0E0C0E0B4C2
:108450000200400678087985E7F230014474FF1283
:10846000CC9774CC12B9B67808E212B9B6850C0F65
:10847000850D10850E1112DF0974AA12B9B612E12A
:108480003390516F1204E475F003120C7CD202D0C9
:10849000E0B402004009B40700500412C4B4E4C0C0
:1084A000E0D0E0C0E030020DB40200400812C4B4D5
:1084B000D0E0E4C0E0B402004005B40A004003028A
:1084C00084F5E56B456C456D700B12C4B4D0E0E4E7
:1084D000C0E00284F5AD6BAE6CAF6D12DD2A6005B5
:1084E000742002836C7837798B12E1A6856B0F8537
:1084F0006C10856D11D0E0D0A87003026D51B401ED
:1085000003022F2CB402030240D4B4030302413708
:10851000B4060302415DB407030275CFB409030238
:1085200041AC80FEE56BC50FF56BE56CC510F56CD5
:10853000E56DC511F56D22C0A8C0D0C0E0C0F0C087
:1085400083C082E8C0E0E9C0E0C2AF1098030287B0
:108550001EE599202CF8B47F030285EB20450280AC
:10856000ED758200B40202800CB430024005B43ACA
:1085700000400280D9F58379CE7499F309758201A0
:10858000E583B40230E4F583109808D5E0FAD5838A
:10859000F78037E599B430004005B43A004016B48E
:1085A0000302802AB40D23E4F583109821D5E0FA64
:1085B000D583F78019F58374CE2582F9E583F30519
:1085C00082E582B41400500280BB79CD8010202A4D
:1085D00005740112E1F674CE2582F97414F309B919
:1085E000E200400302871EE4F380F312E188400BAF
:1085F00030470B12DB9A74C012CD2602871EF8C2D8
:10860000E4B4CF028003B4CC0612DF6D02871EB43F
:10861000C502800754C0B48030803112DB9A74C523
:1086200012CD2612B4504077F854C06480601DE823
:10863000C2E4B4C0028012B4CC028003B4CF0512ED
:10864000DF6D800574C312CD2602871EC24612D983
:108650002B404CB47F02D246798075820012D92B10
:10866000403D304621B403028030B41006747FC20E
:1086700046801AB9CE005027C0E0747FF32582F5FA
:108680008209C246D0E0B47F04D24680D0B9E2006D
:10869000500DF3092582F58280C312D92B50028038
:1086A0007D2582603674C612CD2612B450406FF814
:1086B00054C0B480028095E8C2E4B4CF02805FB4B5
:1086C000C002805A12DB9AB4CC0A12DF6D74CC124D
:1086D000CD2680D674C312CD268043E85407F5F02A
:1086E000E51A540765F0600A74CC12CD2612DF6DCE
:1086F00080B8051AE8A2E49244400874CA12DB9AD2
:1087000012CD267980E3B401097487C0E074BBC040
:10871000E032B402097409C0E074BFC0E032C2990B
:10872000D0E0F9D0E0F8D082D083D0F0D0E0D0D043
:10873000D0A832740512AC26908322600390832661
:1087400012A4B712D61D60FB64186003026D7D127F
:10875000C27612D0E160028005120BB7600612A942
:108760004C026D7D90813912A4B7740512AC26605D
:108770000B12D99B6003B445E502271BC21B740290
:1087800075F00002683212C4B4E53104F53012C34A
:10879000E1547FC52F5480452FF52F02706500AF3F
:1087A00081A72F0C00A081B00000010F81B9E01D4E
:1087B000013881BEE02F013881C3E038012881C82B
:1087C0002729012881CD271B00A081D20000012884
:1087D00081DBE026012881E0593E012881E5E04166
:1087E000012881EA2730012881EF2722012881F41E
:1087F000A7CB0003820D000001188216D5CF01A877
:10880000821C892C01B882231E8901B87C2E1CFD94
:1088100001B87C351CF801B882FF1CF301B883074E
:108820001CEE01A87C3C21CF1100000099B3010887
:108830007B8F28C601087B9628C101987B9D14F286
:1088400001987BA012280100826E445300B0822A56
:108850000000017881F9BE03017881FE78890178F2
:108860008203A16F013D827644590000823C0000E2
:10887000010082BE9110018082C2CDB301A082CFDF
:108880007E2C01008265E18E0100825DE194010091
:108890008255E0DB01008245E0CB0100824DE0D350
:1088A000010082EF2E75010082F72E71EE00AF817C
:1088B000A72F0C00A0830E00000108831BD57D119B
:1088C000000000873301288317E026010F8319E099
:1088D0001D0003820D000001188216D5CF01A88269
:1088E0001C892C01B882231E8901B87C2E1CFD0135
:1088F000B87C351CF801B882FF1CF301B883071C53
:10890000EE01A87C3C21CF1100000099B301087B47
:108910008F28C601087B9628C101987B9D14F2011F
:10892000987BA012280100826E4453EE752300123A
:10893000D99B6012B42304D21F800BB44502800679
:1089400012A94C0270657C0090030012DFEF7911D0
:1089500075F02612DFDB756B01E56B1475F003A46F
:108960002467F58274AC35F0F58375F003786D12E9
:10897000DF9FE56B142411F8E2F56C12DBF678BB8F
:10898000744FF608744DF6E56B78BE12D04278C18C
:10899000E56C12D04212DD1212C27660FBB43A13BB
:1089A00012CF9BB4070512B1C780EDB408EA1200DC
:1089B0006180E5B4120EE56BB40200500280D91557
:1089C0006B028959B4130EE56BB42600400280C8CF
:1089D000056B028959B4170280EDB4192D301F08B8
:1089E000742312A94C02897B90817C12A4B712C215
:1089F0007660FBB41C0302897BB418F2781190AC4A
:108A00004175F02612DE4E028956B41C03028956C7
:108A1000B41139787975F00212E11B7C037D027E76
:108A2000027F0079797B027410128E34B420030225
:108A3000897B7979E7700302897B12D7AAB4270072
:108A4000400512C7FA80CCF56B028959B4185DE570
:108A50006D30E70B301F08742312A94C02897B7814
:108A6000C0743DF67879E4F608F67C067D027E0255
:108A70007F0079797410128E346418600302897B48
:108A80007979E712D7AAF533E56ED39533500AE525
:108A90006F04C533B53300400512C7FA80C6F56CC4
:108AA000E56B142411F8E56CF2028959B4152A908B
:108AB000818312A4B712C27660FBB41C03027065F6
:108AC000B418F27C0090030012DFEF791175F026E4
:108AD00012DFC712E133027065B42008E56D30E69D
:108AE00003E480BA12C7FA028998740912A94C707B
:108AF000F912C4B402717D7989E7F58209E7F5833B
:108B000009E7FC12DFEF12B538B4AA1A12B538B46F
:108B1000CA14788C75F00C12B538FFE66F70070830
:108B2000D5F0F4028B4F7989E7F58209E7F58309DF
:108B3000E7FC12DFEF74AA12B9B674CA12B9B6799B
:108B40008C75F00C12DFD174AA12B9B612E1337829
:108B500098E6F516740202832A780C798975F00874
:108B600012DEC3600512A94C80FE740302832A74CE
:108B70000602832A740702832A7891798975F0079F
:108B800012DFA9740902832A7989780F75F0061219
:108B9000CD557990E7F52009E7F51709E7F51509AF
:108BA000E7F51609E7F53209E7C0E009E7F52A0914
:108BB000E7F52909E7F52380197989E7F52009E721
:108BC000F51709E7C0E009E7F52A09E7F52909E7FC
:108BD000F5239081A012A4B7740F12AC2612071EC1
:108BE0007988E7B40B030268B80269117989E7C094
:108BF000E009E7F51709E7F5159081A012A4B7740D
:108C00001012AC2612071E798CE7F52009E7F52A29
:108C100009E7F58209E7F583E473E4C0E075155AC6
:108C20009081A012A4B77988E7B40E03025DE2B484
:108C30000F03025E1BB41003025E45B41103025E13
:108C4000C6B41203025F2580FE7804798875F0119E
:108C500012DFA97908E3F5207904E3B41403027A5A
:108C600042B41503027B28B41603027B63B41703D6
:108C7000027B75028AEA75301D90822A12A4B7120F
:108C8000C27660FB02702302466F0247067889E6CF
:108C9000F54A08E6F54C0227F975A880781E798117
:108CA00075F00312DFA97802790F75F00612DFA9BB
:108CB000D2077862791E75F00312DFB3800AE517D8
:108CC00012BB2B2402128E21856282856383AC64E1
:108CD00012DFEF12B538B4AA0A12B538F51712BB75
:108CE0002B7007742012A94C80FE200703028D8D83
:108CF000E517B4C903028D3EB4CA03028D23B4CB79
:108D0000028003B4CCB8741AD2A912A94C780F7996
:108D10000275F00612DFB312DBDC12DBF612DAC9E1
:108D200002424BC207851282851383AC1412DFEF17
:108D300012B538B4AA028003028CE3028CB2E517A4
:108D40007983F30912BB2B04F5F012DFDB7985E39D
:108D50006008B404005003028D067827798612E17A
:108D60009A7879790C75F00712DEEB5005740302DE
:108D70008CE57879798612DD9650057424028D0889
:108D80007889796275F00312CD55028CBEC206E572
:108D900017B4A103028DD9B4A303028DD9B4A502DF
:108DA0008037B4A6028032B4A802802DB4AB028012
:108DB00028B4B5028023B4B602801EB4B70280196D
:108DC000B4B8028014B4B902800FB4C902800AB4E6
:108DD000CA04D2068045028CE3E5177983F30912B1
:108DE000BB2BF5F012DFDB851282851383AC1412E6
:108DF000DFEF12B538B4AA028003028CE3E5171244
:108E0000BB2B04F5F0798312DFC7850C12850D1397
:108E1000850E1474AA12B9B6028CBE12D49A0240FE
:108E200067C0E02562F562E43563F563E43564F517
:108E300064D0E022C020541C4401F520893520056F
:108E40000B128FAFF5F0E4F709D5F0FB8D37EC2D61
:108E5000B409004004B3028FAC74BB2CF536200576
:108E6000117A00300307D207EFFB028FA77B0002C5
:108E70008F70128FAFF5F01429F9E5F0C333F5F0D8
:108E8000E730F003198001C4540F7003D5F0F1AA44
:108E9000F0EFFB300305D207028FA7028F7012E1BB
:108EA0006DB4990280F8B420062002F2028FACB4AF
:108EB0001C3C300203028FACBB000310072DBA002C
:108EC00003028EF3A935128FAFF5F02914F978005B
:108ED000E754F048C4C7540FF819D5F0F31A30031B
:108EE00003028FA7BB0003028F701B028F70B41B9D
:108EF00015800612C7FA028E9E200705D207028F40
:108F000070741B028FAC12DA594003028FACF8BAAE
:108F100000117009200303200709028E9EB40A0382
:108F2000028E9EB40A03D206C3B3EA9E400612C75D
:108F3000FA028E9E20030C300709B80A01C3B3EB76
:108F40009F50EBB80A027800EE04C313F5F0A93580
:108F5000E7C454F048C7C4540FF809D5F0F2300301
:108F6000070A1006DE028FA70A3007010B1006D38E
:108F7000EA300706D39B5002EB04E537FCEBFD1209
:108F80008FAFF5F0A836A935E52054F8440912A6AC
:108F90004230070DBB000AE536253714F8E6448059
:108FA000F612DD12028E9EAC37EF80D2D02022EE78
:108FB000C313340022C0A875A880C020F520C016B5
:108FC000C2067982E4F375340312E00B12DFEF126C
:108FD000B538B4AA02800574200290F812B5386042
:108FE000F6B4FF12E516B4CA028008B4CC028003BE
:108FF000B4CBE402909CF51612BB2B700280D8F51E
:10900000F0E516B4A3028017B4A5028012B4A8023A
:10901000800DB4AB028008B4AD028003B4AE36E577
:10902000F0C394202534B45E00400675160002900B
:109030009C74802534F9E516F30975F00412DFDB22
:10904000742012CC9775F00D12DFDBE51612BB2BE6
:10905000C3941E8023E5F02534B45E0040057516E8
:1090600000803974802534F9E516F30905F012DF24
:10907000DBE51612BB2B04042534F534E51612BBD0
:109080002B040412D5EAE516B4CA02800FB4CC0250
:10909000800AB4CB028005028FC9C206D244E5160D
:1090A000B4CA028008B4CC028003B4CB02C24478B4
:1090B000007480F27801E534F230060512C89F8012
:1090C0000312AED65016300702802DB44902800339
:1090D000B448C712DF0912DB9A028FC2A24492067B
:1090E000E516B4CA028010B4CC02800BB4CB028067
:1090F0000612DB9A028FC2E4C0E079CE75F014E468
:10910000F309D5F0FAD0E0C244D020D016D0A8227E
:109110009020807C0012DFEF796B75F00D12DFE597
:10912000786B75F00D12E05C700A786F75F006745C
:109130003012E12375170012DBF678BBE517700CCF
:109140007431F60808796B12D3458033B401117479
:1091500045F6087472F6796EE778C112D042801F26
:10916000B4020F744DF60808796F75F00612CD55EC
:10917000800D7517037432F60808797512D34512FD
:10918000DD1212C27660FBB4200B786B75F00D1205
:10919000E11B029254B4170F0517E517B404004001
:1091A00003751700029137B41102800BB415030246
:1091B000924012C7FA80CBE5177008AD6BAE6CAF6A
:1091C0006D805BB4013178C0743DF679887C067D92
:1091D000027E027F007414128E34B418147888E66C
:1091E00012D7AAB416004009B435005004F56E80B9
:1091F0000312C7FA029137B4021A78BC743DF878AA
:109200008812E092B4180A786F798875F00612CD4A
:10921000550291377875E6FD08E6FE08E6FF78BC52
:10922000743DF61294FD64186003029137786BE583
:109230001760027875790575F00312CD55029137E4
:1092400090818312A4B712C27660FBB41C03027033
:1092500065B418F29020807C0012DFEF796B75F016
:109260000D12DFD112E133027065C020C017C016A5
:10927000E9C0E0788875F01E12E11B797975F0037A
:10928000E77003098014B4060050157403C395F009
:109290001293B1F8E7F60809E7F609D5F0E2800580
:1092A00074320293A6751700E5171293B1F8E670B1
:1092B00003029399797912E17464AA600574320209
:1092C00093A6E5171293B12402F87979E7F60978A5
:1092D000A675F00212CD55D0E0C0E0F9786B12E12E
:1092E000B2751600E516B5170040030293321293CB
:1092F000B1F9E760310909E7C2076002D20709E561
:10930000171293B105E0F8E6C3138516F005F0C314
:1093100013D5F0FB786B500820070B12DB41800659
:1093200030070312DDC60516E516B403005003022C
:1093300092E4787212DDDE7872797A75F00212CDDD
:1093400055786B797212DB5012DBE9786B797A759C
:10935000F00712CD55787212DDDE78747401F6E5EF
:10936000171293B12402F9E76015787279A675F0A7
:1093700002C3E736D4F60809D5F0F7E436D4F67818
:109380006B797212E07712DBE9E5161293B12403D0
:10939000F8797A75F00712CD550517E517B4030073
:1093A00050030292A8E4C9D0E0C9D016D017D0204B
:1093B00022C0F075F00AA42488D0F022C0A8C2AF61
:1093C000C0D0C0E0C0F0C083C082E8C0E0129458B2
:1093D0004074304571202C6EF5F078CEE27067E570
:1093E000F0B4020878CE7499F2088016B4300040C8
:1093F00025B43A005020F5F078CE7499F208E5F0E3
:10940000F208129469400FB430004014B43A00508E
:1094100005F208B8E2EC78CEE4F208B8E2FB802668
:10942000B403028003B40D028003B40AE97414F299
:1094300008E4B8E2005004F20880F7129469202A88
:1094400005740112E1F6D0E0F8D082D083D0F0D0DC
:10945000E0D0D0C28BD0A832C0F0C083C082C2D5C9
:1094600075830CD583FD02948DC0F0C083C082C289
:10947000D5E4F58230B30DD5E0FA30B307D582F4E8
:10948000D30294F420B3ED758315D583FD7583085D
:10949000A2B3000000000000000033D583F2700288
:1094A0008003D2D50075830ED583FD75F008741640
:1094B000D5E0FD758308A2B30000000000000000A5
:1094C00033D583F2F46004F4C38004000000D3E5D4
:1094D0008213F5827412D5E0FDD5F0D2740BD5E07D
:1094E000FD758308A2B30000000033D583F6F46055
:1094F00002D2D5C3E582D082D083D0F022C02075BD
:109500002000753300790578BD12D34512DD1212A3
:10951000C27660FBB4181EBF0400400DBE0002807E
:1095200008BD0002800302960E7D007E007F0012BF
:10953000C7FA0294FFB41C0302960EB413030295FB
:10954000FFB4200302960EB41210AC33BC000675B3
:109550003305029505153302950512DA59400302C9
:10956000950FF5F0AC33BC0010E5F0B404030295A0
:10957000F8ED12962BFD0295FFBC0110ED1296320C
:10958000B4320040030295F8FD0295FFBC0212E5DB
:10959000F0B4020040030295F8EE12962BFE0295FD
:1095A000FFBC0310EE129632B4130040030295F88C
:1095B000FE0295FFBC0408EF12962BFF0295FFBC3C
:1095C0000534EF129632FFEF12D7AAB4040050030D
:1095D0000295F875F00484E5F090961E700390965D
:1095E00011EE12D7AA93C39D501512C7FA7D007EC3
:1095F000007F000294FF7C0012C7FA1C02950F0541
:1096000033AC33BC06004003753300029505D0200F
:1096100022003129313031303131303130310031B7
:109620002831303130313130313031C454F045F0EF
:10963000C42254F045F022303E39C0E0C0F0C0D022
:10964000C28CC28D30341D741475F05DA4C3C58AFC
:1096500074FF958AC58A74FF95F0F58CC234D28C5C
:10966000D2A68008C234D2A6C23EC2A9D0D0D0F0C1
:10967000D0E032202C4A303747C0A8C2AFC0E0C08B
:10968000D0753B10753E05753F72120AC5D2CA30BF
:10969000CFFDD53FF5D53EEFC2CFC2CA75CDDB7544
:1096A000CCD3D2CA30CFFD120B9353A0F0751C005F
:1096B000D23012CFE21538C237D0D0D0E0D0A832A5
:1096C000C0A8C2A9C0D0C0E0E8C0E0C0F0C082E538
:1096D0001E531EF0540F04B40A005005421E029798
:1096E0001B303012E51C04B40400400BE420930648
:1096F000D5E0FA120C45E4F51CE51E531E0F54F09C
:10970000C404B40A005006C4421E02971BD22905A5
:109710001DE51DB43C004003751D0012BFB3602C55
:10972000D22C754801B4CE02802212CFC5F5F0B418
:109730000104D237801653A8F978CEE27005E5F01F
:10974000F2800908B8E20040F275480F302C102072
:109750002A07E54812E1F68000C2B5C22CC22F12DA
:10976000CFE2D082D0F0D0E0F8D0E0D0D0D0A83294
:10977000C0A875A88075F014E41297B3D5F0F974F9
:10978000031297B31875F0061297ED401A20F003F4
:10979000088002C446F6D5F0EF75F00C1297ED4044
:1097A00006D5F0F830D50474278001E4C298C29938
:1097B000D0A822C0A8C2AFC0F0C0E0C2B175F0BC52
:1097C000D5F0FD75F00813C0E092B174BAD5E0FD94
:1097D000D0E0D5F0F1D0E0A2D092B174BDD5E0FDDB
:1097E000D2B175F0C8D5F0FDD0F0D0A822C0A875D0
:1097F000A880C0F0C2D5E4F5F075821420B0033023
:10980000B018D5E0F720B00330B00FD5F0EE20B09F
:109810000330B006D582E5D380441298635004D259
:10982000D58004C2D500007435D5E0FD75F008126E
:1098300098631300758234D582FDD5F0F2129863D7
:10984000400730D00BD2D5800720D004D2D50000FD
:10985000758232D582FD1298634002D2D5C3D0F012
:10986000D0A822C0F0C0E0007441D5E0FD75F0083A
:10987000A2B03300000000D5F0F6C370070000006E
:109880000000800BF46004D2D58004D30000007483
:109890001BD5E0FDD0E0D0F022C0A8C020532000AE
:1098A00075A880C0F0CEC0E0CECFC0E0CFC0E0E869
:1098B000300302E582543FFE7F05E52054707004BA
:1098C00074D0800FB4100974A2BC000774A0800388
:1098D0000299A212BF5E50127432D5E0FD12BBE3B2
:1098E0007432D5E0FDDFD30299A2E8300309E583A5
:1098F00012B95640E3E58212B95640DCE520540720
:109900006003B40306D0E0C0E08007B40103E78041
:1099100001E312B956500612BBE30299A2E52054A6
:10992000037002804B09200303088008A3E58245E9
:109930008370010CD5F00280370EEE543F70BD7F6E
:1099400065D38017D3E5829400E5839400EC9401FD
:10995000400474A2800274A012BF5EC0D012BBE3A8
:10996000D0D040030298AF7419D5E0FDDFD6803225
:109970007F65D38017D3E5829400E5839400EC944F
:1099800001400474A2800274A012BF5EC0D012BB5A
:10999000E3D0D0500E200303C380087419D5E0FD36
:1099A000DFD3D3D0E0CFD0E0CFD0E0CED0F0D02006
:1099B000D0A82278BB742DF60890811C75F0071290
:1099C000DE6F78F1E2F51778C212D04212DD121282
:1099D000D61D60FB64116003026D7D12C2761243D6
:1099E000F2700A12D99B600BB44502800612A94C92
:1099F000026D7D78C1743DF612DD1212C27660FBF5
:109A0000B41C030299C212DA5950F8B4040050F39E
:109A1000F515E51578C212D04212DD1212C2766039
:109A2000FB6418600612C7FA0299C290812112A441
:109A3000B7E52254037008750D64750E008011B4EB
:109A40000108750D7E750E008006750DED750E0012
:109A5000758200850D83AC0E74FF75F00012DEAFC9
:109A60004063050DE50D7002050EE5225403700DEF
:109A7000E50DC39480E50E940040D5801BB4010D24
:109A8000E50DC39400E50E940140C5800BE50DC3C0
:109A90009400E50E940240B8786B9000007C00754D
:109AA000F00712DED7401EE515F570256D256E25F1
:109AB0006FF571796B9000007C0075F00712DEA5E0
:109AC00040030271DA740512A94C80FE755B0575BE
:109AD0005C088859895A7879855CF0E4F608D5F0F5
:109AE000FBA95A855BF0E7700809D5F0F9D3029B12
:109AF000747A047C007D00A859A95A129B755015F0
:109B0000A859C202129B8EA859A95A129B75501BC4
:109B1000DAEE029B740AA85AD202129B8EA859A9A7
:109B20005A129B7550EFA85A129BB97B00A859A9ED
:109B30005A855BF0C3E69712D8A5F60809D5F0F56B
:109B4000EC9D12D8A5FC40030B80E2A859A95A85C8
:109B50005BF0C3E637D4F60809D5F0F7EC3DD4FC4A
:109B60007879129B837879E64BF6A859C202129B4A
:109B70008EDAB8C322855BF0C3E6970809D5F0F901
:109B8000EC9D22855BF005F005F0D2038005855B36
:109B9000F0C2037E00E6C454F04EC6C4540FFE0863
:109BA000D5F0F2200311200208ECC454F04EFC80E2
:109BB00006EDC454F04EFDEE22E55BF5F005F0280D
:109BC000F87E00EDC4540FCD8006E6C4540F4EC697
:109BD000C454F0FE18D5F0F2EE226025742112ACC8
:109BE00026601E5403601AC0E0120761F5F0748508
:109BF000788812E123D0E0C0E0120508D0E0D5E07B
:109C0000F6788812DCE0C2227894791712DB147897
:109C10009E12DB6E762A18E8C0E0C3940AF8791227
:109C20007C0B7D03740175F00512DD5AD0E0F8124B
:109C3000C059788875F01812D9D1E8C0E0791DE3D1
:109C4000788812D042764308764B782712DE1724A4
:109C500002F5F0D0E0C0E0C39490400495F05003CA
:109C6000029CA0E5F02402F5F0D0E0F9C395F0F8ED
:109C700074A0C399F5F012DB7D782712DE17240457
:109C8000F5F074A0D395F0F87927ACF07D0274015B
:109C900075F00512DD5A789E12DB6E763D029CCC83
:109CA000D0E0120508D222788812DCE07894792777
:109CB00012DB14302209789E12DB6E763D800D781F
:109CC00088791DE312D042764308764B789F791C41
:109CD000E3600424408002742DF6120508E422D2C9
:109CE0004378F1E264026005740602AE38784A797E
:109CF0008275F00212DFB3784F794A12D1C3784FE0
:109D000012CCF74005741102AE38854F828550831E
:109D10001582E582B4FF021583744012D561FC12EE
:109D2000C78312DFEF12B538B4AA02801BB4A502B4
:109D3000801630430A054FE54F70C3055080BF7948
:109D4000827409F374038013F5F07982E4F309E572
:109D5000F0F30975F03F12DFDB74437801F2204421
:109D600023780A12B4505005D8F902D905F5F0B499
:109D7000C5028010B4CC0512DF6D8008B4CF02801C
:109D80003902D90512DB9AE51B54074480A244929C
:109D9000E412CD267901E3F5F0798012C14578050A
:109DA00012B4505005D8F902D905B4C60280D5B412
:109DB000CC0512DF6D80CDB4CF0E12DF6D12DB9AB1
:109DC00074C012CD2602D905B4CA05051B02D905F7
:109DD000B4DAFA051B029D35C0A8C02075A88075AD
:109DE00020018961792C12A88C4009F5607918123C
:109DF000A88C50057403029EC4F55F700BE560B437
:109E0000A003029E3E029E46E560700BE55FB4A093
:109E100003029E46029E3EE55FB4A50CE560B4AA2F
:109E2000028023B4A0028016E560B4A50CE55FB4FF
:109E3000AA02800AB4A003800DB4AA028008D20747
:109E4000E55FC560F55F74D012BF5E50137432D504
:109E5000E0FD12BBE37464D5E0FDD582E9029EC447
:109E60007418300702742C12B95640E174A012B96C
:109E70005640DA7F00A96175F012E7300001E3F483
:109E80002FFFE7300001E312B95640C109D5F0EACF
:109E9000EF12B95640B712BBE3E560B4AA0474A54B
:109EA0008006B4A5028022E47818200702782C12DC
:109EB0009899400E74AA7818300702782C12989955
:109EC0005007740312A94C80FEC3D020D0A822C032
:109ED000A8C2A9C2AC75F00A90FFFF7C0174AA1257
:109EE000DEB95005D5F0F1801290FFFF7C0112DE43
:109EF000E140F1B4AAEE7402029F4075F00A907F2F
:109F0000FF7C00745512DEB9402790FFFF7C00747F
:109F1000AA12DEB9401B907FFF7C0012DEE14011E7
:109F2000B4551490FFFF7C0012DEE1400464AA6087
:109F30000DD5F0CA029FA864AA70F6E480027401ED
:109F40005322FC4222756BAA756C55756D0B756EAC
:109F5000C8F56F75700024D3F5719000007C00790E
:109F60006B75F00712DEA5403F7403F50A75820099
:109F7000850A83AC0B74FF75F00012DEAF40290533
:109F80000AE52254037009E50AB4800040DF801F0F
:109F9000B40106E50A70D68016E50A70D0050BE517
:109FA0000BB4020040C78007740512A94C80FEE480
:109FB000D0A82275330012DBF6790578BB12D46085
:109FC00012DD1212C27660FBB4180302A093B41B18
:109FD0000302A093B41C0302A093B4200302A09335
:109FE000B4130302A084B41210E533B40006753331
:109FF00005029FB61533029FB612DA594003029F3D
:10A00000C3F5F0AC33BC0010E5F0B4030302A07E4E
:10A01000ED12962BFD02A084BC0110ED129632B415
:10A020002400400302A07EFD02A084BC0212E5F0E1
:10A03000B40600400302A07EEE12962BFE02A0841E
:10A04000BC0310EE129632B46000400302A07EFE04
:10A0500002A084BC0412E5F0B40600400302A07E16
:10A06000EF12962BFF02A084BC0510EF129632B4BB
:10A070006000400302A07EFF02A08475330012C777
:10A08000FA029FC30533E533B4060040037533007D
:10A09000029FB62280000080A58A80000000A59261
:10A0A00080A59B00000080000000000080000000F0
:10A0B000000000000000A5AD00A5B600A5BF00A5EA
:10A0C000C800A5D100A5DA00A5E300A5EC00A5F520
:10A0D00000A5FE00A61900A62000A63000A63900A3
:10A0E0000000000000000000000000000000000070
:10A0F0000080000080000000000000A63900000081
:10A10000000000000000000000000000000000004F
:10A11000000000000000000000000000000000003F
:10A1200000000000000000800000000000000000AF
:10A13000000000000000000000000000000000001F
:10A14000000000000000000000000000000000000F
:10A150000000000000A5A400A60700A61000A5832B
:10A16000000000000000000000000000000000C22D
:10A170000775F003120C7C12B762740A12AC261237
:10A18000071E90578B2007039057721204E4751531
:10A190005A751700790012E14A790012C60912A116
:10A1A000A97003027B5B027065C020C207754A017B
:10A1B000200703754A00124C47124CE4C2001249B2
:10A1C0003C6016B43804E402A1D6B43C04D200804A
:10A1D0000812A94CE5F0D02022124CDD7920E4755C
:10A1E000F01720070375F02A124C336005B43CE1E8
:10A1F000D200792012473D3000069057A41204E4A3
:10A20000120C79124CDD1247EB124CF680ABE7D3FF
:10A21000940009E7942022C0F0EFC0E0780575F0C3
:10A2200002D3E2FFE39F0809D5F0F7D0E0FFD0F0BA
:10A2300022C9C87905124DB940037001D3C8C9229B
:10A24000E3F58209E3F58322D24378F1E264026008
:10A2500005740602AE3879ADE3B40500400302AEE2
:10A2600036784A798475F00212DFB3784F794A1252
:10A27000D1C3784F12CCF74005741102AE38854F28
:10A28000828550831582E582B4FF021583744012E3
:10A29000D561FC12C78312DFEF78B8E2F54A75F09A
:10A2A0000712E089798275F036E54AB4AA0375F0A1
:10A2B0004012DFC720430712E133E402AE3812DB5D
:10A2C0009A74CAD2E412CD26780512B4505005D83B
:10A2D000F902A316F854C0B48030798012B82F5018
:10A2E0000FB4460912DB9A74C612CD2680DA802696
:10A2F000E85407F5F0E51A540765F0700302A2561A
:10A3000012DB9A74CC12CD2680BEE8B4CC02800356
:10A31000B4CF0312DF6D12E13302D905C020532000
:10A32000F8C0F08859755B05E914F55A755C057835
:10A330007975F00E760008D5F0FAE55CC333F55C6C
:10A340007C00C202A95AEC30E008E7300001E3C407
:10A35000800809E7300001E3895A540FFEEC30E031
:10A360000114C3132479F9AD5BA859E6300101E269
:10A37000540F8EF0A475F00A84C445F0F55E755D47
:10A3800000E6300101E2C4540F8EF0A475F00A8497
:10A39000C5F0C4255ED4F55EE5F0355DD4F55DEC21
:10A3A00030E01EE55E540FC427D4F709E55E54F093
:10A3B000455DC4720237D4F7501409E437F71980A9
:10A3C0000DE7255ED4F709E77202355DD4F79202F6
:10A3D000DD0A0CECB55C00500702A3440802A36B35
:10A3E00030020609E73401D4F7D0F0D02022C02093
:10A3F000F52053200F85F065D205BD0002C205E5AA
:10A4000065C333F56630010302A447E56529F98584
:10A4100066F020F00119E7300601E320F001C45492
:10A420000F7003D5F0ECE5F0700104F566ED6009FE
:10A43000C395664004ED04F566E5F0B403004007FB
:10A4400014C313C9C399F9ECA2059566400EA20284
:10A4500094005017C20220031202A4B2D2042003B7
:10A460000302A4B22566F566C202E4600C3000095E
:10A47000F5F07420F608D5F0FB300204742DF608D0
:10A48000E566C31329F98566F030050FE5F004D3BE
:10A490009D7008742EF608C20580EE20F00119E7C1
:10A4A000300601E320F001C4540F2430F608D5F043
:10A4B000D8C37204D02022C0A8C02075201075A86F
:10A4C00080E8C0E020071D78B8E520F6E52054308C
:10A4D000700678B9E9F6800CB4100978B9E582F60F
:10A4E00008E583F6D203782775F008E52012A55C0D
:10A4F000601DA2E7C0D0C2E712B13ED0D072E79291
:10A50000E712A51F18E52012A56BD5F0DE8008E440
:10A5100012A51F18D5F0F8D0E0F8D020D0A822C09E
:10A52000F0C0E075F014747012BF5E5014E4D5E012
:10A53000FD92D112BBE372D1E4D5E0FDD5F0E78006
:10A5400016E812B95640E6D0E0C0E012B95640DD38
:10A5500092D112BBE372D1D0E0D0F022543070021D
:10A56000E722B41003E493227420225430700209CD
:10A5700022B410080582E582700205832220202083
:10A58000414D0048452050453E004D335920484537
:10A590004800334D204845484F5000335920484526
:10A5A000484F5000454C204845484F500045727276
:10A5B00020454C30310045727220454C3032004508
:10A5C000727220454C30330045727220454C303455
:10A5D0000045727220454C30350045727220454C62
:10A5E00030360045727220454C303700457272207B
:10A5F000454C30380045727220454C303900457268
:10A600007220454C31300045727220454C3131008A
:10A6100045727220454C3132004D59204845480062
:10A62000202020483659004D4550453E50453800C1
:10A630004D4F7D48203E4D59004D504F38204F43DF
:10A640003E00C020F52053200F85F02DD205BD001F
:10A6500002C205E52DC333F52E30010302A69BE5AA
:10A660002D29F9852EF020F00119E7300601E320AD
:10A67000F001C4540F7003D5F0ECE5F0700104F55F
:10A680002EED6009C3952E4004ED04F52EE5F0B4DF
:10A690000300400714C313C9C399F9ECC3952E40B6
:10A6A0000EA20294005017C20220031202A702D287
:10A6B0000420030302A702252EF52EC202E4600C3B
:10A6C000300009F5F07420F608D5F0FB3002047470
:10A6D0002DF608E52EC31329F9852EF020F0011977
:10A6E000E7300601E320F001C4540F2430F63005B2
:10A6F0000CE5F0D39D7006E64480F6C20508D5F05F
:10A70000DBC37204D02022C0A8C2ACC2A975090064
:10A7100078F1E2B40221E52254037008750A6475E9
:10A720000B008032B40108750A7E750B0080277516
:10A730000AED750B00801FE522540370E7750A804F
:10A74000750B008011B40108750A00750B018006B5
:10A75000750A00750B02C3E5099400F509E50A9432
:10A7600022F50AE50B9400F50B9022007C0074AAF8
:10A7700012DEB9750C00750D22750E00A375F0FF81
:10A78000800B75F000850D83850C82AC0E74FF1272
:10A79000DEAF402C050DE50D7002050E150AE50A29
:10A7A000B4FF02150BE50A450B70D7E50C6018F5F0
:10A7B000F074FF850C82850D83AC0E12DEAF50075E
:10A7C000740512A94C80FEE4D0A82275F003120C87
:10A7D0007C12B762741012AC2612071E9056271214
:10A7E00004E4796F12E14A796F12C609780075F0B6
:10A7F000C012E089754AFF784C75F00474FF12E1CD
:10A8000023740912DA79E54AB4FF0890563B120422
:10A81000E48059756B00788812DCE0E56B75F0090F
:10A82000A4F9C0E009E3F56C756D007888796C12C5
:10A83000DE85788D742DF608756D59796C12DE857C
:10A84000120508788812DCE07891D0E02402F91231
:10A85000DB237888743DF608748512D9E312050865
:10A86000056BE56BD3954A500302A816796B12D19C
:10A8700079796B12D443786B12C98B786E12D2DE61
:10A8800012D10712D36612DA06027065C0A8C02082
:10A8900053200075A880C0F0CFC0E0CF7F05E52031
:10A8A0005470700474D0800FB4100974A2BC0007F7
:10A8B00074A0800302A94012BF5E500EE4D5E0FDF3
:10A8C00012BBE3D5E0FDDFD68076E9300309E583EE
:10A8D00012B95640E7E58212B95640E0D2977404A7
:10A8E000D5E0FDD2967408D5E0FDE52054707004E3
:10A8F00074D1800FB4100974A3BC000774A1800345
:10A9000002A94012BF5E500602A8BC12CE9612CC1D
:10A91000C7C0E0E52054077004D0E0801DB40105F5
:10A92000D0E0F68003D0E0F2200303098008A3E51D
:10A9300082458370010C08D5F0D112BBE3C38001BE
:10A94000D3CFD0E0CFD0F0D020D0A822C0A875A817
:10A9500080C020C083C082C8C0E0C8C0E07827B4EF
:10A960004A00501D12A9F8E49354FCF520A3E49387
:10A97000C0E0A3E493F582D0E0F5834582600280D5
:10A980004CE4C20090A9F375F005E49312B13E12B5
:10A99000A51FA318D5F0F3D0E0C0E075F06484F5EE
:10A9A00083E5F075F00A84F582E5F0C58324301262
:10A9B000B13E12A51F18E582243012B13E12A51F28
:10A9C00018E583243012B13E12A51F800312DEFF6A
:10A9D00012C7FAD2A9D2AF12C276B41702800512FA
:10A9E00003D160F3D0F0C8D0E0C8D082D083D020AB
:10A9F000D0A82245727220201475F003A42494F587
:10AA000082E5F034A0F58322C0A8C2AC7520001204
:10AA1000DBF678BB74313007027432F608743DF609
:10AA2000E4FDFEFF1294FDB418028018B41C04C2A9
:10AA30000780DCC0E012C7FAD0E0B420E374FFC0A6
:10AA4000E002AAB92007338D6B8E6C8F6D7883E29C
:10AA5000644B6002803B79847894E2B44B0279962F
:10AA6000786E75F00312DFB312D50D401C7007E548
:10AA700071B40200401BD2078095ED656B700AEE41
:10AA8000656C7005EF656D600812C7FAC20702AA0F
:10AA90000F796B12D529780A74AA129899500C1262
:10AAA000C7FA7403C0E012A94C800EE4C0E09081A4
:10AAB0009112A4B712C27660FBD0E0D0A822C017D2
:10AAC000C016C0207520007830793712E19A7830AE
:10AAD000794512DC517830793E12DCC6E52054C04D
:10AAE000B4C00302AB6B300708788375F02812E01E
:10AAF00089751700E51712E143F812E04A6063E533
:10AB00001775F010901E0012DAB97C0012DFEF12F8
:10AB1000B53864AA6005743202AB6B797975F006BA
:10AB200012DFE5E51712E143F912926A3007297541
:10AB30001600E51675F00AA42488F9E7601114756B
:10AB4000F008A42483F80909E7F2080912DDA20538
:10AB500016E516B4030040DA12CFEF7830796B12A5
:10AB6000DDA20517E517B405004089D020D016D026
:10AB70001722C0A875A88090811312A4B7787975A0
:10AB8000F00712E11B751700754A00124C47124C72
:10AB9000E412493C70100517124CDD1247EB124CC1
:10ABA000F6124CE480EBB438028005B404E8801A55
:10ABB000E517700302AC23124CDD1247EB124D0077
:10ABC000798375F02A124C33600612A94C02AC232B
:10ABD000798AE3F56B09E3F56C754A02124C47126A
:10ABE0004CE4754A02124CDD12493C600BB4380348
:10ABF00002AC2312A94C80FE1247EB7983124C332E
:10AC000070F17883E2D3956B08E2956C4007787910
:10AC1000798812DD96124CDD1247EB124CF6124C7D
:10AC2000E480BFD0A822C082C083142400F582E44F
:10AC30003403F5837C0012DFEF12B538D083D08265
:10AC400022010103010000010103030107030401C4
:10AC500003060301000000000000000000000100E6
:10AC600000000000000000C0000340000440000A93
:10AC700040000AC000014000014000014000010006
:10AC800001040001040001040001070001040001A7
:10AC900005000104000104000608400005C0000191
:10ACA000400001C00001400001C00001C00001C01F
:10ACB00000014000014000004000000000040000CE
:10ACC00062C00001C00001400003400002400001DA
:10ACD000400001400001400001D22412C68DB41C86
:10ACE0000122B4150122C22412C1E0B41C0122B415
:10ACF00015012212AD00B41C0122B415012280D925
:10AD000012DBF678BB9080C512BC9A120711700254
:10AD10007403F56BF56CC20002AD7C12C27660FB69
:10AD2000B4170122B41C0122B4150122B4140890F6
:10AD3000004A1204E480E4B42C0AE56C1207031202
:10AD400000B880D7B411D478C1743DF612DD12D2A8
:10AD50000012C27660FBB41C0280A5B41807E56C33
:10AD6000120703809BB41208E56C60E5156C800C3B
:10AD7000B413DEE56CB4050050D7056C78C2E56C01
:10AD80002430F612DD122000C88090C24378027988
:10AD90000F75F00612DFA9786B798275F00212DF69
:10ADA000B3E56B456C700512D8DF805312D989600A
:10ADB000137409C0E0780F790275F00612DFB3D082
:10ADC000E002AE388D0F8E108F1179807401F30977
:10ADD000740E304302740FF312DF097480304402A2
:10ADE00074C0128FB5600FB42004741280C5B448CB
:10ADF00002800C02D90512DF1320430302AE251294
:10AE0000E00B12DFEF12B538B4AA0280057412020B
:10AE1000ADB312B538B4FF0302ADB112BB2B60ED78
:10AE2000D24402ADCA780F790275F00612DFB30280
:10AE3000D9057401800274037982F375F00374807C
:10AE40007900F37901E5F0F312DB9A2044287814B5
:10AE500012B4505005D8F902D905F954CFB4C5023F
:10AE60008011B4CC0512DF6D8009B4CF0312DF6D01
:10AE700002D90512DB9AE51B540744A012CD2679AE
:10AE800001E3F5F07900E3F912C145780A12B450F4
:10AE90005005D8F902D90512DB9AF5F054C064C008
:10AEA000600302D905E5F0A2E4924454CFB4CA028B
:10AEB000051B02D905B4C6028091B4CC0512DF6D22
:10AEC0008089B4CF0612DF6D02D905B4C50574C000
:10AED00012CD2602D905C015C01775171912B45026
:10AEE0005009D517F8742AD302AF75F854CFB4C5FA
:10AEF000028014B4C00302AF59B4CF0302AF60B4F0
:10AF0000CC02804702AF6F12DB9AE51B540744A0C6
:10AF1000A24492E412CD267901E3F5F07900E3F939
:10AF200012C14575150A12B4505007D515F8742A88
:10AF3000803FB4CA07051BC24402AF74B4DA0705E8
:10AF40001BD24402AF74C2E4B4CC0512DF6D80B7EB
:10AF5000B4C60302AF07B4C00374498014B4CF076A
:10AF600012DF6D7448800A12DB9A74C312CD267406
:10AF70002BD38001C3D017D01522C0E0788812DC13
:10AF8000E07891798512DB23789F12DB6E7480F66E
:10AF90007983E39052BEB404039052B5788875F07B
:10AFA0001812BC9A1205082212DB5F7888E56F70D0
:10AFB000129052A775F01812BC9AE56B2430788E67
:10AFC000F6800E796F75F00CE76006F60809D5F08B
:10AFD000F7786F75F00512E11B7897796D7C057D28
:10AFE00002740175F00512A3EE789C76251205080F
:10AFF00012DB5F7890797B7C0F75F0077D0274011E
:10B0000012A3EEE56C9052DD700390516078887564
:10B01000F00612BC9A120508E42212CD84F5203005
:10B0200007081243F2601002B0A630060A791F1218
:10B030004420600302B0A630050812D0E16003028C
:10B04000B0A630040D12D99B6008B44502800302FB
:10B05000B0A6300308120BB7600302B0A6E5205477
:10B0600007B4074812C007C0E0600AB4390280057F
:10B07000D0E002B0A6791E12C58312E133D0E07889
:10B0800082F2B4390B12D0E1600302B0A602B0AC78
:10B09000786B12C98B7984786E75F00312DFB31266
:10B0A000D50D5008740B12A94C74FF22E422C01570
:10B0B000C017751719C246C298800D12CD26E51724
:10B0C000B40300500375170312B4505008D517F895
:10B0D000742A02B138F51554C0B48002802212DB04
:10B0E0009AE51554CFB4C50474C780CFB4C00280AC
:10B0F000D7B4CF08744812DF6D02B13874C380BB77
:10B10000798012B82F5011B42A0302B0C812DB9A0A
:10B11000B446B574C602B0BB12DB9AE5155407F508
:10B12000F0E51A5407B5F00B74CA12CD26051AC300
:10B13000E4800674CC02B0BBD3D017D01522C0D0A7
:10B1400024E383D0D022008621490C63422000BE34
:10B150000046044080523F065B4F666D7D077F6F5F
:10B1600041000048315300777C395E79713D760F9C
:10B170001E723837543F73BF506D783E0000006E2A
:10B180004C7D640F000820777C585E79716F7404E1
:10B190000E723854545C7367506D781C0000006E5A
:10B1A0000000305F01080000000000000000000007
:10B1B000000000000000000000000000000000008F
:10B1C000000000000000809050E11204E474267535
:10B1D000F00284F51725F0F5167E0078889050F47B
:10B1E00075F01812DE6FEE04788C12D04274112EB6
:10B1F000F8E2FD789012D042EE90AC41936D60057C
:10B200007888742AF6EEB517005027EE25160478D4
:10B210009812D042EE25162411F8E2FD789C12D047
:10B2200042EE251690AC41936D60057894742AF631
:10B23000800A789475F00E742012E1231205080E2E
:10B24000EEB5160040951204CE75F005120C7C2266
:10B25000C017783E75F03112E053700302B2D41279
:10B2600004CE79379051B212E1C9784512E04A60B4
:10B2700008794590524112E1C9783E12E04A6008CF
:10B28000793E90523912E1C9751700E51775F0083B
:10B29000A4248304C0E0F812E04A7004D0E08028BF
:10B2A000E51775F010901D0012DAB97C0012DFEF7F
:10B2B000796B75F01012DFE5E51704F56BD0E0F956
:10B2C000787B12E1B212AFA80517E517B40500406C
:10B2D000BA1204CED01722C0A875A880E4F56BF589
:10B2E0006C800512D3E7E5F0F56DB418028003B465
:10B2F000120EE56CB418028003B412047401805479
:10B30000E56B24028380181314151617180D0E0F01
:10B310001011120708090A0B0C010203040506B5F7
:10B320006D0C056BE56BB418004003E48026856D59
:10B330006C78BB742075F00812E123E56B78BB12C2
:10B34000D04278BE742DF60808E56D12D04212DDA9
:10B350001202B2E3D0A822C020532000788812DC69
:10B36000E07883E2B4B202802BB4B4028026B4B198
:10B37000028003B4B304D200801AB4B7028037B499
:10B38000B9028032B4B6028003B4B804D200802679
:10B39000741A803E7987789412DB14789F798CE355
:10B3A0007004742D80022440F678889051C53000D6
:10B3B000039051BE80127891798512DB23788890B2
:10B3C00051C53000039051BE75F01812BC9A120599
:10B3D00008E4D02022C031C020D200E8C0E078BB11
:10B3E00074CDF608743FF679BD75F006745FF70901
:10B3F000D5F0F9D0E0C0E0F875330002B43512C2E0
:10B400007660FBB41C0302B3E7B4150302B4471221
:10B41000DA595005B40A00400512C7FA80E024301A
:10B42000F5F0F608E53324BDF9300004742D8002F0
:10B43000E5F0F7053312DD12E533B40600500302E0
:10B44000B3FE08E4F67418C8D0E0C8D020D031228A
:10B45000C2987582A6109808D5E0FAD582F7806365
:10B46000E599B47FF075F012109808D5E0FAD5F0A0
:10B47000F780E2E599B402DD75F012109808D5E086
:10B48000FAD5F0F780CFE599B518CA75F012109883
:10B4900008D5E0FAD5F0F780BCE599F58354C0B43F
:10B4A000400302B45575F012109808D5E0FAD5F0B3
:10B4B000F780A2E59925832518600302B455E5833A
:10B4C000C38001D322C020C017C032753200751767
:10B4D0000075200074BB2532F8745FF6087420F6FE
:10B4E00012DD1212C27660FBB42003D38043B41C79
:10B4F0000D80DBE517700274012440C3803312DA3B
:10B5000059400512C7FA80DB300012C51775F00AE2
:10B51000A42517B40500400512C7FA80B1D200F582
:10B520001774BB2532F8E51712D04212DD1280C322
:10B53000D3D032D017D02022C0A8C020752000E878
:10B54000C0E0E9F8C0F08007E8C0E0E9F8C0F0C268
:10B55000ACC2A9850C82850D83AC0EE52054077022
:10B560000B12DEE14033C5F07401801BB4010712F9
:10B57000DED740258008B4022012DECD401BE8F95A
:10B58000E4C5F0D0E0C0E0250CF50CE4350DF50D78
:10B59000E4350EF50EC5F08007740512A94C80FE47
:10B5A000D0F0C8D0E0C8D020D0A822E8C0E075F024
:10B5B0002C12E089D0E0C0E0F8904FC875F010126E
:10B5C000DE64901C007C0012DFEFD0E0C0E02410AD
:10B5D000F975F00C12DFDBD0E0C0E0241CF89057C6
:10B5E000CA75F00812DE6474C875F06484600424BF
:10B5F00030F208E5F075F00A842430F208E5F02412
:10B6000030F2D0E02428F879F1E3F208740AF275F8
:10B61000F02C22F5F0E4F3E5F009F30922C0A87557
:10B62000A88012D99B7002805EB4200512A94C80BC
:10B63000FEB423028003E4804E786B797F12BA1542
:10B64000786F12C98B786D796F12BA15C3E56D9555
:10B650006BF56DE56E956CF56E5004740B8028707B
:10B6600007E56DB4020040047423801B700280174C
:10B67000786B12D2DE74247982D39712D8A5256B09
:10B68000D4B4240050E2E4D0A8227985E3B40202C5
:10B69000804CB403028047740E12AC2612071E7948
:10B6A0008612CEEF740D12AC2612071E7985E3B414
:10B6B00001028039B404028025788D12E04A602DA1
:10B6C000798D9051FE12E1C97827798612DCC6790E
:10B6D0002790521012E1C9792712D6F7800F740E05
:10B6E00012AC2612071E7985E30912D093740D124D
:10B6F000AC2612071E22C0A875A88012B76212DB02
:10B700005F7888904FC875F00E12BC9A7997774E83
:10B71000901C007C0012DFEF799875F00C12DFE5C9
:10B7200012050812DB5F78889057BF75F01012BCC5
:10B730009A789874C812D66812050890004B75F074
:10B74000187888740112DE6F120508E46005D2A92A
:10B7500012A94C12E15F1204CE75F006120C7CD0D7
:10B76000A822C020C200C20190040030000390054E
:10B77000007C0012DFEF12B53812071E7400C0E023
:10B7800075F020A49004013000039005012582F596
:10B7900082E5F03583F5837C0012DFEF798875F060
:10B7A0002012DFE57988E76005D201120508D0E0B4
:10B7B00004B40600500280C62000062001031204D3
:10B7C000CE740D12AC2612071ED02022C034F534E0
:10B7D000788812DCE090532D788875F00612BC9AB8
:10B7E000788CE5342430F6E5341475F020A49021EB
:10B7F0008012CDE17C0012DFEF798E75F01212DF3E
:10B80000E512050890530F788875F00412BC9AE58C
:10B81000341475F020A490210012CDE17C0012DFD9
:10B82000EF798C75F01412DFE5120508D03422127E
:10B83000D92B404BC24675820012D92B404130466D
:10B8400021B403028034B41006C246747F801AC04B
:10B85000E0B9CE005018747FF32582F58209C24604
:10B86000D0E0B47F04D24680D0B9CE004004744703
:10B870008018F3092582F58280BF12D92B500574F8
:10B880002A02B88A258260057446D38004E9C394ED
:10B890008322C02053203FC0F012DBF678BB7C0827
:10B8A00075F0047D02740130060512A64280031271
:10B8B000DD4278BB75F002E6B4200408D5F0F8D07C
:10B8C000E0C0F020070C600F78BB12D0427463F622
:10B8D000800578BB743DF6D0E06015B402028003A9
:10B8E00020070D78BB75F003E64480F608D5F0F824
:10B8F000C3D02022C01712DBF678BB7448F6800351
:10B9000012C7FA7C027D067E067F00796B741412E2
:10B910008E34B41C02800BB418E612D98960071269
:10B92000A94C74018025C0A875A8807802790F758C
:10B93000F00612DFA98D0F8E108F1112D298780F9A
:10B94000790275F00612DFB3D0A8E4C0E0E412DBA0
:10B95000F6D0E0D01722C0F075F00833202B049207
:10B960009780029295C0E07401D5E0FDD296E43054
:10B9700096FD209608D5E0F7D0E0D380367402D546
:10B98000E0FDC296D0E0D5F0D212BC247403D5E01D
:10B99000FD75F000D2963096FD209606D5F0F7D3CF
:10B9A000801175F001D5F0FD12BC36C29675F0011C
:10B9B000D5F0FDD0F022C0A8C020752000C0F0C096
:10B9C000E0850C82850D83AC0EE5205407700BD00A
:10B9D000E012DEB9402274018025B4010DD0E012DE
:10B9E000DEA54014D0E0C0E08015B4020BD0E01218
:10B9F000DE9BD0E0C0E05007740512A94C80FE2504
:10BA00000CF50CE4350DF50DE4350EF50EE4D0F033
:10BA1000D020D0A82276000876000909E712D7AA1C
:10BA2000F5F090016D12D561A68318A682E5F0C0ED
:10BA3000E0240375F0048412E0FBD0E075F0048488
:10BA4000C2D5E5F07002D2D51919E712D7AA14129F
:10BA5000E0FB09E712D7AA146017F5F090961E30A4
:10BA6000D503909611E5F09312D7AA12E0FBD5F01A
:10BA7000F422C0F0C0205320E075F0057D05C3C05E
:10BA8000D0E6300201E2FCE4200313E5205403B4C5
:10BA90000205E493A380077003E78001E309200413
:10BAA00008D0D03CD4C0D08009D0D0CC9C12D8A52E
:10BAB000C0D0200203F68001F208D5F002800920F0
:10BAC00003BFDDBDD20380B9D0D0D020D0F0227822
:10BAD0000EE2F58208E2F58308E2FC12DFEF12B510
:10BAE00038B4AA4512B538C0E012B538D0E0B4A1D8
:10BAF0000C791275F00C12DFDB74A1802D64A36049
:10BB0000028026786B75F00912E11B796B75F003E2
:10BB100012DFE5742012CC97791275F00512DFDB85
:10BB2000C24875150174A38001E422B4A1004055F8
:10BB3000B4B0005014C394A083220D003000000D57
:10BB400000300000000D300000B4B1004037B4C038
:10BB5000005014C394B083220A0A0A0A0008080895
:10BB600008000000000000B4C1004019B4D000502B
:10BB700014C394C083220000000000000000100CD9
:10BB80000101000000E42275A8807881E26005B41C
:10BB90001900400302AE3290C30A1475F00312DAA2
:10BBA000B9E493F58330271220E70A792FE3600A7E
:10BBB000740802AE38740202AE38E58330E60A1229
:10BBC000D99B6005740702AE387981E31475F003E0
:10BBD00090C30A12DAB9740193F5F0740293C0E0CD
:10BBE000C0F022C0A8C2AFC0F012BC2D75F003D5C2
:10BBF000F0FDD29675F0003096FD209606D5F0F750
:10BC0000D3801C75F001D5F0FD12BC2475F004D56D
:10BC1000F0FDC33096FD209606D5F0F7D38000D016
:10BC2000F0D0A822202B03D29722D29522202B03DA
:10BC3000C29722C29522202B03A29722A295227D91
:10BC400000D2D57982E3B40600400302AE3675F027
:10BC500020BD00059004008006BD0108900500602D
:10BC600001A3800CBD020590210080039021801467
:10BC700012DAB97C0012DFEF7982E30975F0203027
:10BC8000D50875F021600315F00912DFC712E13302
:10BC90007882E4F275F00302AE3EC02053200074B7
:10BCA00001C0F0B40F0040028046C202C44220D05E
:10BCB000F0C0F0E49370028013B40D04D202800C43
:10BCC000200003F68001F208A3D5F0E7300321E558
:10BCD000F0600D7420200003F68001F208D5F0F327
:10BCE00030020DA3E4936008E52054F0C4D5E0BA17
:10BCF000D0F0D0202278F1E2B4022AE52254037079
:10BD00000BD37463951374009514B322B4010BD351
:10BD1000747D951374009514B322D374EC95137449
:10BD2000009514B322E5225403700BD3747E95134F
:10BD300074009514B322B4010BD374FE95137400F0
:10BD40009514B322D374FE951374019514B3227D18
:10BD500000D2D57982E3B40600400302AE3612B6B3
:10BD60001375F020BD00059004008006BD01089009
:10BD700005006001A3800CBD0205902100800390A6
:10BD800021801412DAB97C0012DFEF75F02120D582
:10BD90000375F0207983E30930D505600315F009B8
:10BDA00012DFDB75F02502AE3E78F1E26402600539
:10BDB000740602AE38754F01755000788275F00A2E
:10BDC00012E089784F12CCF74004E402AE38854F78
:10BDD000828550831582E582B4FF02158374401278
:10BDE000D561FC12C783743612CDE1E43CFC12DF4E
:10BDF000EF798275F00A12DFC7054FE54F70C40571
:10BE00005080C0752080780475F02012E089C2004F
:10BE100012DBF690810130000390810578BB75F04C
:10BE20000812BC9A12DD12E4FDFEFF1294FD6418A4
:10BE30006003027B85781C3000027805EDF208EE85
:10BE4000F208EFF2200004D20080C5791C12A23162
:10BE5000500302790012C7FA027B85C020C0177414
:10BE600088C0E0740C12AC2612071E740C12AC26AB
:10BE7000120761F517C2077888D0E0F98517F0E35B
:10BE80007003F6800EF60809D5F0F4E36005E9C00A
:10BE9000E0D2077888E66003120508300707E51747
:10BEA000B420D2D0E0740D12AC2612071ED017D0E9
:10BEB000202278F1E2781418B40227E522540370A6
:10BEC0000AC374649608740096B322B4010AC3745A
:10BED0007E9608740096B322C374ED96087400969B
:10BEE000B322E5225403700AC3747F960874009647
:10BEF000B322B4010AC374FF9608740096B322C338
:10BF000074FF9608740196B32275A880D244788194
:10BF1000E26005B41000400302AE3290CE3C1475CE
:10BF2000F00312DAB9E493F58330E70820270574AB
:10BF30000202AE3830270D30E60A792FE36005742F
:10BF40000802AE387981E31475F00390CE3C12DA22
:10BF5000B9740193F5F0740293C0E0C0F022C22BD3
:10BF6000B470028003B47102D22BC0F0C0E075F04F
:10BF70000012BC36829640257402D5E0FD12BC2D1D
:10BF80007405D5E0FDD2967403D5E0FD12BC24748F
:10BF900002D5E0FDD5F0DAD0E0D0F0D32212BC2DEE
:10BFA0007404D5E0FDC2967403D5E0FDD0E0D0F076
:10BFB00002B956C0F0C082C020752000E4F582129C
:10BFC000C91C403560F9B4FF0280F4C0E054C0B42D
:10BFD000C002D200D0E0543FC5F085F08275F00673
:10BFE000A4C58275F006134003D5F0FA70CEC37471
:10BFF0000795F02582F58280C6E58230000274CE76
:10C00000D020D082D0F022788375F01412E08975A8
:10C01000174B791F1244206019C0E0781F75F00C8F
:10C02000743F12D964D0E0751700B439028003025E
:10C03000C058E517781EF27883F2644B60057439B6
:10C0400002C0587812124829600302C058788479D7
:10C050001275F00312DE59E422E8F975F000E7B436
:10C060002E051905F0801DB43002800CB43100405B
:10C0700005B43A00400E80221905F0E5F0B40C003A
:10C0800040DC8023E5F0601F75F00AE7B4200280F1
:10C0900009F67420F71819D5F0F1E6B420028007EC
:10C0A0007420F618D5F0F322301B4BC020C9C0E035
:10C0B000788812DCE0C2009051A6301B0FB9030251
:10C0C000800AB904028005D2009051AB788875F0DF
:10C0D0000612BC9AD0E0F9788C300002788E7C0889
:10C0E00075F0043000047C0615F07D00740212DD4A
:10C0F0005A120508D020227879793012E1B2787985
:10C10000792712DD96500122787912C13050012230
:10C110007830797912E1A67837792712DC51781CCA
:10C12000E27001221412E143F8792712DC51C32294
:10C13000740428F8E654F0700A08E6700608E67001
:10C1400002C322D322C082C2467599001099028090
:10C15000FB758200C299E3F599B47F02D24625822D
:10C16000F5823099FDC299304607759910C2468014
:10C17000F109D5F0E175997F3099FDC29975990360
:10C180003099FDC299E582F404F5993099FDC29980
:10C19000D08222788275F00812E089E47883302713
:10C1A0000104F23027067808E27887F2120BB760B4
:10C1B00013B4170474018009B41804740280027463
:10C1C000047885F2788674FFF230270C782EE278B6
:10C1D0008AF2782FE2788BF275F00AD24402AE3EF2
:10C1E000C0A8752000787D12D2DE78BB797D12D48C
:10C1F0006012DD1212C2767008743212D86902C160
:10C20000E5B4111A30240512C7FA80D9E4FDFEFF07
:10C21000129FB3B41805790512DAD802C1E5B41734
:10C220000280051203D160BDD0A822788475F02465
:10C23000743012D9647582187583207C0012DFEF88
:10C24000798475F02412DFC77517017884E5172407
:10C2500030F2E82406F80517E517B4050040EE753E
:10C2600082007583207C0012DFEF798475F018124C
:10C27000DFC712E13322C0D0C2D5C0F0E8C0E0C0B1
:10C28000A853A8F9741424CEF875F00018E2C5F08C
:10C29000F2B8CEF8D0A8C0A8E5F0700A30D507747F
:10C2A0000A12D86980DBD0A8D0E0F8E5F0D0F0D051
:10C2B000D07009C0E0740A12D869D0E0202CFD22A9
:10C2C000C0A8C2ACC2A9786B9000007C0075F007D2
:10C2D00012DED750047405802EE56BB4AA27E56CF6
:10C2E000B45522E56D256E256F257065717016E5D4
:10C2F0006F5322FC4222E570B40400500878F1E547
:10C3000070F2E480027401D0A82200DB8C00D8F225
:10C3100000BD4FC0BC3F00E1CEC0E1D300CF1A80CA
:10C32000CC3600D636C0D4B7C0AE3200E01400C957
:10C33000F900AD8B80E1D800E1DD00E1E2809CDF17
:10C3400080A248C0BDA900D73CC0D75200E1E7C0D9
:10C35000E1EC75F006A42400F582E5F03420F583C5
:10C36000227937124419600FB43921783774307547
:10C37000F006F208D5F0FB786B793775F006E366C6
:10C38000600374FF220809D5F0F4E42212A94C746A
:10C39000FF22E53012C3E1E49322C020789A798A23
:10C3A00012D7C0786B7979E709C4540FB40500B38C
:10C3B00075F009E73400F60809D5F0F77898E4F647
:10C3C000786B799112E06E7979E709C4540FB4055E
:10C3D00000B375F007E73400F60809D5F0F7D02070
:10C3E00022C0F075F006A4207F0C249EF58274878D
:10C3F00035F0F583800C24ADF582748835F0F58333
:10C400008000E493D0F022E52F5403F5F0AE30AF76
:10C41000300EEE12C3E1B4EE02EF225403B5F00485
:10C42000EEFF80ED50EBEF22C0E01475F020A42465
:10C4300000F582E5F0341FF583A37C0012DFEF786E
:10C440008876230875F017E412E123798975F016D0
:10C4500012DFE5740B12AC2612071E7989E7600320
:10C46000120508740D12AC2612071ED0E022C0A8D7
:10C4700075A88012E00B12DFEF12B538B4AA028063
:10C480000812D599B420EC80237983E312BB2B707A
:10C49000047407801704F5F012DFC7850C12850DB0
:10C4A00013850E1474AA12B9B6E4800512A94C8043
:10C4B000FED0A822C0A8C08275A88075826474D0FE
:10C4C00012BF5E50127432D5E0FD12BBE37464D526
:10C4D000E0FDD582E98019741812B95640E775F06D
:10C4E00028E412B95640DED5F0F712BBE3C380054D
:10C4F000740312A94CD082D0A822C0A875A880903D
:10C500001C007C0012DFEF796B75F00812DFE57814
:10C510006B793775F008E36670070809D5F0F78086
:10C520001B901C007C0012DFEF793775F008E36088
:10C530000712B9B609D5F0F6E412B9B6D0A822C0F0
:10C540003375F00512E11BC3E89405F8E712D794A0
:10C55000F608A6F0180987331975F008E53333F5A6
:10C5600033501AC0F0740415F0A424EFF582E5F0FE
:10C5700034CDF58312D95118181818D0F0D5F0DC45
:10C58000D03322C0A875A880E9C0E0901C107C00C0
:10C5900012DFEF796B75F00D12DFE5D0E0C0E0F946
:10C5A000786B75F00DE34670090809D5F0F7D0E017
:10C5B0008011901C107C0012DFEFD0E0F975F00DB7
:10C5C00012DFC7D0A822C0A8C2AFC28E752000E576
:10C5D000285407700474FA801BB4010474FD80149D
:10C5E000B4020674FDD207800BB4030474FF800408
:10C5F00074FFD207F58BF58DE5874520F587759893
:10C6000070532807D28ED0A822E9C0E0788812DCC7
:10C61000E0788874C4F608743AF6D0E0F9788A7C39
:10C62000087D00740275F00412DD5A78949052C6A9
:10C63000E515B45A07E51770039052C775F00A1252
:10C64000BC9A12050875F001120C7C22C0A875A8CE
:10C650008078807403F2087401F20812B5AB74801C
:10C6600075F02BC24478007480F27801742BF212BA
:10C67000AED6400512B0AE5009B42A02800C742B1D
:10C6800080087982E3600312D3A7D0A82275200026
:10C6900012DBF6787912C98B78BC797912D34512FE
:10C6A000DD1212C27660FBB4112130240512C7FAE4
:10C6B00080E112C007600FB43902800AB4420280E0
:10C6C0000512A94C80C712AA0880C2228AEA8AF7FA
:10C6D0008B598AEA8AEA8B6F8B748AEA8B798AEAA9
:10C6E0008B888BB98BEC8C1A8C1A8C1A8C1A8C1A3E
:10C6F0008AEA8C498C498C498C498AEA8AEA8AEA16
:10C700008AEA8C768C878C8A8C8DC020752000708C
:10C710000474008009B401047404800274082400C5
:10C72000F582E4341AF5837C0012DFEF75F004E53E
:10C7300020600512DFC7800CE9C0E012DFDBD0E02B
:10C74000F812D82AD02022C020D207788812DCE044
:10C75000789120070512E0F3800312DB23789F1203
:10C76000DB6EE8C39488F5F012D5B4C395F0500A97
:10C77000788875F01812BC9A80031204E412050838
:10C78000D02022E5225403701174002582F58274B2
:10C79000643583F58374003CFC22B40111740025D8
:10C7A00082F582747E3583F58374003CFC2274002C
:10C7B0002582F58274ED3583F58374003CFC22C03C
:10C7C000A875A880C02053200FD206C017787979A9
:10C7D0000C75F00712DEEB5004740380167879793B
:10C7E0006B30070512DDC6800312DB415004742450
:10C7F0008001E4D017D020D0A822740FC0A8C0F0C8
:10C80000C020C007C2AFD2B5C200F50775F0322014
:10C810000004D2B58002C2B5B200E4D5E0FDD5E097
:10C82000FDD5F0EB1507E50770E2C2B5D007D020C3
:10C83000D0F0D0A822C020C20712DBF678BB7C085B
:10C840007D0275F005740912DD4278BBE6C0E07820
:10C85000BB743D2007027423F6D0E06420600D789D
:10C86000BB75F003E64480F608D5F0F8D02022C06E
:10C87000A8C015C017C2AC12DB9AE51B540744A030
:10C88000A24492E412CD267901E3F5F07900E3F9B0
:10C8900012C145051BD244C3D017D015D0A822C061
:10C8A00015C01775171902AF07788474A1F208E450
:10C8B00075F01F12D964751700E51775F020A424D0
:10C8C00000F582E5F0241FF5837C0012DFEF798408
:10C8D00075F02012DFC70517E517B4040040DA121F
:10C8E000E13322788812DCE0788D9051A175F00355
:10C8F00012BC9A901C007C0012DFEF799175F00851
:10C9000012DFE5901C107C0012DFEF12B538789929
:10C91000B44B05768208768312050822C0A8C2AF00
:10C92000E4D3D2B220B22A747112BF5E401312CC8B
:10C93000C7400EF5F012CE96400712CCC7400280D9
:10C9400001E4C0E0E4D5E0FD92D112BBE372D1D0A6
:10C95000E0D0A822788812DCE078977C087D00740B
:10C960000175F00412DD5A789F12DB6EE8C39488DB
:10C97000F5F012D5B4C395F0500A788875F0181206
:10C98000BC9A80031204E412050822C0207520001E
:10C99000C0A875A880C0F0E9C0E0790475F0021263
:10C9A000A88C200703F68001F20809D5F0F112A83F
:10C9B0008C200703F68001F2D0E0F9D0F0D0A8D0A7
:10C9C0002022C0A8C2AFE4D5E0FD75F064D290D2B9
:10C9D00091E400000000209106D5E0F8E48015C243
:10C9E00090E400000000209107D5E0F87401800475
:10C9F000D5F0DAE4D290D0A8227982E36005B406BB
:10CA000000400302AE321475F010901D0012DAB926
:10CA100075F010C0F07982E4F3097C0012DFEFD0EA
:10CA2000F0C0F012DFDBD0E02403F5F002AE3EC030
:10CA300020532000C0F075F005E5F028F8E5F0C3BC
:10CA400033F5F018E6300001E2C0E054F06004D0A5
:10CA5000E0800B15F0D0E0540F7003D5F0E5E5F061
:10CA6000D0F0D02022C02053200075F00212D20B4B
:10CA700012D9BF742E300402743A12D1E70809D5D6
:10CA8000F0EB30040D30050A12D19E742012D1E76C
:10CA9000800612D20B12D9BFD02022C0A875A88060
:10CAA000C0177879790C75F00812DEEB5004740326
:10CAB0008019787975170075F007E6F42517F517D2
:10CAC00008D5F0F6E6651760027408D017D0A822E2
:10CAD000788812DCE07888798912DE907891798CF8
:10CAE00012DE7A201B1B9051A6789775F00612BCB7
:10CAF0009A7985789B7C0575F0047D00740B12DDB6
:10CB00005A12050822C0A875A880C0177914788128
:10CB100075F00375170012A88C4018F6F42517F568
:10CB2000170809D5F0F012A88C4008651760067444
:10CB30000880027403D017D0A822C0A875A880C0AE
:10CB4000177814790F75170075F003E7F42517F5BA
:10CB500017E7129899400F0809D5F0EFE5171298DA
:10CB6000994003E480027403D017D0A822C020C0EB
:10CB700017751700E51704798312CF7064AA600B4C
:10CB80000517E517B4050040EB800F90514B1204D8
:10CB9000E41217FC75F001120C7CE4D017D02022AF
:10CBA000C0E01475F020A4241BF582E5F0341FF5D5
:10CBB000837C0012DFEF797975F00512DFE5787973
:10CBC00012D3C77003C380077879792712DC5ED04F
:10CBD000E022C0205320F0C0F075F005EFC0E0EE79
:10CBE000C0E07F00C312D301FE12D20BCE9E4FFFD6
:10CBF00012D32312D425D5F0ECD0E0FED0E0CFD074
:10CC0000F0D02022C0F0850C82850D83AC0EE4129A
:10CC1000DEAF5007740512A94C80FED0E075F0001D
:10CC2000700375F001250CF50CE5F0350DF50DE4FC
:10CC3000350EF50EE4227982E36005B40500400369
:10CC400002AE361475F020901F0012DAB97C001283
:10CC5000DFEF798375F02012DFC712E1337982E4C8
:10CC6000F375F00302AE3EC0A875A880C017780C1B
:10CC700075F007751700E4129899401174FF251795
:10CC8000F51708D5F0F0E517129899500474038051
:10CC900001E4D017D0A822C0A875A88030E717F407
:10CCA00004C3C50C950CF50CE50D9400F50DE50ECF
:10CCB0009400F50E800E250CF50CE4350DF50DE411
:10CCC000350EF50ED0A822C0F075F008C0E0D2965F
:10CCD000E43096FD209608D5E0F7D0E0D380151219
:10CCE000BC36C296D0E033C0E07401D5E0FDD5F08B
:10CCF000DDD0E0C3D0F022E6700708E6187002C36A
:10CD000022E522700AD3E6946408E618940022B45F
:10CD1000010AD3E694F408E618940122D3E694E8D5
:10CD200008E618940322C29975997F3099FDC2993B
:10CD30007599023099FDC2998518993099FDC2996B
:10CD4000D2E5F5993099FDC2992518F404F599308A
:10CD500099FDC29922C0205320F8E52054037003A6
:10CD6000E78008B40103E38002E493200203F68025
:10CD700001F2E5205403B40203A380010908D5F0B1
:10CD8000D9D02022E53012C3E17401932212C3E10D
:10CD9000740293F5F074039385F083F58245F022D5
:10CDA00012C3E1740493F5F074059385F083F58262
:10CDB00045F02212DBF6786B12E092B41820740969
:10CDC00012C3527C0012DFEF796B75F00612DFD1CF
:10CDD00012E13390819112A4B712C27660FB027007
:10CDE00065C0E02582F582E43583F583D0E02256E4
:10CDF00002000012050000241000004820000096E8
:10CE000040000092810000846301006827030074E1
:10CE10000A12AC2612071E12CAD0C224788EE2B4BF
:10CE20004B02D2247984E30912C0A8788FE212B7AA
:10CE3000CC12D60412D27512C8E3E42240C193404A
:10CE4000DF1D40D81580DF2780DF3180DF3B80DFAA
:10CE500045C0DF4F00D76840E18240D0BA00DAE732
:10CE600040DF5940DF6340D9ADC0A8C02075A8801D
:10CE70007989F709E517F709E515F709E520F709B5
:10CE8000E52AF709E582F709E583F77988740DF754
:10CE9000752000029DE2C0E012BC2D7403D5E0FDB8
:10CEA000D296E43096FD209607D5E0F7D0E0D32265
:10CEB0007402D5E0FDC29612BC247401D5E0FDD009
:10CEC000E0C322E7602612D7254021B43200501C6F
:10CED00009E7601812D7254013B41300500E09E774
:10CEE00012D7254007B404004002E422740B2290BC
:10CEF00051B97480C0E0E9C0E0788812DCE078883D
:10CF000075F01812BC9A7891D0E0F912DB23789F63
:10CF100012DB6ED0E0F6120508227982E36005B4D8
:10CF20000500400302AE3612B61315F07420901FB0
:10CF30000012DAB97C0012DFEF75F02012DFDB752A
:10CF4000F02402AE3EC0A8C0D0C0E0C0F0C083C094
:10CF500082E8C0E0E9C0E0C2AF78807401F20874F2
:10CF60000FF20875F00412E089D243C24402AD8D7D
:10CF7000C020D2001475F010901D0012DAB97C00A8
:10CF800012DFEF12B538C0E075F00F30000512DF88
:10CF9000DB800312DFE5D0E0D020229080AF12A426
:10CFA000B712C27660FBB41C0574FFC3800A12DAA4
:10CFB00059400512C7FA80E9C0D0C0E0E412DD1282
:10CFC000D0E0D0D0222401832200303A1B11141863
:10CFD00031323313121734353619201C3738392CB7
:10CFE0000115C28CC28D758CB7758AA8D28C22C0EF
:10CFF00017786B12DDDE751700E5171293B1F9E7AC
:10D00000600B0909E77006786B0912DB410517E52B
:10D0100017B4030040E3D01722C0D0C0E0E520548D
:10D020000CB4C002800E4002801319B4080FB9FF7F
:10D030000C1A80091582E582B4FF021583D0E0D076
:10D04000D022C0205320F175F064846006D20324FE
:10D0500030F608E5F075F00A8470033003042430DC
:10D06000F608E5F02430F608D02022E612D7254055
:10D070001FB42400501A08E612D7254013B46000EC
:10D08000500E08E612D7254007B460005002E42293
:10D09000744022B402059052B5801A50089051FE97
:10D0A000742002CEF4B403059052BE80089052164C
:10D0B000742002CEF4748002CEF4901E007982E3D4
:10D0C000C0E0E4F309D0E01475F01012DAB97C0086
:10D0D00012DFEF75F01012DFDB75F013D24402AEF1
:10D0E0003EC0A875A880790A12A88C64AA6004744E
:10D0F0000A8011786B12C98B796B12CEC3600474ED
:10D100000B8001E4D0A822C020752000C0201204AA
:10D11000CE12D6B112D27512C8E3D0E0700C905086
:10D120003D1204E475F005120C7CD020227A05E54E
:10D13000F07002801CC0F0E8F98AF07B00E7C4546C
:10D140000FCBC7C454F047F709D5F0F1D0F0D5F0B4
:10D15000E4C322C0D0C0E0E520540CB480078AA00C
:10D16000D0E0F380114004D0E0800BB40405D0E09F
:10D17000F38003D0E0F7D0D022C020C20090180086
:10D180007C0012DFEFE9F875F00420000812DFE5FB
:10D1900012D87D800612DFDB12D82AD02022C0D020
:10D1A000C0E0E5205403B4030280074002800FB4BE
:10D1B000020B1582E582B4FF051583800118D0E0CB
:10D1C000D0D022C083C08209E712D7AA75F064A428
:10D1D000F58285F08319E712D7AA12CDE1A682085D
:10D1E000A683D082D08322C0D0C0E0E5205403B40F
:10D1F0000205D0E0F080114004D0E0800BB40105BE
:10D20000D0E0F28003D0E0F6D0D022C0D0E52054A8
:10D210000CB40C04E49380144003E4800FB40805BC
:10D220008AA0E38007B40403E38001E7D0D022148E
:10D2300075F020A42400F582E5F0341FF5837C000E
:10D2400012DFEF741A12CC9712B538B40A004001FD
:10D25000E422787975F00112E1F1787AE6C4540F8E
:10D26000B4050908E6C4540F20E0042250012278D6
:10D270007B12D89122788812DCE0788C76C808740A
:10D28000CDF608F6901C117C0012DFEF799075F056
:10D290001012DFE512050822C0A875A880C020D2B0
:10D2A0004712B762904FD91204E412DF09740D12CD
:10D2B000AC2612071E751704026868C0A875A880FE
:10D2C000C020D24712B7629052791204E412DF09EB
:10D2D000740D12AC2612071E751704026868C02070
:10D2E000752000C0A875A88075F003790212A88C7B
:10D2F000200703F68001F21908D5F0F1D0A8D0205C
:10D3000022C0D0E5205403B40304E4938012400308
:10D31000E4800DB40203E08007B40103E28001E67B
:10D32000D0D022C0D0C0E0E520540CB40C03A380C0
:10D330000F4002800B09B40807B900040A800109F4
:10D34000D0E0D0D02212D20B12D9BF18E64480F61A
:10D35000080912D20B12D9BF18E64480F608091248
:10D36000D20B12D9BF22E8C0E0C0F0C0A8C2AF788B
:10D37000CE75F014E4F208D5F0FAE4F548C22CD0EA
:10D38000A8D0F0D0E0F822C0A8C02078B8E6F520F8
:10D390000854307005E6F902A4BEB41007E6F58221
:10D3A00008E6F58302A4BEB404005003742B22B433
:10D3B0000903742E22B40A03742D22B40B037429BA
:10D3C00022B413E8744422C020C0F0C20075F005F6
:10D3D000E8C0E0E6300001E2700408D5F0F5C8D0FE
:10D3E000E0C8D0F0D02022C0A8C2A912BFB360FB11
:10D3F000C0E0740112E1F6D0E0B4CE0280EDF5F0A9
:10D4000012CFC5D0A82290510A1204E49052387964
:10D410002012C747905240792712C74790522E7961
:10D420001212C74722C0D0C0E0E5205403B4030362
:10D43000A3800B40028007B40203A3800108D0E060
:10D44000D0D022C020C2009018007C0012DFEF75FF
:10D45000F00420000512DFD1800312DFC7D02022A4
:10D4600012D20B12D9BF742DF6080912D20B12D9A1
:10D47000BF742DF6080912D20B12D9BF22C0A8C260
:10D48000A9C0D0C2D5C8C0E0C878CEF2E408F2B8CE
:10D49000E1FBD0E0F8D0D0D0A822C0A875A880C009
:10D4A00020D24712B76212DF09740D12AC261207A0
:10D4B0001E7517050268689003007C0012DFEF7983
:10D4C0008275F02612DFC712E1337982E4F375F03A
:10D4D0000302AE3EE9C0E074002451F582E4340654
:10D4E000F5837C0012DFEFD0E0F975F00712DFDB87
:10D4F00022B400028012B40102800DB4020280083E
:10D50000B403028003B40402E42274012278717926
:10D510006B12BA157873796E12BA15E571C39573EB
:10D52000F571E5729574F57222C0A875A880C0F0F7
:10D530000909780675F003E71298991918D5F0F7DC
:10D54000D0F0D0A822781190AC4175F02612DE4EB2
:10D550007C0090030012DFEF791175F02612DFC70F
:10D5600022C0F0C0E08582F0A4F582E58385F083D7
:10D57000D0F0A42583F583E435F0D0F022E4F52043
:10D58000786B12D2DEAD6BAE6CAF6D129FB3B41878
:10D5900005790512DAD8027065C0A8C02075200090
:10D5A0007D007E227F00740A756B00756C00756DBE
:10D5B00000026121C0F075F000E5F093600CB40D3D
:10D5C00002800705F0E5F070F0D3E5F0D0F022120C
:10D5D000C0076010B43902800BB44202800612A961
:10D5E0004C02706512AA08027065C8C0E0C87812C3
:10D5F000C0F075F003C336F608E4D5F0F9D0F0C8F2
:10D60000D0E0C822201B15742212AC262401F5F0AC
:10D61000120C7C9053141204E4120C7922E8C0E03E
:10D6200078CEE2C8D0E0C87009C0E0740A12D869A8
:10D63000D0E0202CFD227982E4F3099003007C00E5
:10D6400012DFEF75F02612DFDB75F02902AE3EC067
:10D65000205320F8432002C0F08859755B07E91475
:10D66000F55A755C0702A32F75F064842430F60820
:10D67000E5F075F00A842430F608E5F02430F60869
:10D6800022C017E8C0E0780EE2421708B811004047
:10D69000F7D0E0F8E517D017221475F020A4240085
:10D6A000F582E5F0341FF5837C0012DFEF12B53808
:10D6B00022788812DCE07890796B12CA65789B79C1
:10D6C0006E12DE85120508E422B40002800DB40259
:10D6D000028008B403028003B40402E4227401222D
:10D6E000781212E065700578137410F278127917C9
:10D6F00012DE3812D2522212DBF678BC7C077D0291
:10D70000740175F00512DD4278BB7443F622C02027
:10D71000F52053200FE4936009F608A3DCF7D0202E
:10D72000C32202A3F5C0E0540FB40A00500AD0E0AF
:10D73000C0E0C4540FB40A00B3D0E0227D02C2D5C9
:10D740007982E3700204F3B40500400302AE3602AE
:10D75000BD5E7D02C2D57982E3700204F3B4050098
:10D76000400302AE3602BC4EC2AC7882E2F5F01243
:10D770000C7C7882E4F275F003D24402AE3E7E0067
:10D780007F00900000E4932EFEE43FFFA3E5824576
:10D790008370F22275F06484C0E0C5F075F00A84ED
:10D7A000C445F0C5F0D0E0C5F022C0F0C0E0C454DC
:10D7B0000F75F00AA4F5F0D0E0540F25F0D0F02258
:10D7C000C0205320F8C0F08859755B07E914F55A5A
:10D7D000755C0702A32FC0A8C0E0C0F0C2AFE4F59B
:10D7E000F0D5E0FDD0F0D0E0D0A822C0A8C2AFC2F2
:10D7F0008CC28D758CB7758AA8D28CD0A8D2A9227C
:10D80000780875F038E412989908D5F0F8780B7418
:10D81000AA129899227882E4F20812E0A37886127C
:10D82000E0AB75F009D24402AE3EC0F0C0205320F8
:10D83000E843200CD3C0D075F0047D0002BA81C04B
:10D84000F0C0205320F8432018D3C0D075F0047DD9
:10D850000002BA81C0F0C0205320F843201CD3C07E
:10D86000D075F0047D0002BA81C0F075F0E70000C9
:10D8700000000000D5F0F7D5E0F1D0F022C0F0C0F4
:10D88000205320E8D203D3C0D075F0047D0002BA43
:10D8900081C0F0C0205320E8D203D3C0D075F00778
:10D8A0007D0002BA81C0D030D603C39406D0D0C068
:10D8B000D05003C39460D0D022787FE6700C75F00E
:10D8C0000308E67005D5F0F9C322D322F5F0780EEF
:10D8D000E225F0F208E23400F208E23400F22275A8
:10D8E0000F00751022751100751200751322751442
:10D8F00000227882E4F20812E0A3788612E0AB7589
:10D90000F00902AE3ED0E0F9D0E0F8D082D083D06A
:10D91000F0D0E0D0D0D0A822741D12AC26F5287427
:10D920001E12AC2612D794F518E42275F022E410EA
:10D930009808D5E0FAD5F0F7D322E599C3229003F1
:10D94000007C0012DFEF7A2275F00012CC04DAF8C6
:10D9500022C0F075F004C3E49336D4F6A308D5F0E2
:10D96000F6D0F022C020752001200003F68001F2DD
:10D9700008D5F0F5D02022C0E0780EE512F208E5D7
:10D9800013F208E514F2D0E022C0A8C020752000F0
:10D990007D007E227F00740E026121C0A8C0207528
:10D9A00020007D007E227F00740D026121C2AC78D0
:10D9B00082E4F20812B5AB75F02CD24402AE3EC040
:10D9C000E0C4540F2430F608D0E0540F2430F60899
:10D9D00022C0F0E670028007B4200508D5F0F4E418
:10D9E000D0F022C0F075F018C6B42005E608D5F0D6
:10D9F000F7C6D0F022E50F6512700AE510651370C6
:10DA000004E511651422C0A8C2AF532807759870A9
:10DA1000C247D0A8D2AC22C0A875A880C017E4F530
:10DA20000FF510F51102CB41C0205320F8D201C0F0
:10DA3000F08859755B0702A328C0A875A880C0208C
:10DA400053200F43208002C7CBC0A875A880C020F8
:10DA500053200F4320C002C7CBB43B00500AB43060
:10DA6000005002C3229430B322B45100500AB44192
:10DA7000005002C3229440B322C0A8C02075208069
:10DA80007D007E227F00026121C0205320F04320D0
:10DA900004C0F075F00702CBDCEFC39B700122508D
:10DAA0000122F5F07A0502D12FEFC39B70012250BD
:10DAB0000122F5F07A0702D12FC0E0A42582F58279
:10DAC000E5F03583F583D0E02278C27430F6301C5F
:10DAD0000618F6184480F622780275F003E71298CB
:10DAE000991809D5F0F72212D7D67982E4F375F0A8
:10DAF00003D24402AE3E74002582F582E5173583D9
:10DB0000F5837C0022C0207520417C0E7D0275F0DB
:10DB10000702A649C0207520417C0B7D0275F005E7
:10DB200002A3F5C0207520417C0F7D0275F007022D
:10DB3000A3F5C0F0C0205320E075F0077D0502BAC0
:10DB40007EC0F0C0205320E075F0077D0702BA7E4A
:10DB5000C0205320F8C0F08859755B0702A328C085
:10DB600020752000742075F018788802D969C0F0FB
:10DB7000E6B42002800418D5F0F6D0F022C0F0E719
:10DB8000F67420F70809D5F0F6D0F0227882E4F296
:10DB90000812B5AB75F02C02AE3EC0E075F026D58C
:10DBA000E0FDD5F0FAD0E022E8C0E0782FE204F200
:10DBB000C8D0E0C822780EE2F58208E2F58308E2D8
:10DBC000FC22C0A875A880C02053200F02C7CBC07C
:10DBD000E0782E75F04112E089D0E022C0E07811A3
:10DBE00075F01D12E089D0E0227879E608B4500083
:10DBF000400312D8912278BB75F0087420F608D53E
:10DC0000F0F9229006007C0012DFEF7A1602D94864
:10DC10009006007C0012DFEF7A1602D948C0A8C037
:10DC20002075A880752000029DE2C020532000438B
:10DC30002001C0F002CA39C0F0C0205320E04320C8
:10DC40000502BA79C0F0C0205320E043200502DB72
:10DC500039C0F0C0205320E043200502DB48C0F06B
:10DC6000C0205320F043201102BA79C0F0C02053E5
:10DC700020F043201402BA79C0F0C0205320E043C2
:10DC8000201502BA79C0F0C0205320F043201102C1
:10DC9000DB39C0F0C0205320F043201402DB39C030
:10DCA000F0C0205320E043201502DB39C0F0C02033
:10DCB0005320F043201102DB48C0F0C0205320F075
:10DCC00043201402DB48C0F0C0205320E04320155D
:10DCD00002DB48C0205320F0432005C0F002CBDC1B
:10DCE000C020752000742075F01802D969C0E0C406
:10DCF000540F600302D9C402D9C7C017C016C02090
:10DD00007520C002AAC7C017C016C02075208002A7
:10DD1000AAC7C0A8C02075200079BB02A4BEC0203D
:10DD2000C017C03275320702B4CEC0A8C02075201B
:10DD300000740C026121C0A8C020752000740B0281
:10DD4000D5A8C020F52053200FD20602A649C02036
:10DD5000F52053200FD20602D715C020F5205320FE
:10DD60000FD20602A3F5C0F0C0205320E0D200027B
:10DD7000BA79C0F0C0205320E0D20202BA79C0F0D4
:10DD8000C0205320E0D20002DB39C0F0C020532075
:10DD9000E0D20202DB39C0F0C0205320E0D2000202
:10DDA000DB48C0F0C0205320E0D20202DB48C0F0C4
:10DDB000C0205320F0D20402BA79C0F0C020532012
:10DDC000F0D20402DB39C0F0C0205320F0D20402AC
:10DDD000DB48C020C0F0C20075F00702D3D0C020DD
:10DDE000752000E475F00702D969C020752001E4B0
:10DDF00075F00702D9697C047D047E047F027414E7
:10DE000022C020541C4421F520028E3CC0F075F045
:10DE100007A42480D0F022C0205320004320010218
:10DE2000CA34C0205320F043200D02CBD7C020536A
:10DE300020F043200302CBD7C0205320F843200317
:10DE400002A321C3E697F60809E697F61822C02038
:10DE50005320F843200602CD5AC0205320F8432017
:10DE60000502CD5AE4936006F2A308D5F0F622C06D
:10DE70002053200043200802BC9FC02053200043B1
:10DE8000203402CA6AC02053200043203002CA6AEC
:10DE9000C02053200043200402CA6AC0A8C02075D5
:10DEA000201A0298A0C0A8C0207520190298A0C00E
:10DEB000A8C02075201B0298A0C0A8C020752018FB
:10DEC0000298A0C0A8C0207520010298A0C0A8C0D8
:10DED0002075201A02A893C0A8C02075201902A896
:10DEE00093C0A8C02075201802A893C0A8C02075B0
:10DEF000200102A893C0A8C02075203002A4BEC093
:10DF0000A8C02075209002A4BE850F12851013852D
:10DF100011142285120F85131085141122C2AC74BE
:10DF20009A12D47D02D905C2AC749A12D47D02D95A
:10DF300005C2AC749A12D47D02D905C2AC749A128F
:10DF4000D47D02D905C2AC749A12D47D02D905C21F
:10DF5000AC749A12D47D02D905C2AC749A12D47DE5
:10DF600002D905C2AC749A12D47D02D905C0E0E48E
:10DF7000F51AF51BD0E022C020532000C0F002CAE1
:10DF800039C0205320F8D20102A321C0205320F829
:10DF9000D20002A321E627F60809E637F61822C0C8
:10DFA000205320F8D20102CD5AC0205320F8D202CB
:10DFB00002CD5AC0205320F8D20002CD5AC02053BF
:10DFC0002000D20402CA6AC0A8C02075200202B98B
:10DFD000BDC0A8C02075200102B9BDC0A8C0207571
:10DFE000200202B548C0A8C02075200102B54885AE
:10DFF000820C85830D8C0EE422780EE4F208F20880
:10E00000F222C020D207C20602B897851282851379
:10E0100083AC1422901E0075F05002CA13751700CD
:10E0200075155A02594475170075155802594475EB
:10E03000170175155A02594475170575155A025975
:10E0400044751705751558025944C020C0F0D20018
:10E0500002DDD8C020C0F0D20002D3D0C020C0F072
:10E06000C20002D3D0C020C0F0D20002D3CD755B75
:10E0700008755C0B029AD2755B07755C0A029AD22E
:10E0800016E6B4FF0308161822C020752001E4022A
:10E09000D969C031C020C20002B3DB78F1E2781147
:10E0A00002BEB7C02075208002C990C020752080B4
:10E0B00002D2E37980F309E5F0F322C02075205500
:10E0C00002C70FC02075200102D10CC20712011433
:10E0D000027065C207120110027065C2071201B218
:10E0E000027065C02075200102DB0AC02075200186
:10E0F00002DB19C02075200102DB2826F650030838
:10E1000006182206E6700308061822E582F608E5DE
:10E1100083F622E7F58209E7F58322C020E4F520A3
:10E1200002D969C02075200002D96978BB75F00852
:10E1300002DE6FE4F50CF50DF50E22E4F50CF50D9D
:10E14000F50E2275F007A4244C22C020D20002D183
:10E150007DC020D20002D447C020C20702C74BC0F6
:10E1600020D20002B766C020D20702C839C0D0D280
:10E17000D502C27AC020C20002CF74E6700308E65E
:10E180001822901D0002D0BD75820102B46512B242
:10E19000D70270651200B802706575F00702DE598B
:10E1A00075F00502DE5975F00702DFA975F005026A
:10E1B000DFA975F00702DFB375F00502DFB375F074
:10E1C0000702CD550010000000742002CEF47D013E
:10E1D00002BD517D0102BC41D24302AD8DC243025A
:10E1E0009CE1C24302A24A7D0302D73E7D0302D7CF
:10E1F000547A0802D12F02C7FC02C7FAD29022C279
:10E200009022E422E422FFFFFFFFFFFFFFFFFFFF5A
:10E21000FFFFFFFFFFFFFFFFFFFFFFFFFFFFFFFF0E
:10E22000FFFFFFFFFFFFFFFFFFFFFFFFFFFFFFFFFE
:10E23000FFFFFFFFFFFFFFFFFFFFFFFFFFFFFFFFEE
:10E24000FFFFFFFFFFFFFFFFFFFFFFFFFFFFFFFFDE
:00000001FF
